:020000040800F2
:1000000000060020E1010008F90E0008790E000842
:10001000D10E0008790E0008A50E0008E3010008C3
:10002000E3010008E3010008E3010008B927000824
:10003000E3010008E3010008E3010008E301000810
:10004000E3010008E3010008E3010008E301000800
:10005000E3010008E3010008553800088138000872
:10006000AD380008D938000805390008E301000858
:10007000E3010008E3010008E3010008E3010008D0
:10008000E3010008E3010008E3010008E3010008C0
:10009000E3010008E3010008E3010008313900082A
:1000A000E3010008E3010008E3010008E3010008A0
:1000B000C9360008E3010008E3010008E301000875
:1000C000E3010008E3010008E3010008E301000880
:1000D000E3010008510F0008E3010008E3010008F4
:1000E00099390008E3010008E3010008E301000872
:1000F000E3010008E3010008E3010008E301000850
:10010000E3010008E3010008E3010008E30100083F
:10011000E3010008E3010008E3010008E30100082F
:10012000E3010008E3010008E3010008E30100081F
:10013000E3010008E3010008E3010008E30100080F
:10014000E3010008E3010008E3010008F12E0008C4
:10015000E3010008E3010008E3010008E3010008EF
:10016000E3010008E3010008E3010008E3010008DF
:10017000E3010008E3010008E3010008E3010008CF
:10018000E3010008E3010008E3010008E3010008BF
:10019000E3010008E3010008E3010008E3010008AF
:1001A000E3010008E3010008E3010008E30100089F
:1001B000E3010008E3010008E3010008E30100088F
:1001C000E3010008E3010008E3010008E30100087F
:1001D000E3010008E3010008E3010008E30100086F
:1001E00002E000F000F8FEE772B63A4880F30888B3
:1001F000394880F3098839484EF60851CEF200019B
:10020000086040F20000CCF200004EF63471CEF2ED
:1002100000010860BFF34F8FBFF36F8F40F2000003
:10022000C0F2F0004EF68851CEF200010860BFF334
:100230004F8FBFF36F8F4FF00000E1EE100A4EF6C4
:100240003C71CEF200010860062080F31488BFF3F1
:100250006F8F02F031FB02F00DFB03F099F94FF0C4
:1002600055301F491B4A91423CBF41F8040BFAE745
:100270001C49194A91423CBF41F8040BFAE71A495C
:100280001A4A1B4B9A423EBF51F8040B42F8040B2A
:10029000F8E700201749184A91423CBF41F8040B87
:1002A000FAE702F0EBFA03F0C7F9144C144DAC4234
:1002B00003DA54F8041B8847F9E700F041F8114CC1
:1002C000114DAC4203DA54F8041B8847F9E702F0F9
:1002D000D3BA000000060020002200200000000821
:1002E0000000002000060020083E00080022002038
:1002F000402200204022002020300020E0010008A1
:10030000E0010008E0010008E00100082DE9F04FDD
:100310002DED108AC1F80CD0C3689D46BDEC108A43
:10032000BDE8F08F002383F311882846A047002002
:1003300001F04EFEFEE701F0C9FD00DFFEE7000020
:1003400038B502F009FA054602F02CFA0446D8B98D
:100350000F4B9D421AD001339D4218BF044641F213
:10036000883504BF01240025002002F0FFF90CB1FC
:1003700000F056F800F028FD00F0A2FB284600F03F
:10038000A7F800F04DF8F9E70025EDE70546EBE7A3
:10039000010007B008B500F05FFBA0F12003584250
:1003A000584108BD07B541F21203022101A8ADF87A
:1003B000043000F06FFB03B05DF804FB10B52023A0
:1003C00083F311881248C3680BB101F087FE114A0C
:1003D0000F4800234FF47A7101F044FE002383F3A9
:1003E00011880D4C236813B12368013B23606368B7
:1003F00013B16368013B6360084B1B7833B96368D2
:1004000023B9022000F052FC3223636010BD00BF0C
:1004100040220020BD0300085C230020542200205D
:10042000254B264A10B51C461968013142D00433C9
:100430009342F9D16268224B9A423BD9214B9B6887
:1004400003F1006303F580339A4233D2002000F0B9
:1004500051FB1D4B0220187000F018FC1B4B1A6C4E
:1004600000221A64196E1A66196E596C5A64596E14
:100470005A665A6E5A6942F080025A615A6922F0ED
:1004800080025A615A691A6942F000521A611A6967
:1004900022F000521A611B6972B64FF0E02320214E
:1004A000C3F8084DD4E9003281F311889D4683F3E7
:1004B0000888104710BD00BF000001082000010897
:1004C000FFFF0008002200205422002000380240D4
:1004D0002DE9F04F93B0A94B00902022FF210AA8EC
:1004E0009D6800F01BFCA64A1378A3B9A54801211A
:1004F000C3601170202383F31188C3680BB101F02E
:10050000EDFDA14A9F4800234FF47A7101F0AAFD46
:10051000002383F31188009B9C4A03B113609C491C
:10052000009C00230B70536098469B461E469A46DB
:10053000012000F0ABFB24B1944B1B68002B00F0B2
:100540001682002000F088FA0390039B002BF2DB58
:10055000012000F08BFB039B213B162BE8D801A266
:1005600052F823F0C1050008E90500087D060008DF
:1005700031050008310500083105000811070008A1
:10058000E3080008FD0700085F0800088708000866
:10059000AD08000831050008BF0800083105000853
:1005A00031090008610600083105000875090008D6
:1005B000CD05000861060008310500085F08000845
:1005C0000220FFF7E7FE002840F0FB81009B02219C
:1005D000B8F1000F08BF1C4605A841F21233ADF870
:1005E000143000F057FAA3E74FF47A7000F034FAB1
:1005F000071EEBDB0220FFF7CDFE0028E6D0013F0F
:10060000052F00F2E081DFE807F0030A0D10133632
:1006100005230593042105A800F03CFA17E057488C
:100620000421F9E75B480421F6E75B480421F3E77E
:100630004FF01C09484600F05FFA09F104090590E3
:10064000042105A800F026FAB9F12C0FF2D10120FF
:1006500000FA07F747EA0B0B5FFA8BFB4FF0000A33
:1006600000F0A8FB26B10BF00B030B2B08BF0024F6
:10067000FFF798FE5CE749480421CDE7002EA5D09E
:100680000BF00B030B2BA1D10220FFF783FE0746D3
:1006900000289BD001203E4E00F02CFA0220307042
:1006A00000F0F4FA4FF000085FFA88F9484600F0CD
:1006B00031FA044690B1484600F03CFA08F10108CE
:1006C0000028F1D1B846044641F21213022105A8D0
:1006D000ADF814303E4600F0DDF929E70123022091
:1006E000337000F0C3FA2546244B9B68AB4207D910
:1006F000284600F001FA013040F068810435F3E744
:10070000234B00251D70214BB8465D603E46A7E790
:10071000002E3FF45BAF0BF00B030B2B7FF456AFB7
:100720001B4B0220187000F0B1FA322000F094F94F
:10073000B0F10009FFF64AAF19F003077FF446AFA6
:100740000E4A926809EB050393423FF63FAFB9F5B5
:10075000807F3FF73BAF124B0193B94522DD4FF449
:100760007A7000F079F90390039A002AFFF62EAF11
:10077000019B039A03F8012B0137EDE700220020CB
:100780005823002040220020BD0300085C230020E5
:100790005422002004220020082200200C220020E5
:1007A00058220020C820FFF7F5FD074600283FF437
:1007B0000DAF1F2D11D8C5F120024A450AAB25F017
:1007C000030028BF4A4683490192184400F080FA8A
:1007D000019A8048FF2100F0A1FA4FEAA9037D4960
:1007E0000193C9F38702284600F0A0FA06460028C4
:1007F0003FF46AAF019B05EB830531E70220FFF769
:10080000C9FD00283FF4E2AE00F0BEF900283FF435
:10081000DDAE0027B946704B9B68BB4218D91F2F2D
:1008200011D80A9B01330ED027F0030312AA1344F8
:1008300053F8203C05934846042205A900F05EFBCE
:1008400004378146E7E7384600F056F90590F2E7AD
:10085000CDF81490042105A800F01CF900E700234E
:10086000642104A8049300F00BF900287FF4AEAED5
:100870000220FFF78FFD00283FF4A8AE049800F097
:100880006BF90590E6E70023642104A8049300F0C7
:10089000F7F800287FF49AAE0220FFF77BFD0028CE
:1008A0003FF494AE049800F067F9EAE70220FFF7FE
:1008B00071FD00283FF48AAE00F076F9E1E70220EE
:1008C000FFF768FD00283FF481AE05A9142000F071
:1008D00071F904210746049004A800F0DBF83946BA
:1008E000B9E7322000F0B8F8071EFFF66FAEBB077D
:1008F0007FF46CAE384A926807EB0A0393423FF6E6
:1009000065AE0220FFF746FD00283FF45FAE27F0FA
:1009100003075744BA453FF4A3AE504600F0ECF845
:100920000421059005A800F0B5F80AF1040AF1E7E2
:100930004FF47A70FFF72EFD00283FF447AE00F029
:1009400023F9002844D00A9B01330BD008220AA9BE
:10095000002000F0EBF900283AD02022FF210AA85D
:1009600000F0DCF9FFF71EFD1C4801F037FB13B067
:10097000BDE8F08F002E3FF429AE0BF00B030B2BDC
:100980007FF424AE0023642105A8059300F078F8D5
:10099000074600287FF41AAE0220FFF7FBFC8146D1
:1009A00000283FF413AEFFF7FDFC41F2883001F060
:1009B00015FB059800F040FA4E4600F0FBF93C4666
:1009C000B6E506464CE64FF0000AFFE5B8467BE682
:1009D000374679E65822002000220020A086010038
:1009E000F7B5194E0C464FF47A7102FB01F396F9F4
:1009F00000200546501C0BD114480193026829467B
:100A0000176A2246B8478442019B03D1002310E0B5
:100A1000002AF1D096F90020511C01D0012A0DD1F5
:100A20000B4802682946166A2246B047844205D11F
:100A30000123084A0120137003B0F0BD4FF4FA708F
:100A400001F0CCFA0020F7E710220020C827002090
:100A5000A8230020A423002007B50023024601217B
:100A60000DF107008DF80730FFF7BAFF20B19DF8B0
:100A7000070003B05DF804FB4FF0FF30F9E700001A
:100A80000A4608B50421FFF7ABFF80F00100C0B2B1
:100A9000404208BD30B4074B0A461978064B53F85C
:100AA00021402368DD69054B0146AC46204630BC39
:100AB000604700BFA4230020F83A0008A086010088
:100AC00070B501F03BFD094E094D308000242868C7
:100AD0003388834208D901F02BFD2B68044401338D
:100AE000B4F5803F2B60F2D370BD00BFA623002079
:100AF0006423002001F0E4BD00F1006000F58030C7
:100B00000068704700F10060920000F5803001F04D
:100B100063BD0000054B1A68054B1B889B1A834276
:100B200002D9104401F004BD002070476423002066
:100B3000A623002038B5074D04462868204401F05C
:100B4000FFFC28B928682044BDE8384001F010BDFA
:100B500038BD00BF6423002010F003030AD1B0F5B4
:100B6000047F05D200F10050A0F51040D0F8003805
:100B7000184670470023FBE700F10050A0F5104035
:100B8000D0F8100A70470000064991F8243033B1BC
:100B90000023086A81F824300822FFF7B3BF012040
:100BA000704700BF68230020014B1868704700BFE2
:100BB000002004E070B52A4B1B68C3F30B02044607
:100BC0001B0C62B140F21340824230D040F2194017
:100BD00082422ED040F2214082422CD10322214D6C
:100BE0000C2000FB0252556842F20102934224D0CD
:100BF000B3F5805F23D041F20102934221D041F24C
:100C0000030293421FD041F20702934214BF3F23D5
:100C10003123013C0C44013D0A46A24215D215F98C
:100C2000016F501C9EB100F8016C0246F5E70122ED
:100C3000D5E70222D3E70C4DD6E73323E9E741237A
:100C4000E7E75A23E5E75923E3E7104605E02C25BB
:100C50008442157001D9901C5370401A70BD00BFBA
:100C6000002004E0C83A00089C3A0008022804D199
:100C7000054B4FF080429A6170470128FCD1024B2E
:100C80004FF00052F7E700BF00000240022804D1F5
:100C9000054B4FF480429A6170470128FCD1024B0A
:100CA0004FF40052F7E700BF00000240022805D1D0
:100CB000064A536983F48043536170470128FCD18D
:100CC000024A536983F40053F6E700BF0000024074
:100CD00010B50023934203D0CC5CC4540133F9E730
:100CE00010BD000010B5013810F9013F3BB191F97A
:100CF00000409C4203D11AB10131013AF4E71AB124
:100D000091F90020981A10BD1046FCE703460246F0
:100D1000D01A12F9011B0029FAD170470244034688
:100D2000934202D003F8011BFAE770472DE9F8431C
:100D30001F4D144695F824200746884652BBDFF81D
:100D400070909CB395F824302BB92022FF2148469F
:100D50002F62FFF7E3FF95F82400C0F10802A242DA
:100D600028BF2246D6B24146920005EB8000FFF72D
:100D7000AFFF95F82430A41B1E44F6B2082E17448A
:100D80009044E4B285F82460DBD1FFF7FDFE002833
:100D9000D7D108E02B6A03EB82038342CFD0FFF761
:100DA000F3FE0028CBD10020BDE8F8830120FBE74B
:100DB00068230020024B1A78024B1A70704700BF5C
:100DC000A42300201022002038B5154C154D2046D4
:100DD00000F01AFC2946204600F042FC2D6812481B
:100DE0006A6DD2F8043843F00203C2F8043801F007
:100DF000F5F80E49284600F039FD6A6D0C48D2F826
:100E000004380C4923F00203C2F80438A0424FF41E
:100E1000E1330B6003D0BDE8384000F055BB38BD6E
:100E2000C8270020003C000840420F00083C000892
:100E3000A82300209023002038B50B4B1A780B4BC9
:100E400053F822500A4B9D4204460CD0094B002116
:100E500018461422FFF762FF046001462846BDE8E9
:100E6000384000F031BB38BDA4230020F83A000818
:100E7000C82700209023002000B59BB0EFF3098124
:100E800068226846FFF724FFEFF30583044B9A6B53
:100E9000DA6A9A6A9A6A9A6A9A6A9A6A9B6AFEE710
:100EA00000ED00E000B59BB0EFF3098168226846D1
:100EB000FFF70EFFEFF30583044B9A6B9A6A9A6A69
:100EC0009A6A9A6A9A6A9B6AFEE700BF00ED00E0A0
:100ED00000B59BB0EFF3098168226846FFF7F8FE82
:100EE000EFF30583034B5A6B9A6A9A6A9A6A9A6A75
:100EF0009B6AFEE700ED00E0FEE7000030B5094D1B
:100F00000A4491420DD011F8013B5840082340F3A8
:100F10000004013B2C4013F0FF0384EA5000F6D19B
:100F2000EFE730BD2083B8ED024AD36843F0C00339
:100F3000D360704700100140044B5A6810439A6810
:100F400058600AB1181D1047704700BFA823002041
:100F50002DE9F0413C4ED6F85C52EF682B68DA057B
:100F60009CB20CD5202383F311884FF40070FFF757
:100F7000E3FF6FF480732B60002383F31188202339
:100F800083F31188DFF8C08014F02F0339D183F385
:100F90001188380613D5210611D5202383F3118833
:100FA0002A4800F0EFF900284CDA0820FFF7C4FFC8
:100FB0004FF67F733B40EB60002383F311887A0682
:100FC00015D5630613D5202383F31188D6E913239F
:100FD0009A4209D1336C3BB127F040073F041020FF
:100FE0003F0CFFF7A9FFEF60002383F31188D6F8C9
:100FF0006422D3680BB110699847BDE8F04101F055
:101000000FBC230712D014F0080F0CBF0020802063
:10101000E10748BF40F02000A20748BF40F0400071
:10102000630748BF40F48070FFF786FFA4066B6833
:1010300005D596F860124046194000F053FA2C6826
:10104000A4B2A1E76860B7E7A8230020E02300204E
:1010500010B5054C054A0021204600F013FA044B58
:10106000C4F85C3210BD00BFA8230020290F00087F
:101070000010014038B52A4C037C002918BF0C46EB
:10108000012B0546C0F8644210D1264B98420DD181
:10109000254B5A6C42F010025A645A6E42F010020C
:1010A0005A660B2125205B6E00F046F8D5F85C22CD
:1010B0001E4923688A424FEA530003D001F580613C
:1010C0008A422AD11A490144B4F90400B1FBF3F36E
:1010D0000028BEBF23F0070003F0070343EA4003E4
:1010E000A1889360E38843F040031361238943F0B0
:1010F0000103536141F4045343F02C03D36001F422
:10110000A05100231360B1F5806F136853680CBFC2
:101110007F23FF2385F8603238BD0649D3E700BF3F
:10112000003B0008A82300200038024000100140C6
:1011300000BD010580DE800200F1604303F56143DC
:101140000901C9B283F80013012200F01F039A407D
:1011500043099B0003F1604303F56143C3F8802119
:101160001A607047F8B5154682680669AA420B46B0
:10117000816938BF8568761AB54204460BD2184695
:101180002A46FFF7A5FDA3692B44A361A3685B1B57
:10119000A3602846F8BD0CD918463246FFF798FDE3
:1011A000AF1BE1683A463044FFF792FDE3683B44E9
:1011B000EBE718462A46FFF78BFDE368E5E70000FA
:1011C00083689342F7B51546044638BF8568D0E971
:1011D0000460361AB5420BD22A46FFF779FD6369DF
:1011E0002B446361A36828465B1BA36003B0F0BD7A
:1011F0000DD932460191FFF76BFD0199E068AF1BF5
:101200003A463144FFF764FDE3683B44E9E72A4688
:10121000FFF75EFDE368E4E710B50A440024C3610C
:10122000029B8460C0E90000C0E90511C160026151
:10123000036210BD08B5D0E90532934201D182683E
:1012400082B98268013282605A1C42611970D0E909
:1012500004329A4224BFC3684361002100F0DAFEE1
:10126000002008BD4FF0FF30FBE7000070B52023E1
:1012700004460E4683F31188A568A5B1A368A26948
:10128000013BA360531CA36115782269934224BFDC
:10129000E368A361E3690BB120469847002383F319
:1012A0001188284607E03146204600F0A3FE0028BA
:1012B000E2DA85F3118870BD2DE9F74F04460E463A
:1012C00017469846D0F81C904FF0200A8AF31188F0
:1012D0004FF0000B154665B12A4631462046FFF710
:1012E00041FF034660B94146204600F083FE0028D6
:1012F000F1D0002383F31188781B03B0BDE8F08F91
:10130000B9F1000F03D001902046C847019B8BF331
:101310001188ED1A1E448AF31188DCE7C0E9051133
:10132000C160C3611144009B8260C0E9000001619B
:1013300003627047F8B504460D461646202383F332
:101340001188A768A7B1A368013BA36063695A1C11
:1013500062611D70D4E904329A4224BFE36863617C
:10136000E3690BB120469847002080F3118807E01D
:101370003146204600F03EFE0028E2DA87F311886D
:10138000F8BD0000D0E905239A4210B501D182686A
:101390007AB98268013282605A1C82611C780369C2
:1013A0009A4224BFC3688361002100F033FE2046C7
:1013B00010BD4FF0FF30FBE72DE9F74F04460E4616
:1013C00017469846D0F81C904FF0200A8AF31188EF
:1013D0004FF0000B154665B12A4631462046FFF70F
:1013E000EFFE034660B94146204600F003FE0028A8
:1013F000F1D0002383F31188781B03B0BDE8F08F90
:10140000B9F1000F03D001902046C847019B8BF330
:101410001188ED1A1E448AF31188DCE702684368DC
:101420001143016003B11847704700001430FFF703
:1014300043BF00004FF0FF331430FFF73DBF000003
:101440003830FFF7B9BF00004FF0FF333830FFF7F7
:10145000B3BF00001430FFF709BF00004FF0FF31A9
:101460001430FFF703BF00003830FFF763BF000000
:101470004FF0FF323830FFF75DBF000000207047AB
:10148000FFF7E6BD37B515460E4A026000224260FE
:10149000C0E902220122044602740B46009000F1CA
:1014A0005C014FF480721430FFF7B6FE00942B46B7
:1014B0004FF4807204F5AE7104F13800FFF72EFF8F
:1014C00003B030BD143B000810B52023044683F35D
:1014D0001188FFF7CFFD02232374002383F31188C3
:1014E00010BD000038B5C36904460D461BB9042180
:1014F0000844FFF793FF294604F11400FFF79AFE12
:10150000002806DA201D4FF48061BDE83840FFF75F
:1015100085BF38BD026843681143016003B11847B5
:101520007047000013B5446BD4F894341A681178EE
:10153000042915D1217C022912D11979128901239C
:101540008B4013420CD101A904F14C0001F026FF9D
:10155000D4F89444019B21790246206800F0CEF92A
:1015600002B010BD143001F0A9BE00004FF0FF33EF
:10157000143001F0A3BE00004C3001F07BBF00002E
:101580004FF0FF334C3001F075BF0000143001F014
:1015900077BE00004FF0FF31143001F071BE000043
:1015A0004C3001F047BF00004FF0FF324C3001F0EB
:1015B00041BF00000020704710B5D0F894341A687D
:1015C00011780429044617D1017C022914D15979D4
:1015D000528901238B4013420ED1143001F00AFED0
:1015E000024648B1D4F894444FF48073617920687E
:1015F000BDE8104000F070B910BD0000406BFFF76F
:10160000DBBF0000704700007FB5124B0360002372
:101610004360C0E90233012502260F4B05740446DE
:101620000290019300F18402294600964FF48073E2
:10163000143001F0BBFD094B0294CDE9006304F5C1
:1016400023724FF48073294604F14C0001F082FEAE
:1016500004B070BD3C3B0008FD15000825150008CE
:101660000B68202282F311880A7903EB82029061D1
:101670004A79093243F822008A7912B103EB8203D6
:10168000986102230374C0F89414002383F3118833
:101690007047000038B5037F044613B190F854300A
:1016A000ABB9201D01250221FFF734FF04F114001E
:1016B00025776FF0010100F0B9FC84F8545004F173
:1016C0004C006FF00101BDE8384000F0AFBC38BD00
:1016D00010B5012104460430FFF71CFF00232377D7
:1016E00084F8543010BD000038B50446002514308D
:1016F00001F074FD04F14C00257701F043FE201D3C
:1017000084F854500121FFF705FF2046BDE838401A
:10171000FFF752BF90F8443003F06003202B07D14D
:1017200090F84520212A4FF0000303D81F2A06D83D
:1017300000207047222AFBD1C0E90E3303E0034AA0
:1017400082630722C26303640120704711220020D4
:1017500037B5D0F894341A681178042904461AD1A0
:10176000017C022917D11979128901238B40134278
:1017700011D100F14C05284601F0C4FE58B101A971
:10178000284601F00BFED4F89444019B21790246CF
:10179000206800F0B3F803B030BD0000F0B500EBF6
:1017A000810385B09E6904460D46FEB1202383F374
:1017B000118804EB8507301D0821FFF7ABFEFB689D
:1017C0005B691B6806F14C001BB1019001F0F4FD50
:1017D000019803A901F0E2FD024648B1039B2946A6
:1017E000204600F08BF8002383F3118805B0F0BD8C
:1017F000FB685A691268002AF5D01B8A013B134026
:10180000F1D104F14402EAE7093138B550F821403A
:10181000DCB1202383F31188D4F89424136852791F
:1018200003EB8203DB689B695D6845B104216018A6
:10183000FFF770FE294604F1140001F0E5FC204694
:10184000FFF7BAFE002383F3118838BD704700000C
:1018500001F0A8B8012303700023C0E90133C3617C
:1018600083620362C36243620363704738B5044610
:10187000202383F311880025C0E90355C0E90555ED
:10188000416001F09FF80223237085F3118838BD71
:1018900070B500EB810305465069DA600E461446C8
:1018A00018B110220021FFF739FAA06918B11022EF
:1018B0000021FFF733FA31462846BDE8704001F0B9
:1018C0004BB90000826802F0011282600022C0E978
:1018D0000422826101F0CCB9F0B400EB81044789A5
:1018E000E4680125A4698D403D43458123600023C0
:1018F000A2606360F0BC01F0E7B90000F0B400EB57
:1019000081040789E468012564698D403D430581B0
:1019100023600023A2606360F0BC01F061BA0000A4
:1019200070B50223002504460370C0E90255C0E9E2
:101930000455C564856180F8345001F0A9F86368E6
:101940001B6823B129462046BDE87040184770BD8A
:10195000037880F850300523037043681B6810B586
:1019600004460BB1042198470023A36010BD00007A
:1019700090F85020436802701B680BB1052118478E
:101980007047000070B590F83430044613B100235E
:1019900080F8343004F14402204601F08BF963688A
:1019A0009B68B3B994F8443013F0600535D000213A
:1019B000204601F0DDFB0021204601F0CFFB6368EB
:1019C0001B6813B1062120469847062384F834305B
:1019D00070BD204698470028E4D0B4F84A30E26B46
:1019E0009A4288BFE36394F94430E56B002B4FF0D3
:1019F000200380F20381002D00F0F280092284F898
:101A0000342083F311880021D4E90E232046FFF708
:101A100075FF002383F31188DAE794F8452003F07B
:101A20007F0343EA022340F20232934200F0C58072
:101A300021D8B3F5807F48D00DD8012B3FD0022BA1
:101A400000F09380002BB2D104F14C02A263022279
:101A5000E2632364C1E7B3F5817F00F09B80B3F5B7
:101A6000407FA4D194F84630012BA0D1B4F84C307B
:101A700043F0020332E0B3F5006F4DD017D8B3F551
:101A8000A06F31D0A3F5C063012B90D8636894F8A0
:101A900046205E6894F84710B4F848302046B047B6
:101AA000002884D04368A3630368E3631AE0B3F5B6
:101AB000106F36D040F6024293427FF478AF5C4B11
:101AC000A3630223E3630023C3E794F84630012BAA
:101AD0007FF46DAFB4F84C3023F00203C4E90E5527
:101AE000A4F84C30256478E7B4F84430B3F5A06F1F
:101AF0000ED194F8463084F84E30204601F020F89C
:101B000063681B6813B101212046984703232370A3
:101B10000023C4E90E339CE704F14F03A3630123C0
:101B2000C3E72378042B10D1202383F311882046A8
:101B3000FFF7C8FE85F311880321636884F84F50CE
:101B400021701B680BB12046984794F84630002B53
:101B5000DED084F84F300423237063681B68002BA9
:101B6000D6D0022120469847D2E794F848301D0687
:101B700003F00F0120460AD501F08EF8012804D0A9
:101B800002287FF414AF2B4B9AE72B4B98E701F018
:101B900075F8F3E794F84630002B7FF408AF94F81B
:101BA000483013F00F01B3D01A06204602D501F0D9
:101BB000F3FAADE701F0E6FAAAE794F84630002B15
:101BC0007FF4F5AE94F8483013F00F01A0D01B0657
:101BD000204602D501F0CCFA9AE701F0BFFA97E768
:101BE000142284F8342083F311882B462A46294690
:101BF0002046FFF771FE85F31188E9E65DB11522F5
:101C000084F8342083F311880021D4E90E23204680
:101C1000FFF762FEFDE60B2284F8342083F311887F
:101C20002B462A4629462046FFF768FEE3E700BF19
:101C30006C3B0008643B0008683B000838B590F82E
:101C400034300446002B3ED0063BDAB20F2A34D89B
:101C50000F2B32D8DFE803F037313108223231312F
:101C60003131313131313737C56BB0F84A309D42AF
:101C700014D2C3681B8AB5FBF3F203FB12556DB98E
:101C8000202383F311882B462A462946FFF736FE88
:101C900085F311880A2384F834300EE0142384F885
:101CA0003430202383F3118800231A461946204636
:101CB000FFF712FE002383F3118838BD036C03B1D4
:101CC00098470023E7E70021204601F051FA002160
:101CD000204601F043FA63681B6813B106212046D1
:101CE00098470623D7E7000010B590F83430142B3E
:101CF000044629D017D8062B05D001D81BB110BD3A
:101D0000093B022BFBD80021204601F031FA0021CB
:101D1000204601F023FA63681B6813B106212046B0
:101D20009847062319E0152BE9D10B2380F83430AE
:101D3000202383F3118800231A461946FFF7DEFD9E
:101D4000002383F31188DAE7C3689B695B68002B83
:101D5000D5D1036C03B19847002384F83430CEE723
:101D6000024B0022C3E900339A607047102600201E
:101D7000002303748268054B1B6899689142FBD26B
:101D80005A68036042601060586070471026002057
:101D900008B5202383F31188037C032B05D0042B83
:101DA0000DD02BB983F3118808BD436900221A6056
:101DB0004FF0FF334361FFF7DBFF0023F2E7D0E989
:101DC000003213605A60F3E7002303748268054B06
:101DD0001B6899689142FBD85A68036042601060A2
:101DE0005860704710260020054B19690874186860
:101DF00002681A605360186101230374FEF786BA03
:101E00001026002030B54B1C0B4D87B0044610D077
:101E10002B690A4A01A800F025F92046FFF7E4FFE4
:101E2000049B13B101A800F059F92B69586907B058
:101E300030BDFFF7D9FFF8E710260020911D0008FC
:101E400038B50C4D41612B6981689A68914204460E
:101E500003D8BDE83840FFF78BBF1846FFF7B4FF43
:101E600001232C61014623742046BDE83840FEF76B
:101E70004DBA00BF10260020044B1A681B699068F9
:101E80009B68984294BF00200120704710260020D4
:101E900010B5084C236820691A682260546001223A
:101EA00023611A74FFF790FF01462069BDE81040D6
:101EB000FEF72CBA1026002008B5FFF7DDFF18B199
:101EC000BDE80840FFF7E4BF08BD0000FFF7E0BF32
:101ED000FEE7000010B50C4CFFF742FF00F0B4F82D
:101EE0000A498022204600F03BF8012344F8180CF0
:101EF000037400F071FC002383F3118862B6044878
:101F0000BDE8104000F04CB838260020703B0008B7
:101F1000803B000800F01CB9EFF3118020B9EFF30B
:101F20000583202282F311887047000010B530B974
:101F3000EFF30584C4F3080414B180F3118810BDD5
:101F4000FFF7BAFF84F31188F9E70000034A5168EC
:101F500053685B1A9842FBD8704700BF001000E03E
:101F600082600222028270478368A3F17C0243F8F8
:101F70000C2C026943F83C2C426943F8382C074A80
:101F800043F81C2CC26843F8102C022203F8082CDA
:101F9000002203F8072CA3F118007047250300085E
:101FA00010B5202383F31188FFF7DEFF00210446DC
:101FB000FFF746FF002383F31188204610BD000081
:101FC000024B1B6958610F20FFF70EBF102600203F
:101FD000202383F31188FFF7F3BF000008B5014603
:101FE000202383F311880820FFF70CFF002383F3DD
:101FF000118808BD49B1064B42681B6918605A60D8
:10200000136043600420FFF7FDBE4FF0FF307047C0
:10201000102600200368984206D01A6802605060BB
:1020200059611846FFF7A4BE7047000038B5044652
:102030000D462068844200D138BD036823605C608F
:102040004561FFF795FEF4E7054B03F11402C3E980
:1020500005224FF0FF310022C3E90712704700BF8D
:102060001026002070B51C4EC0E9032305460C461F
:1020700001F07AFA334653F8142F9A420DD13062A8
:10208000C5E901242A600A2C2CBF00190A30C6E9D0
:102090000555BDE8704001F055BA316A431AE3189E
:1020A00038BF1C469368A34202D9081901F058FAB8
:1020B00073699A6894420CD85A68AC602B606A6065
:1020C00015609A685D60121B9A604FF0FF33F361F0
:1020D00070BD1B68A41AECE71026002038B51B4C15
:1020E000636998420DD0D0E9003213605A60002233
:1020F0008168C2609A680A449A604FF0FF33E361D6
:1021000038BD2246036842F8143F002193425A60CA
:10211000C16003D1BDE8384001F01CBA9A688168FB
:10212000256A0A449A6001F01FFA63699A68411BA4
:102130008A42E5D9AB181D1A092D206A98BF01F112
:102140000A02BDE83840104401F00ABA1026002007
:102150002DE9F041184C002704F11406656901F0DF
:1021600003FA236AAA68C11A8A4215D81344236263
:10217000D5E9003213605A606369D5F80C80EF60CE
:10218000B34201D101F0E6F987F311882869C0470D
:10219000202383F31188E1E76169B14209D0134438
:1021A0001B1ABDE8F0410A2B2CBFC0180A3001F001
:1021B000D7B9BDE8F08100BF10260020002070478D
:1021C000FEE70000704700004FF0FF30704700004E
:1021D00002290CD0032904D00129074818BF002088
:1021E0007047032A05D8054800EBC2007047044831
:1021F00070470020704700BF643C00082022002088
:10220000183C000870B59AB00546084601A9144666
:1022100000F0C2F801A8FEF779FD431C5B00C5E998
:1022200000340022237003236370C6B201AB023472
:102230001046D1B28E4204F1020401D81AB070BD2A
:1022400013F8011B04F8021C04F8010C0132F0E73A
:1022500008B5202383F311880348FFF779FA002398
:1022600083F3118808BD00BFC827002090F84430D0
:1022700003F01F02012A07D190F845200B2A03D151
:102280000023C0E90E3315E003F06003202B08D1D2
:10229000B0F848302BB990F84520212A03D81F2ADE
:1022A00004D8FFF737BA222AEBD0FAE7034A826351
:1022B0000722C26303640120704700BF1822002078
:1022C00007B5052917D8DFE801F0191603191920F9
:1022D000202383F31188104A01900121FFF7D8FAD7
:1022E00001980E4A0221FFF7D3FA0D48FFF7FCF9D7
:1022F000002383F3118803B05DF804FB202383F3EC
:1023000011880748FFF7C6F9F2E7202383F3118805
:102310000348FFF7DDF9EBE7B83B0008DC3B0008BA
:10232000C827002038B50C4D0C4C0D492A4604F145
:102330000800FFF767FF05F1CA0204F11000094920
:10234000FFF760FF05F5CA7204F118000649BDE801
:102350003840FFF757BF00BF902C002020220020FC
:10236000983B0008A23B0008AD3B000870B504464E
:1023700008460D46FEF7CAFCC6B220460134037873
:102380000BB9184670BD32462946FEF7ABFC002853
:10239000F3D10120F6E700002DE9F84F05460C4681
:1023A000FEF7B4FC2B49C6B22846FFF7DFFF08B1A1
:1023B0000536F6B228492846FFF7D8FF08B110368F
:1023C000F6B2632E0DD8DFF88C80DFF88C90234FA7
:1023D000DFF890A0DFF890B02E7846B92670BDE8FF
:1023E000F88F29462046BDE8F84F01F04FBB252E57
:1023F0002BD1072241462846FEF774FC58B9DBF87A
:1024000000302360DBF804306360DBF80830A36041
:1024100007350C34E0E7082249462846FEF762FCFF
:1024200098B90F4BA21C197809090232C95D02F84C
:10243000041C13F8011B01F00F015345C95D02F89C
:10244000031CF0D118340835C6E704F8016B0135D8
:10245000C2E700BF843C0008AD3B0008993C00087F
:10246000107AFF1F1C7AFF1F8C3C0008BFF34F8FB0
:10247000024AD368DB03FCD4704700BF003C024033
:1024800008B5094B1B7873B9FFF7F0FF074B1A69C2
:10249000002ABFBF064A5A6002F188325A601A68A1
:1024A00022F480621A6008BDEE2E0020003C02403B
:1024B0002301674508B50B4B1B7893B9FFF7D6FF8F
:1024C000094B1A6942F000421A611A6842F48052BC
:1024D0001A601A6822F480521A601A6842F4806204
:1024E0001A6008BDEE2E0020003C02400B28F0B51B
:1024F00016D80C4C0C4923787BB90C4D0E460C2396
:102500004FF0006255F8047B46F8042B013B13F0B2
:10251000FF033A44F6D10123237051F82000F0BDA7
:102520000020FCE7202F0020F02E0020AC3C00080B
:10253000014B53F820007047AC3C00080C2070475A
:102540000B2810B5044601D9002010BDFFF7CEFFBF
:10255000064B53F824301844C21A0BB90120F4E793
:1025600012680132F0D1043BF6E700BFAC3C000832
:102570000B2838B5044628D8FFF7CEFCFFF776FFC6
:10258000FFF77EFF124AF323D360E300DBB243F48C
:10259000007343F002031361136943F48033136142
:1025A00005462046FFF762FFFFF7A0FF094B53F8EF
:1025B000241000F0E9F82846FFF77CFFFFF7B6FC8F
:1025C0002046BDE83840FFF7BBBF002038BD00BF44
:1025D000003C0240AC3C000812F001032DE9F04140
:1025E00005460E4614464BD18218B2F1016F61D8F0
:1025F000314B1B6813F001035CD0304FFFF78CFCAC
:10260000FFF73EFFF323FB60FFF730FF314640F258
:102610000128032C18D824F00104284E0C446D1A0C
:1026200040F20118A142336905EB01072AD123F0DA
:1026300001033361FFF73EFFFFF778FC0120BDE89F
:10264000F081043C0435E4E7AB07E4D13B6923F4B3
:1026500040733B613B6943EA08033B6151F8046BFB
:102660002E60BFF34F8FFFF701FF2B689E42E8D02B
:102670003B6923F001033B61FFF71CFFFFF756FCAA
:102680000020DCE723F440733361336943EA080335
:1026900033610B883B80BFF34F8FFFF7E7FE3F8826
:1026A00031F8023BBFB2BB42BCD0336923F0010317
:1026B0003361E1E71846C2E700380240003C0240BF
:1026C000084908B50B7828B11BB9FFF7D9FE0123DB
:1026D0000B7008BD002BFCD0BDE808400870FFF768
:1026E000E9BE00BFEE2E002010B50244064BD2B268
:1026F000904200D110BD441C00B253F8200041F8B4
:10270000040BE0B2F4E700BF502800400F4B30B597
:102710001C6F240407D41C6F44F400741C671C6FE6
:1027200044F400441C670A4C236843F4807323601C
:102730000244084BD2B2904200D130BD441C00B2DA
:1027400051F8045B43F82050E0B2F4E7003802404F
:10275000007000405028004007B5012201A9002068
:10276000FFF7C2FF019803B05DF804FB13B5044600
:10277000FFF7F2FFA04205D0012201A90020019439
:10278000FFF7C4FF02B010BD70470000034B1A688A
:102790001AB9034AD2F874281A607047242F00200F
:1027A0000030024008B5FFF7F1FF024B1868C0F394
:1027B000407008BD242F0020EFF3098305494A6BC0
:1027C00022F001024A63683383F30988002383F30C
:1027D0001188704700EF00E0202080F3118862B676
:1027E0000C4B0D4AD96821F4E0610904090C0A4335
:1027F000DA60D3F8FC20094942F08072C3F8FC206B
:102800000A6842F001020A601022DA7783F8220097
:10281000704700BF00ED00E00003FA05001000E083
:1028200010B5202383F311880E4B5B6813F400630B
:1028300014D0F1EE103AEFF30984683C4FF0807346
:10284000E361094BDB6B236684F30988FFF714FB14
:1028500010B1064BA36110BD054BFBE783F3118854
:10286000F9E700BF00ED00E000EF00E037030008EB
:102870003A03000870470000FEE700000A4B0B48CF
:102880000B4A90420BD30B4BDA1C121AC11E22F0DA
:1028900003028B4238BF00220021FEF73FBA53F8F3
:1028A000041B40F8041BECE7483E000820300020E1
:1028B00020300020203000207047000070B5D0E9A3
:1028C00015439E6800224FF0FF3504EB421351017F
:1028D000D3F800090028BEBFD3F8000940F08040BB
:1028E000C3F80009D3F8000B0028BEBFD3F8000BD3
:1028F00040F08040C3F8000B013263189642C3F8E1
:102900000859C3F8085BE0D24FF00113C4F81C3833
:1029100070BD00001D4B03EB80022DE9F043D2F89F
:102920000CC05D6DDCF81420461CD2F800E005EB0D
:10293000063605EB4018516871450AD3D5F834388E
:10294000012202FA00F023EA0000C5F83408BDE8CD
:10295000F083BCF81040AEEB0103A34228BF23462E
:10296000D8F81849A4B2B3EB840FF0D89468A4F156
:10297000040959F8047F3760A4EB09071F44042FAA
:10298000F7D81C440B4494605360D4E7282F0020F0
:10299000890141F02001016103699B06FCD41220EA
:1029A000FFF7D4BA10B5054C2046FEF753FF4FF0A1
:1029B000A0436365024BA36510BD00BF282F002014
:1029C000003D000870B50378012B054650D12A4B15
:1029D000446D98421BD1294B5A6B42F080025A63D6
:1029E0005A6D42F080025A655A6D5A6942F080026F
:1029F0005A615A6922F080025A610E2143205B69B4
:102A0000FEF79AFB1E4BE3601E4BC4F80038002310
:102A1000C4F8003EC02323606E6D4FF40413A3631B
:102A20003369002BFCDA012333610C20FFF78EFAA7
:102A30003369DB07FCD41220FFF788FA3369002BD7
:102A4000FCDA0026A6602846FFF738FF6B68C4F85A
:102A50001068DB68C4F81468C4F81C684BB90A4BEA
:102A6000A3614FF0FF336361A36843F00103A360E8
:102A700070BD064BF4E700BF282F0020003802404D
:102A80004014004003002002003C30C0083C30C02D
:102A9000F8B5446D054600212046FFF779FFA96D82
:102AA00000234FF001128F68C4F834384FF00066ED
:102AB000C4F81C284FF0FF3004EB431201339F424F
:102AC000C2F80069C2F8006BC2F80809C2F8080B26
:102AD000F2D20B686A6DEB656362102313611669AD
:102AE00016F01006FBD11220FFF730FAD4F80038A8
:102AF00023F4FE63C4F80038A36943F4402343F091
:102B00001003A3610923C4F81038C4F814380A4B21
:102B1000EB604FF0C043C4F8103B084BC4F8003BD7
:102B2000C4F81069C4F80039EB6D03F1100243F4E6
:102B30008013EA65A362F8BDDC3C00084080001009
:102B4000426D90F84E10D2F8003823F4FE6343EA49
:102B50000113C2F8003870472DE9F84300EB8103F8
:102B6000456DDA68166806F00306731E022B05EB46
:102B700041130C4680460FFA81F94FEA41104FF09D
:102B80000001C3F8101B4FF0010104F1100398BFBE
:102B9000B60401FA03F391698EBF334E06F18056F5
:102BA00006F5004600293AD0578A04F15801490138
:102BB00037436F50D5F81C180B43C5F81C382B1839
:102BC0000021C3F8101953690127611EA7409BB368
:102BD000138A928B9B08012A88BF5343D8F85C2044
:102BE000981842EA034301F1400205EB8202C8F85B
:102BF0005C00214653602846FFF7CAFE08EB8900B7
:102C0000C3681B8A43EA8453483464011E432E512F
:102C1000D5F81C381F43C5F81C78BDE8F88305EBD0
:102C20004917D7F8001B21F40041C7F8001BD5F85D
:102C30001C1821EA0303C0E704F13F0305EB8303FB
:102C40000A4A5A6028462146FFF7A2FE05EB4910C2
:102C5000D0F8003923F40043C0F80039D5F81C3807
:102C600023EA0707D7E700BF008000100004000236
:102C7000826D1268C265FFF721BE00005831436DB6
:102C800049015B5813F4004004D013F4001F0CBF3B
:102C900002200120704700004831436D49015B5814
:102CA00013F4004004D013F4001F0CBF02200120D5
:102CB0007047000000EB8101CB68196A0B68136054
:102CC0004B6853607047000000EB810330B5DD684E
:102CD000AA691368D36019B9402B84BF40231360DD
:102CE0006B8A1468426D1C44013CB4FBF3F46343EB
:102CF000033323F0030302EB411043EAC44343F0E0
:102D0000C043C0F8103B2B6803F00303012B09B24A
:102D10000ED1D2F8083802EB411013F4807FD0F8BE
:102D2000003B14BF43F0805343F00053C0F8003B16
:102D300002EB4112D2F8003B43F00443C2F8003BDF
:102D400030BD00002DE9F041244D6E6D06EB4013BF
:102D50000446D3F8087BC3F8087B38070AD5D6F8B1
:102D60001438190706D505EB84032146DB6828468D
:102D70005B689847FA071FD5D6F81438DB071BD5D0
:102D800005EB8403D968CCB98B69488A5A68B2FBD1
:102D9000F0F600FB16228AB91868DA6890420DD264
:102DA000121AC3E90024202383F311880B4821461B
:102DB000FFF78AFF84F31188BDE8F081012303FA4D
:102DC00004F26B8923EA02036B81CB68002BF3D0FA
:102DD00021460248BDE8F041184700BF282F0020D7
:102DE00000EB810370B5DD68436D6C692668E660B1
:102DF0004A0156BB1A444FF40020C2F810092A6851
:102E000002F00302012A0AB20ED1D3F8080803EB3C
:102E1000421410F4807FD4F8000914BF40F08050B1
:102E200040F00050C4F8000903EB4212D2F8000948
:102E300040F00440C2F80009D3F83408012202FA35
:102E400001F10143C3F8341870BD19B9402E84BF95
:102E50004020206020682E8A8419013CB4FBF6F4DF
:102E600040EAC44040F000501A44C6E7F8B50446B2
:102E70001E48456D05EB4413D3F80869C3F808698B
:102E8000F10717D5D5F81038DA0713D500EB84030E
:102E9000D9684B691F68DA68974218D2D21B00279D
:102EA0001A605F60202383F311882146FFF798FFA3
:102EB00087F31188330617D5D5F834280123A340AA
:102EC000134211D02046BDE8F840FFF723BD01238F
:102ED00003FA04F2038923EA020303818B68002BBF
:102EE000E8D021469847E5E7F8BD00BF282F00202D
:102EF0002DE9F74F984C666D7569B3691D4015F45F
:102F00008058756107D02046FEF70AFD03B0BDE882
:102F1000F04FFFF785BC002D12DAD6F8003E8E4840
:102F20009F071EBFD6F8003E23F00303C6F8003EFD
:102F3000D6F8043823F00103C6F80438FEF718FD6C
:102F4000280505D58448FFF7B9FC8348FEF700FD46
:102F5000A9040CD5D6F8083813F0060FF36823F44B
:102F600070530CBF43F4105343F4A053F3602A078B
:102F700004D56368DB680BB177489847EB0274D4DB
:102F8000AF0227D5D4F85490DFF8CCB100274FF02A
:102F9000010A09EB4712D2F8003B03F44023B3F5D2
:102FA000802F11D1D2F8003B002B0DDA62890AFA8A
:102FB00007F322EA0303638104EB8703DB68DB6822
:102FC00013B1394658469847A36D01379B68FFB245
:102FD0009F42DED9E80617D5676D3A6AC2F30A1038
:102FE00002F00F0302F4F012B2F5802F00F0888097
:102FF000B2F5402F08D104EB83030022DB681B6A83
:1030000007F5805790426DD12903D6F8184813D59B
:10301000E20302D50020FFF795FEA30302D50120AD
:10302000FFF790FE670302D50220FFF78BFE260311
:1030300002D50320FFF786FE6D037FF567AFE0073B
:1030400002D50020FFF712FFA10702D50120FFF7EC
:103050000DFF620702D50220FFF708FF23077FF567
:1030600055AF0320FFF702FF50E7636DDFF8E8B0CC
:10307000019300274FF0010AA36D9B685FFA87F95F
:1030800099453FF67DAF019B03EB4913D3F8002927
:1030900002F44022B2F5802F22D1D3F80029002A71
:1030A0001EDAD3F8002942F09042C3F80029D3F881
:1030B0000029002AFBDB606D4946FFF769FC228985
:1030C0000AFA09F322EA0303238104EB8903DB688C
:1030D0009B6813B14946584698474846FFF71AFC83
:1030E0000137C9E7910708BFD7F80080072A98BFC2
:1030F00003F8018B02F1010298BF4FEA182881E71B
:10310000023304EB830207F580575268D2F818C0E7
:10311000DCF80820DCE9001CA1EB0C0C0021884243
:103120000AD104EB830463689B699A6802449A603D
:103130005A6802445A6067E711F0030F08BFD7F8D6
:1031400000808C4588BF02F8018B01F1010188BF26
:103150004FEA1828E3E700BF282F0020436D03EB58
:103160004111D1F8003B43F40013C1F8003B704714
:10317000436D03EB4111D1F8003943F40013C1F85A
:1031800000397047436D03EB4111D1F8003B23F444
:103190000013C1F8003B7047436D03EB4111D1F8B8
:1031A000003923F40013C1F80039704730B5039C8F
:1031B0000172043304FB0325C0E90653049B036337
:1031C0000021059BC160C0E90000C0E90422C0E9FC
:1031D0000842C0E90A11436330BD0000416A002281
:1031E000C0E90411C0E90A22C2606FF00101FEF7D4
:1031F0001DBF0000D0E90432934201D1C2680AB970
:10320000181D70470020704703691960C2680132B9
:10321000C260C269134482690361934224BF436A56
:1032200003610021FEF7F6BE38B504460D46E3689B
:103230003BB16269131D1268A3621344E36200206C
:1032400007E0237A33B929462046FEF7D3FE00284B
:10325000EDDA38BD6FF00100FBE70000C368C2691A
:10326000013BC3604369134482694361934224BFB5
:10327000436A436100238362036B03B118477047BD
:1032800070B52023044683F31188866A3EB9FFF7A0
:10329000CBFF054618B186F31188284670BDA36A96
:1032A000E26A13F8015BA362934202D32046FFF760
:1032B000D5FF002383F31188EFE700002DE9F84FD5
:1032C00004460E46174698464FF0200989F31188A8
:1032D0000025AA46D4F828B0BBF1000F09D1414619
:1032E0002046FFF7A1FF20B18BF311882846BDE8E7
:1032F000F88FD4E90A12A7EB050B521A934528BFA1
:103300009346BBF1400F1BD9334601F1400251F8FF
:10331000040B43F8040B9142F9D1A36A40334036C1
:10332000A3624035D4E90A239A4202D32046FFF72C
:1033300095FF8AF31188BD42D8D289F31188C9E775
:1033400030465A46FDF7C4FCA36A5B445E44A36260
:103350005D44E7E710B5029C0172043304FB0321CE
:10336000C0E906130023C0E90A33039B0363049BEF
:10337000C460C0E90000C0E90422C0E90842436318
:1033800010BD0000026AC260426AC0E90422002245
:10339000C0E90A226FF00101FEF748BED0E904231C
:1033A0009A4201D1C26822B9184650F8043B0B601A
:1033B0007047002070470000C368C2690133C360D2
:1033C0004369134482694361934224BF436A436162
:1033D0000021FEF71FBE000038B504460D46E36825
:1033E0003BB123691A1DA262E2691344E362002023
:1033F00007E0237A33B929462046FEF7FBFD002873
:10340000EDDA38BD6FF00100FBE7000003691960D9
:10341000C268013AC260C26913448269036193427F
:1034200024BF436A036100238362036B03B118471F
:103430007047000070B520230D460446114683F303
:103440001188866A2EB9FFF7C7FF10B186F311887D
:1034500070BDA36A1D70A36AE26A01339342A3623E
:1034600004D3E16920460439FFF7D0FF002080F340
:103470001188EDE72DE9F84F04460D469046994630
:103480004FF0200A8AF311880026B346A76A4FB985
:1034900049462046FFF7A0FF20B187F31188304648
:1034A000BDE8F88FD4E90A073A1AA8EB0607974255
:1034B00028BF1746402F1BD905F1400355F8042BB0
:1034C00040F8042B9D42F9D1A36A4033A3624036F1
:1034D000D4E90A239A4204D3E16920460439FFF76C
:1034E00095FF8BF311884645D9D28AF31188CDE731
:1034F00029463A46FDF7ECFBA36A3B443D44A362F0
:103500003E44E5E7D0E904239A4217D1C3689BB152
:10351000836A8BB1043B9B1A0ED01360C368013BD6
:10352000C360C3691A44836902619A4224BF436A33
:103530000361002383620123184670470023FBE7E1
:1035400000F088B84FF08043002258631A610222CD
:10355000DA6070474FF080430022DA607047000065
:103560004FF08043586370474FF08043586A70476C
:103570004B6843608B688360CB68C3600B694361B1
:103580004B6903628B6943620B68036070470000FC
:1035900008B5264B26481A6940F2FF110A431A6102
:1035A0001A6922F4FF7222F001021A611A691A6B79
:1035B0000A431A631A6D0A431A651E4A1B6D1146A7
:1035C000FFF7D6FF02F11C0100F58060FFF7D0FF86
:1035D00002F1380100F58060FFF7CAFF02F15401E3
:1035E00000F58060FFF7C4FF02F1700100F5806014
:1035F000FFF7BEFF02F18C0100F58060FFF7B8FF16
:1036000002F1A80100F58060FFF7B2FF02F1C401EA
:1036100000F58060FFF7ACFF02F1E00100F580608B
:10362000FFF7A6FFBDE8084000F09AB80038024056
:10363000000002400C3D000808B500F007FAFEF754
:1036400049FCFFF7A3F8BDE80840FEF76BBE000099
:1036500070470000104B1A6C42F001021A641A6E97
:1036600042F001021A660D4A1B6E936843F0010393
:1036700093604FF0804353229A624FF0FF32DA6238
:1036800000229A615A63DA605A6001225A61082165
:103690001A601C20FDF750BD00380240002004E0F5
:1036A0004FF0804208B51169D3680B40D9B2C943C5
:1036B0009B07116107D5202383F31188FEF72AFCAD
:1036C000002383F3118808BD08B5FFF7E9FFBDE8C3
:1036D0000840FFF7A5B800001F4B1A696FEAC252F5
:1036E0006FEAD2521A611A69C2F308021A614FF0E6
:1036F000FF301A695A69586100215A6959615A693B
:103700001A6A62F080521A621A6A02F080521A62D1
:103710001A6A5A6A58625A6A59625A6A1A6C42F0AC
:1037200080521A641A6E42F080521A661A6E0B4A60
:10373000106840F480701060186F00F44070B0F5AD
:10374000007F1EBF4FF4803018671967536823F459
:103750000073536000F05AB9003802400070004016
:10376000334B4FF080521A64324A4FF4404111609B
:103770001A6842F001021A601A689107FCD59A682B
:1037800022F003029A602A4B9A6812F00C02FBD1D5
:10379000196801F0F90119609A601A6842F48032E0
:1037A0001A601A689203FCD55A6F42F001025A67F8
:1037B0001F4B5A6F9007FCD51F4A5A601A6842F097
:1037C00080721A601B4A53685904FCD5184B1A685A
:1037D0009201FCD5194A9A60194B1A68194B9A4202
:1037E000194B21D1194A1168194A91421CD140F252
:1037F00005121A60144A136803F00F03052BFAD15F
:103800000B4B9A6842F002029A609A6802F00C022E
:10381000082AFAD15A6C42F480425A645A6E42F431
:1038200080425A665B6E704740F20572E1E700BF66
:103830000038024000700040085440070094883867
:10384000002004E011640020003C024000ED00E094
:1038500041C20F41084A08B5516913680B4003F093
:103860000103536123B1054A13680BB150689847AF
:10387000BDE80840FEF7D4BF003C0140A02F002067
:10388000084A08B5516913680B4003F002035361FD
:1038900023B1054A93680BB1D0689847BDE808404A
:1038A000FEF7BEBF003C0140A02F0020084A08B52B
:1038B000516913680B4003F00403536123B1054AB7
:1038C00013690BB150699847BDE80840FEF7A8BFDF
:1038D000003C0140A02F0020084A08B55169136838
:1038E0000B4003F00803536123B1054A93690BB100
:1038F000D0699847BDE80840FEF792BF003C014000
:10390000A02F0020084A08B5516913680B4003F046
:103910001003536123B1054A136A0BB1506A9847EB
:10392000BDE80840FEF77CBF003C0140A02F00200E
:10393000174B10B55A691C68144004F478725A6128
:10394000A30604D5134A936A0BB1D06A9847600660
:1039500004D5104A136B0BB1506B9847210604D560
:103960000C4A936B0BB1D06B9847E20504D5094A1A
:10397000136C0BB1506C9847A30504D5054A936CA2
:103980000BB1D06C9847BDE81040FEF749BF00BFAF
:10399000003C0140A02F00201A4B10B55A691C684A
:1039A000144004F47C425A61620504D5164A136D32
:1039B0000BB1506D9847230504D5134A936D0BB195
:1039C000D06D9847E00404D50F4A136E0BB1506ECA
:1039D0009847A10404D50C4A936E0BB1D06E98475A
:1039E000620404D5084A136F0BB1506F9847230443
:1039F00004D5054A936F0BB1D06F9847BDE81040CE
:103A0000FEF70EBF003C0140A02F0020062108B5A4
:103A10000846FDF791FB06210720FDF78DFB0621E7
:103A20000820FDF789FB06210920FDF785FB06210B
:103A30000A20FDF781FB06211720FDF77DFBBDE87D
:103A4000084006212820FDF777BB000008B5FFF7E6
:103A500043FE00F00DF8FDF713FDFDF7F9FEFDF74D
:103A6000D1FDFFF7F5FDBDE80840FFF769BD000097
:103A70000023054A19460133102BC2E9001102F157
:103A80000802F8D1704700BFA02F0020034611F8AC
:103A9000012B03F8012B002AF9D1704753544D3301
:103AA00032463F3F3F00000053544D3332463430DE
:103AB000780053544D3332463432780053544D33EA
:103AC0003246343436585800000000009C3A000852
:103AD0003F00000013040000A83A00083F00000067
:103AE00019040000B23A00083F0000002104000061
:103AF000BC3A00083F000000C8270020A82300208F
:103B0000009600000000000000000000000000001F
:103B100000000000000000004914000835140008EF
:103B2000711400085D140008691400085514000899
:103B3000411400082D1400087D1400080000000046
:103B4000811500086D150008A915000895150008D5
:103B5000A11500088D1500087915000865150008E5
:103B6000B515000800000000010000000000000082
:103B70006D61696E0000000069646C650000000002
:103B8000783B000850260020C827002001000000D4
:103B9000D11E0008000000004172647550696C6F0E
:103BA000740025424F415244252D424C0025534577
:103BB0005249414C250000000200000000000000B6
:103BC0009D1700080918000840004000602C0020E4
:103BD000702C002002000000000000000300000024
:103BE000000000004D180008000000001000000058
:103BF000802C0020000000000100000000000000F8
:103C0000282F002001010200C1220008D121000854
:103C10006D2200085122000843000000203C0008EB
:103C200009024300020100C032090400000102023F
:103C300001000524001001052401000104240202F2
:103C40000524060001070582030800FF090401009E
:103C5000020A00000007050102400000070581027A
:103C600040000000120000006C3C0008120110012E
:103C70000200004009124157000201020301000046
:103C80000403090425424F41524425004D617465E7
:103C90006B463430352D54450030313233343536AF
:103CA0003738394142434445460000000040000097
:103CB0000040000000400000004000000000010043
:103CC00000000200000002000000020000000200EC
:103CD00000000200000002000000020000000000DE
:103CE000851900083D1C0008E91C00084000400040
:103CF000882F0020882F002001000000982F00202E
:103D00008000000040010000030000000001A81630
:103D100000000000AAAAAAAA00001400EF9F000059
:103D20000000000070A70A0000040001000000006D
:103D3000AAAAAAAA00000001DFFF000000000000FC
:103D4000000000000400001400000000AAAAAAAAB3
:103D500004000014FFFF000000000000000000004D
:103D60000000000000000000AAAAAAAA00000000AB
:103D7000FFFF000000000000000000000000000045
:103D800000000000AAAAAAAA00000000FFFF00008D
:103D90000000000000000000000000000000000023
:103DA000AAAAAAAA00000000FFFF0000000000006D
:103DB000000000000000000000000000AAAAAAAA5B
:103DC00000000000FFFF00000000000000000000F5
:103DD00000000000000000000A00000000000000D9
:103DE00003000000000000000000000000000000D0
:103DF00000000000000000000000000000000000C3
:103E000000000000000000001E0400000000000090
:103E100000000F0000000000FF00960000000008F6
:103E2000009600000000080004000000803C00082C
:103E30000000000000000000000000000000000082
:103E40000000000000000000FFFFFFFFFFFFFFFF7A
:103E5000FFFFFFFFFFFFFFFFFFFFFFFFFFFFFFFF72
:103E6000FFFFFFFFFFFFFFFFFFFFFFFFFFFFFFFF62
:103E7000FFFFFFFFFFFFFFFFFFFFFFFFFFFFFFFF52
:103E8000FFFFFFFFFFFFFFFFFFFFFFFFFFFFFFFF42
:020000040801F1
:1000000000060020B5120108C55109082151090850
:100010008D5109082151090859510908B7120108E1
:10002000B7120108B7120108B7120108DDB00B08BA
:10003000B7120108B7120108B7120108B712010878
:10004000B7120108B7120108B7120108B712010868
:10005000B7120108B712010875BC0B089DBC0B084C
:10006000C5BC0B08EDBC0B0815BD0B08AD5F0B083C
:10007000D55F0B0801600B082D600B0859600B0859
:1000800081600B08AD600B08315F0B08B7120108E7
:10009000B7120108B7120108B71201083DBD0B08DD
:1000A00089BE0B089DBE0B08B1BE0B08C5BE0B0870
:1000B000C9BE0B08DDBE0B08F1BE0B0839660B0884
:1000C000E1670B08B7120108B7120108B71201085F
:1000D000B712010811BE0B0825BE0B0839BE0B086C
:1000E000A1BD0B08B7120108B712010815BF0B0814
:1000F00029BF0B0849BF0B084DBF0B08D9600B087F
:10010000B7120108B712010805BF0B08B7120108A2
:100110004DBE0B0861BE0B08B7120108B7120108EB
:1001200005610B082D610B0859610B0885610B08EF
:10013000B1610B08B7120108B7120108B712010824
:10014000B7120108B7120108B712010809B80B0865
:10015000D9610B0805620B0831620B0875BE0B08EC
:10016000B7120108B7120108B7120108B712010847
:10017000B7120108B7120108B7120108B712010837
:10018000B7120108B7120108B7120108B712010827
:10019000B7120108B7120108B7120108B712010817
:1001A000B7120108B7120108B7120108B712010807
:1001B000B7120108B7120108B7120108B7120108F7
:1001C000B7120108B7120108B7120108B7120108E7
:1001D000B7120108B7120108B7120108B7120108D7
:1001E00035580108318502089DF3030815AE05084E
:1001F00039B40508ED120608997606085D7E0608F2
:1002000095810608F5E60608110E070885E307083C
:10021000753E0808CD4B08086143090845480908A0
:100220002D410A08A59C0A08FDC20A08E9CE0A0861
:1002300089FE0A08B5040B08000000000000000059
:1002400081F0004102E000BF83F0004330B54FEA87
:1002500041044FEA430594EA050F08BF90EA020FF4
:100260001FBF54EA000C55EA020C7FEA645C7FEA87
:10027000655C00F0E2804FEA5454D4EB5555B8BFAA
:100280006D420CDD2C4480EA020281EA030382EA1B
:10029000000083EA010180EA020281EA0303362DAD
:1002A00088BF30BD11F0004F4FEA01314FF4801C80
:1002B0004CEA113102D0404261EB410113F0004F92
:1002C0004FEA03334CEA133302D0524263EB430349
:1002D00094EA050F00F0A780A4F10104D5F1200EE7
:1002E0000DDB02FA0EFC22FA05F2801841F1000142
:1002F00003FA0EF2801843FA05F359410EE0A5F116
:1003000020050EF1200E012A03FA0EFC28BF4CF046
:10031000020C43FA05F3C01851EBE37101F00045FC
:1003200007D54FF0000EDCF1000C7EEB00006EEB09
:100330000101B1F5801F1BD3B1F5001F0CD3490893
:100340005FEA30004FEA3C0C04F101044FEA4452EA
:1003500012F5800F80F09A80BCF1004F08BF5FEA71
:10036000500C50F1000041EB045141EA050130BD51
:100370005FEA4C0C404141EB0101013C28BFB1F563
:10038000801FE9D291F0000F04BF01460020B1FAAE
:1003900081F308BF2033A3F10B03B3F120020CDA81
:1003A0000C3208DD02F1140CC2F10C0201FA0CF05F
:1003B00021FA02F10CE002F11402D8BFC2F1200CC4
:1003C00001FA02F120FA0CFCDCBF41EA0C0190407A
:1003D000E41AA2BF01EB0451294330BD6FEA0404C3
:1003E0001F3C1CDA0C340EDC04F11404C4F12002AE
:1003F00020FA04F001FA02F340EA030021FA04F3C0
:1004000045EA030130BDC4F10C04C4F1200220FA16
:1004100002F001FA04F340EA0300294630BD21FA54
:1004200004F0294630BD94F0000F83F4801306BF1A
:1004300081F480110134013D4EE77FEA645C18BF0E
:100440007FEA655C29D094EA050F08BF90EA020FA5
:1004500005D054EA000C04BF1946104630BD91EA9D
:10046000030F1EBF0021002030BD5FEA545C05D1A0
:100470004000494128BF41F0004130BD14F58004DF
:100480003CBF01F5801130BD01F0004545F0FE4153
:1004900041F470014FF0000030BD7FEA645C1ABF88
:1004A000194610467FEA655C1CBF0B46024650EABF
:1004B000013406BF52EA033591EA030F41F40021EB
:1004C00030BD00BF90F0000F04BF0021704730B571
:1004D0004FF4806404F132044FF000054FF0000146
:1004E00050E700BF90F0000F04BF0021704730B507
:1004F0004FF4806404F1320410F0004548BF4042DC
:100500004FF000013EE700BF42004FEAE2014FEA30
:1005100031014FEA02701FBF12F07F4393F07F4F0B
:1005200081F06051704732F07F4208BF704793F00E
:100530007F4F04BF41F40021704730B54FF4607421
:1005400001F0004521F000411CE700BF50EA010224
:1005500008BF704730B54FF000050AE050EA0102CD
:1005600008BF704730B511F0004502D5404261EB3D
:1005700041014FF4806404F132045FEA915C3FF47E
:10058000D8AE4FF003025FEADC0C18BF03325FEA1B
:10059000DC0C18BF033202EBDC02C2F1200300FACC
:1005A00003FC20FA02F001FA03FE40EA0E0021FAF1
:1005B00002F11444BDE600BF70B54FF0FF0C4CF4DF
:1005C000E06C1CEA11541DBF1CEA135594EA0C0F91
:1005D00095EA0C0F00F0DEF82C4481EA030621EACC
:1005E0004C5123EA4C5350EA013518BF52EA033507
:1005F00041F4801143F4801338D0A0FB02CE4FF0B9
:100600000005E1FB02E506F00042E0FB03E54FF0E8
:100610000006E1FB03569CF0000F18BF4EF0010EE0
:10062000A4F1FF04B6F5007F64F5407404D25FEADC
:100630004E0E6D4146EB060642EAC62141EA55518F
:100640004FEAC52040EA5E504FEACE2EB4F1FD0CD1
:1006500088BFBCF5E06F1ED8BEF1004F08BF5FEA4F
:10066000500E50F1000041EB045170BD06F0004601
:1006700046EA010140EA020081EA0301B4EB5C04AE
:10068000C2BFD4EB0C0541EA045170BD41F48011A6
:100690004FF0000E013C00F3AB8014F1360FDEBFCB
:1006A000002001F0004170BDC4F10004203C35DAA7
:1006B0000C341BDC04F11404C4F1200500FA05F32A
:1006C00020FA04F001FA05F240EA020001F00042CB
:1006D00021F0004110EBD37021FA04F642EB060141
:1006E0005EEA430E08BF20EAD37070BDC4F10C046B
:1006F000C4F1200500FA04F320FA05F001FA04F22F
:1007000040EA020001F0004110EBD37041F100011A
:100710005EEA430E08BF20EAD37070BDC4F1200525
:1007200000FA05F24EEA020E20FA04F301FA05F28D
:1007300043EA020321FA04F001F0004121FA04F235
:1007400020EA020000EBD3705EEA430E08BF20EA05
:10075000D37070BD94F0000F0FD101F0004640003F
:1007600041EB010111F4801F08BF013CF7D041EAC1
:10077000060195F0000F18BF704703F000465200C5
:1007800043EB030313F4801F08BF013DF7D043EA96
:100790000603704794EA0C0F0CEA135518BF95EA4C
:1007A0000C0F0CD050EA410618BF52EA4306D1D1D3
:1007B00081EA030101F000414FF0000070BD50EAF2
:1007C000410606BF1046194652EA430619D094EA7C
:1007D0000C0F02D150EA013613D195EA0C0F05D166
:1007E00052EA03361CBF104619460AD181EA0301BA
:1007F00001F0004141F0FE4141F470014FF0000072
:1008000070BD41F0FE4141F4780170BD70B54FF00C
:10081000FF0C4CF4E06C1CEA11541DBF1CEA13558C
:1008200094EA0C0F95EA0C0F00F0A7F8A4EB05046E
:1008300081EA030E52EA03354FEA013100F0888065
:100840004FEA03334FF0805545EA131343EA12632E
:100850004FEA022245EA111545EA10654FEA0026E3
:100860000EF000419D4208BF964244F1FD0404F59C
:10087000407402D25B084FEA3202B61A65EB0305F8
:100880005B084FEA32024FF480104FF4002CB6EBB5
:10089000020E75EB030E22BFB61A754640EA0C0035
:1008A0005B084FEA3202B6EB020E75EB030E22BF75
:1008B000B61A754640EA5C005B084FEA3202B6EBB6
:1008C000020E75EB030E22BFB61A754640EA9C0075
:1008D0005B084FEA3202B6EB020E75EB030E22BF45
:1008E000B61A754640EADC0055EA060E18D04FEA03
:1008F000051545EA16754FEA06164FEAC30343EAA3
:1009000052734FEAC2025FEA1C1CC0D111F4801F6F
:100910000BD141EA00014FF000004FF0004CB6E768
:1009200011F4801F04BF01430020B4F1FD0C88BF07
:10093000BCF5E06F3FF6AFAEB5EB030C04BFB6EB12
:10094000020C5FEA500C50F1000041EB045170BD05
:100950000EF0004E4EEA113114EB5C04C2BFD4EB32
:100960000C0541EA045170BD41F480114FF0000EB6
:10097000013C90E645EA060E8DE60CEA135594EA32
:100980000C0F08BF95EA0C0F3FF43BAF94EA0C0F35
:100990000AD150EA01347FF434AF95EA0C0F7FF4AA
:1009A00025AF104619462CE795EA0C0F06D152EAFE
:1009B00003353FF4FDAE1046194622E750EA4106E2
:1009C00018BF52EA43067FF4C5AE50EA41047FF4F3
:1009D0000DAF52EA43057FF4EBAE12E74FF0FF3C58
:1009E00006E000BF4FF0010C02E000BF4FF0010C29
:1009F0004DF804CD4FEA410C7FEA6C5C4FEA430CA2
:100A000018BF7FEA6C5C1BD001B050EA410C0CBFF0
:100A100052EA430C91EA030F02BF90EA020F002052
:100A2000704710F1000F91EA030F58BF994208BFB9
:100A300090422CBFD8176FEAE37040F00100704776
:100A40004FEA410C7FEA6C5C02D150EA013C07D1CD
:100A50004FEA430C7FEA6C5CD6D152EA033CD3D018
:100A60005DF8040B704700BF8446104662468C4612
:100A70001946634600E000BF01B5FFF7B7FF002845
:100A800048BF10F1000F01BD4DF808EDFFF7F4FF6E
:100A90000CBF012000205DF808FB00BF4DF808EDF9
:100AA000FFF7EAFF34BF012000205DF808FB00BF1C
:100AB0004DF808EDFFF7E0FF94BF012000205DF83E
:100AC00008FB00BF4DF808EDFFF7CEFF94BF0120F3
:100AD00000205DF808FB00BF4DF808EDFFF7C4FFEC
:100AE00034BF012000205DF808FB00BF4FEA410C35
:100AF0007FEA6C5C02D150EA013C0AD14FEA430C18
:100B00007FEA6C5C02D152EA033C02D14FF0000054
:100B100070474FF0010070474FEA410212F5001292
:100B200015D211D56FF47873B3EB625212D94FEA34
:100B3000C12343F0004343EA505311F0004F23FA1E
:100B400002F018BF404270474FF00000704750EA73
:100B5000013005D111F0004008BF6FF00040704730
:100B60004FF00000704700BF4A0011D212F500128A
:100B700011D20DD56FF47873B3EB62520ED44FEAF5
:100B8000C12343F0004343EA505323FA02F0704775
:100B90004FF00000704750EA013002D14FF0FF30B3
:100BA00070474FF0000070474FEA4102B2F1E04356
:100BB00024BFB3F5001CDCF1FE5C0DD901F0004C44
:100BC0004FEAC0024CEA5070B2F1004F40EB830094
:100BD00008BF20F00100704711F0804F21D113F1C0
:100BE0003872BCBF01F00040704741F480114FEAF9
:100BF0005252C2F11802C2F1200C10FA0CF320FA82
:100C000002F018BF40F001004FEAC1234FEAD3239E
:100C100003FA0CFC40EA0C0023FA02F34FEA430308
:100C2000CCE77FEA625307D150EA01331EBF4FF091
:100C3000FE4040F44000704701F0004040F0FE40AC
:100C400040F40000704700BF80F0004002E000BFA9
:100C500081F0004142001FBF5FEA410392EA030FA7
:100C60007FEA226C7FEA236C6AD04FEA1262D2EBF1
:100C70001363C1BFD218414048404140B8BF5B42F6
:100C8000192B88BF704710F0004F40F4000020F08F
:100C90007F4018BF404211F0004F41F4000121F0A5
:100CA0007F4118BF494292EA030F3FD0A2F10102EF
:100CB00041FA03FC10EB0C00C3F1200301FA03F12D
:100CC00000F0004302D5494260EB4000B0F5000F50
:100CD00013D3B0F1807F06D340084FEA310102F10F
:100CE0000102FE2A51D2B1F1004F40EBC25008BFC1
:100CF00020F0010040EA03007047490040EB00008B
:100D0000013A28BFB0F5000FEDD2B0FA80FCACF18B
:100D1000080CB2EB0C0200FA0CF0AABF00EBC250B8
:100D200052421843BCBFD0401843704792F0000FA6
:100D300081F4000106BF80F400000132013BB5E7F9
:100D40004FEA41037FEA226C18BF7FEA236C21D06F
:100D500092EA030F04D092F0000F08BF08467047D4
:100D600090EA010F1CBF0020704712F07F4F04D1A2
:100D7000400028BF40F00040704712F100723CBFB5
:100D800000F50000704700F0004343F0FE4040F4DF
:100D9000000070477FEA226216BF08467FEA23639D
:100DA0000146420206BF5FEA412390EA010F40F488
:100DB000800070474FF0000304E000BF10F00043D4
:100DC00048BF40425FEA000C08BF704743F09643BB
:100DD00001464FF000001CE050EA010208BF7047D6
:100DE0004FF000030AE000BF50EA010208BF70475D
:100DF00011F0004302D5404261EB41015FEA010C72
:100E000002BF84460146002043F0B64308BFA3F169
:100E10008053A3F50003BCFA8CF2083AA3EBC2534B
:100E200010DB01FA02FC634400FA02FCC2F120026A
:100E3000BCF1004F20FA02F243EB020008BF20F0A1
:100E40000100704702F1200201FA02FCC2F1200207
:100E500050EA4C0021FA02F243EB020008BF20EAFC
:100E6000DC7070477BB972B90029BEBF00204FF01B
:100E7000004106E008BF00281CBF6FF000414FF0A2
:100E8000FF3000F015BAADF1080C6DE904CE002971
:100E900009DB002B1ADB00F0A3F8DDF804E0DDE944
:100EA000022304B07047404261EB4101002B1BDB81
:100EB00000F096F8DDF804E0DDE9022304B04042DA
:100EC00061EB4101524263EB43037047524263EBD3
:100ED000430300F085F8DDF804E0DDE9022304B007
:100EE000404261EB41017047524263EB430300F023
:100EF00077F8DDF804E0DDE9022304B0524263EB49
:100F00004303704753B94AB9002908BF00281CBFE2
:100F10004FF0FF314FF0FF3000F0CAB9ADF1080CCF
:100F20006DE904CE00F05CF8DDF804E0DDE90223B1
:100F300004B0704730B1012390FAA0F0B0FA80F00D
:100F40001844704708460029FBD02123F4E700BF6E
:100F5000430803F05533C01A830803F0333300F01D
:100F60003330184400EB101000F00F3000EB00207D
:100F700000EB0040000E704707EE900AF5EEC07AD5
:100F8000F1EE10FA01D400F00BB8F1EE677A08B573
:100F900017EE900A00F004F8404261EB410108BDF1
:100FA000D0B5FFF7B1FA0C4B002206460F46FFF70B
:100FB00003FBFFF7D9FD0446FFF784FA074B002235
:100FC000FFF7FAFA02460B4630463946FFF73CF97E
:100FD000FFF7CAFD2146D0BD0000F03D0000F04102
:100FE0002DE9F047089D04468E46002B4DD18A42DC
:100FF000944669D9B2FA82F252B101FA02F3C2F10F
:10100000200120FA01F10CFA02FC41EA030E94409F
:101010004FEA1C48210CBEFBF8F61FFA8CF708FBC0
:1010200016E341EA034306FB07F199420AD91CEB98
:10103000030306F1FF3080F01F81994240F21C81CA
:10104000023E63445B1AA4B2B3FBF8F008FB103312
:1010500044EA034400FB07F7A7420AD91CEB040447
:1010600000F1FF3380F00A81A74240F20781644417
:10107000023840EA0640E41B00261DB1D44000239C
:10108000C5E900433146BDE8F0878B4209D9002D00
:1010900000F0EF800026C5E9000130463146BDE88A
:1010A000F087B3FA83F6002E4AD18B4202D38242F4
:1010B00000F2F980841A61EB030301209E46002DA3
:1010C000E0D0C5E9004EDDE702B9FFDEB2FA82F2F8
:1010D000002A40F09280A1EB0C014FEA1C471FFA56
:1010E0008CFE0126200CB1FBF7F307FB131140EA3D
:1010F00001410EFB03F0884208D91CEB010103F10A
:10110000FF3802D2884200F2CB804346091AA4B2CB
:10111000B1FBF7F007FB101144EA01440EFB00FE9F
:10112000A64508D91CEB040400F1FF3102D2A64504
:1011300000F2BB800846A4EB0E0440EA03409CE7A3
:10114000C6F12007B34022FA07FC4CEA030C20FA50
:1011500007F401FA06F31C43F9404FEA1C4900FA70
:1011600006F3B1FBF9F8200C1FFA8CFE09FB1811ED
:1011700040EA014108FB0EF0884202FA06F20BD960
:101180001CEB010108F1FF3A80F08880884240F2B0
:101190008580A8F102086144091AA4B2B1FBF9F0F4
:1011A00009FB101144EA014100FB0EFE8E4508D9EF
:1011B0001CEB010100F1FF346CD28E456AD9023874
:1011C000614440EA0840A0FB0294A1EB0E01A14259
:1011D000C846A64656D353D05DB1B3EB080261EBC7
:1011E0000E0101FA07F722FA06F3F1401F43C5E9A1
:1011F000007100263146BDE8F087C2F12003D840D7
:101200000CFA02FC21FA03F3914001434FEA1C4718
:101210001FFA8CFEB3FBF7F007FB10360B0C43EA0A
:10122000064300FB0EF69E4204FA02F408D91CEBBA
:10123000030300F1FF382FD29E422DD902386344B8
:101240009B1B89B2B3FBF7F607FB163341EA034158
:1012500006FB0EF38B4208D91CEB010106F1FF38A7
:1012600016D28B4214D9023E6144C91A46EA00469E
:1012700038E72E46284605E70646E3E61846F8E630
:101280004B45A9D2B9EB020864EB0C0E0138A3E779
:101290004646EAE7204694E74046D1E7D0467BE75A
:1012A000023B614432E7304609E76444023842E7D2
:1012B000704700BF02E000F000F8FEE772B6374862
:1012C00080F30888364880F3098836483649086034
:1012D00040F20000CCF200004EF63471CEF2000174
:1012E0000860BFF34F8FBFF36F8F40F20000C0F272
:1012F000F0004EF68851CEF200010860BFF34F8F28
:10130000BFF36F8F4FF00000E1EE100A4EF63C7114
:10131000CEF200010860062080F31488BFF36F8FBF
:10132000A9F03AFFA8F0A2FF4FF055301F491B4A21
:1013300091423CBF41F8040BFAE71D49184A91421B
:101340003CBF41F8040BFAE71A491B4A1B4B9A426F
:101350003EBF51F8040B42F8040BF8E7002018498F
:10136000184A91423CBF41F8040BFAE7A9F018FF74
:10137000A8F0D0FF144C154DAC4203DA54F8041B0E
:101380008847F9E701F002F9114C124DAC4203DA3B
:1013900054F8041B8847F9E7A9F000BF00060020B5
:1013A000002200200000010808ED00E000000020FD
:1013B00000060020D0490E0800220020842C0020C6
:1013C000882C0020285D0120E00101083802010876
:1013D00038020108380201082DE9F04F2DED108A7E
:1013E000C1F80CD0C3689D46BDEC108ABDE8F08FF3
:1013F000002383F311882846A0470020A8F0BCFCF6
:10140000FEE7A8F019FB00DFFEE7000001F0FF0196
:10141000102A2BDB10F0070F08D010F8013B013A1F
:101420008B422DD010F0070F42B3F6D1F0B441EA51
:10143000012141EA014122F007047FF00007002367
:10144000F0E80256083C85EA010586EA010685FABD
:1014500047F5A3FA87F586FA47F6A5FA87F68EB917
:10146000EED1F0BC01F0FF0102F0070232B110F83A
:10147000013B013A83EA010313B1F8D10020704720
:1014800001387047002D06BF35460338073815F080
:10149000010F07D1013015F4807F02BF013015F430
:1014A000C03F0130F0BC0138704700BF10F8012B7D
:1014B00011F8013B012A28BF9A42F7D0D01A704791
:1014C000034613F8012B002AFBD1181A0138704784
:1014D00038B50022002304460D46FFF7DFFA28B98D
:1014E00020462946BDE8384000F00AB8204605F1FC
:1014F000004100F005F8404261EB410138BD00BFFA
:10150000D0B50C4B002206460F46FFF755F8FFF703
:101510002BFB0446FEF7D6FF074B0022FFF74CF8E3
:1015200002460B4630463946FEF78EFEFFF71CFB9F
:101530002146D0BD0000F03D0000F04103680022CC
:101540001B68184710B503685B680446984708B1E4
:1015500094F84D0010BD000038B504467BF008FF3C
:101560000E4B1D680146E86A02681268904751F008
:1015700075FEEB6A93F89C1050F060FE94F83730DB
:101580005BB183F055FEEB6AD3F8A030C01AB0F51A
:10159000FA6F24BF002384F8373038BD942C002024
:1015A00070B50E4605465DF0C5FA5DF087FA10B9D4
:1015B0000124204670BD0A4B93F97633012BF7D1F5
:1015C0005DF0B8FA437A002BF2D15DF0B3FA847A79
:1015D000002CEDD1034A314628467CF00FF9E8E7AC
:1015E000984C00205C350C08034BD3F8E0330BB962
:1015F0007BF074BE01207047984C00202DE9F04329
:101600002DED028BC47F91B006460F468CB990F940
:101610000430002B00F0FE807F4B1D68A86A036831
:101620005B6B9847044650B97C4A394630467CF09B
:10163000E5F8204611B0BDEC028BBDE8F083B3683D
:101640004BB933685B6B3946304611B0BDEC028B49
:10165000BDE8F0431847E86AFFF774FF0446002826
:10166000E7D1394630467CF0A7FFDFF8E481054634
:10167000394630467CF0EAF898EDE27AD8EDE17A26
:10168000B4EEE77A2840F1EE10FAC5B209D598F920
:101690008033032B05D0624A394630467CF0AEF8E1
:1016A0002546D8EDCA7AB0EE088AF4EEC87AF1EE93
:1016B00010FA0BD517EE900AFEF726FF594ACDE92E
:1016C0000001394630467CF099F80025D8EDCB7AF8
:1016D000F4EEC87AF1EE10FA0BD517EE900AFEF789
:1016E00013FF514ACDE90001394630467CF086F8B7
:1016F0000025D8EDCC7AB8EE087AF4EEC77AF1EE90
:1017000010FA0BDD17EE900AFEF7FEFE474ACDE910
:101710000001394630467CF071F80025B8F91433E1
:10172000042B07DC052200923946414A30467CF002
:1017300065F80025D8F8C40B5DF058FA80B198F927
:1017400076336BB1D8F8C43BB8F97823B3F90E30CF
:101750009A4205DA374A394630467CF04FF8002580
:10176000DFF8F09039463046FFF71AFF99F8893DC7
:10177000002B48D100EA05042F484FF4806100F0A7
:10178000FBFE78B1D8F8C43BB3F90C30A3F2E242C7
:1017900092B2B2F5FA7F05D9284A394630467CF034
:1017A0002DF80024264890F824345BB100F21C4048
:1017B0002CF074FE054628B9224A394630467CF0A2
:1017C0001DF82C4600212E2204A80DF10C080391CF
:1017D000ADF086FCD9F8740D4246322108F038F994
:1017E000054600287FF425AFD9F8740D03689B687F
:1017F0009847154ACDF800800346394630467BF0BD
:10180000FDFF2C4615E7114A394630467BF0F6FFBE
:101810000024B1E701240CE7942C00206C350C085F
:1018200083350C08A6350C08C6350C08E8350C08BD
:101830000A360C0829360C08982C002064360C084F
:10184000987C00208C360C08BCE70C084F360C083E
:10185000984C0020986C002070B505460E46FFF7A6
:101860009FFE3146044628467CF052FD2040C0B21F
:1018700070BD0000F0B591B005460E467CF086F8CC
:101880000446D8B1102128467BF08EFDB0B100216E
:101890002E2204A803AF0391ADF022FC10F0D8F97A
:1018A00032233A4601210FF0E1FC044630B9054BE2
:1018B00000973246102128467BF07EFD204611B06D
:1018C000F0BD00BFA0360C0870B505460E46B1B994
:1018D00090F910408CB116480BF020F8DFED157A26
:1018E000B0EEC00AB4EEE70AF1EE10FA07D4124ADD
:1018F000012128467BF082FF3446204670BDAB684C
:101900009BB10E4B1B68D86AFFF71CFE044630B132
:101910005BF01EFC0A4A042154F04EFDEDE731460F
:101920002846BDE870407CF0FDBA0124E5E700BF21
:10193000982C002000000034AC360C08942C0020B9
:10194000BE360C0838B504467CF0F6FE0546A8B154
:101950000B4805F063FB38B10A490B480FF0C6FD90
:1019600010B1074800F0DAFD2046FFF7F5FD01232E
:10197000064984F8373020467CF0EEFD284638BD15
:10198000982C0020908B0020A83F0020E0360C0807
:10199000F8B505460E461746C2B1232901D00129E4
:1019A00014D81E4807F0D8FB044668B1002420462E
:1019B000F8BD95F91030022B08D05BF0C9FB184A2E
:1019C000062154F0F9FCF2E7002EF2D03A463146F7
:1019D00028467CF067FF04460028E7D0114ED6F871
:1019E000742D06F608539A4203D003F214702DF0BA
:1019F0008BF9D6F8740D03689B6B98470A4B83F8F4
:101A0000F0032846FFF7A8FD4FF0FF330749C6F85B
:101A1000A43D28467CF0A0FDC9E700BF982C00201B
:101A2000F0360C08986C0020987C002008370C08D1
:101A3000F8B505460E467BF063FD104B93F94B73EA
:101A40000446CFB90E48BD212DF0F4F838B10D4B46
:101A500032464FF4804128467BF0AEFC3C460848B5
:101A6000BC212DF0E7F838B1074B32464FF48041E6
:101A700028467BF0A1FC00242046F8BD984C0020AD
:101A8000B48000201C370C0848370C080020704731
:101A9000014800F0EBBC00BF982C002003685B6895
:101AA000184700000DF062B864F0F4BB5CF090BF22
:101AB00025F0E4BB50F044BD07F084BC4EF0E4BD1B
:101AC0000AF034BA02F03ABE4DF07AB914F004B913
:101AD00060F0F8BB60F076B80CF048B946F03EB95B
:101AE0000AF09ABF13F056BC66F088B95CF092BC5D
:101AF0005AF09CBD06F096BE04F02ABA09F09EBDCD
:101B00000AF084B90BF066BF0CF0DEB90AF0BCBD78
:101B10000CF086B801F032B900F2845017F0A6B983
:101B200007F0BCB990F8F432B02202FB030390F83E
:101B3000382393F8D13012B1012B28BF0123184666
:101B400070470000034808602C21117008221A60B9
:101B5000704700BF8C3A0C0870B5044604F59855E0
:101B600000F5C04004301035FFF7F6FC0021284690
:101B70000FF0F4FF802120460CF012FC18B126F083
:101B800071FF25F041F804F50053D3EDCA7ADFED7B
:101B9000236A93EDCC7A67EEA67A04F58052FDEEC7
:101BA000E77A02F25C51D1ED006AF8EEE77A02F5CD
:101BB000AB6267EEA67A03F6D833FDEEE77A05F559
:101BC000457017EE901A43F8041CD2ED007AF0EE3F
:101BD000E77A67EE877A04F5B251C3ED007A0831EF
:101BE00029F036FF04F5A04694ED467AD6EDDB7A6F
:101BF000E7EE007AC6EDDB7AB0EE670A27F056FC16
:101C00004FF4001186EDDB0A20460CF0C9FB20B131
:101C10002846BDE870400EF0D7BA70BD0000C8423B
:101C2000FFF79ABF10B500F580430446D3F8740D52
:101C300003689B6B984704F5A04393F8AB333BB91B
:101C400030B104F531503030BDE8104080F0E0BFD5
:101C500010BD0000FFF7E6BF38B54FF48011044611
:101C60000CF09EFB054620B9012120460CF098FBA4
:101C70000546022120460CF093FB48B115B92046D9
:101C800002F000FD04F5985010300EF09BF901E0D1
:101C9000002DF7D14FF4805120460CF081FB28B184
:101CA00004F5BF40BDE8384060F032BC38BD0000EC
:101CB000FFF7D2BF38B54FF4801104460CF070FB2B
:101CC0000121054620460CF06BFB18B115B92046E2
:101CD00002F0D8FC102120460CF062FB60B12046D7
:101CE00002F044FD4FF4800120460CF059FB18B976
:101CF00026F0B8FE25F07AF8202120460CF050FBA3
:101D000028B1204602F0A8FD204602F0C3FE4FF4A1
:101D1000005120460CF044FB10B1204602F0A2FE18
:101D2000802120460CF03CFB28B126F09BFEBDE84C
:101D3000384024F08DBF38BDFFF7BCBF00F58043AD
:101D400000F5BC40D3F8981D5C307EF0A3B90000CC
:101D5000FFF7F4BF10B5044617F078F990F9213079
:101D60008BB190F8403373B194F9A8355BB1064B51
:101D70001B68DB6A93F89C302BB904F28450BDE8F1
:101D8000104016F08BBE10BD942C0020FFF7E2BF70
:101D90002DE9F843434B1B68DB6A93F89C300446FB
:101DA000002B7DD000F5805797F81936002B77D09F
:101DB00007F0D2F9002873D004F5FF5507F58059D4
:101DC000183599F8461128460DF0A0FC002867D078
:101DD00004F590763046FFF7A5FE022860D994F806
:101DE00014344FF0B00808FB034393ED837AF1EE0F
:101DF000007AB4EEE77AF1EE10FA51D499F8461170
:101E000028460DF033FF04F50053B3F9142307EE11
:101E1000902AB8EEE77AB4EEC07AF1EE10FA0CDD53
:101E200094F8142408FB0242F8EE677A92ED837A64
:101E3000F4EEC77AF1EE10FA32DCD7F80825D3F8C1
:101E4000D41B002AB8BF52428A4229DC07F20C5246
:101E5000D2ED007AD3EDCB6A9FED136AF8EEE77A04
:101E600066EE866AF4EEE67AF1EE10FA18DC03F616
:101E7000D83292ED007A27EE067AF4EEC77AF1EEC8
:101E800010FA0DD494F81414B02202FB0161284614
:101E9000B3F9162301F58271BDE8F8430DF04CBA91
:101EA000BDE8F883942C00200000C842FFF770BF03
:101EB0002DE9F04190F814342D4D00EB03132F68F9
:101EC000D3F8C48100F5907604463046FFF72AFE29
:101ED000474514D0022814D904F58047C5F800807E
:101EE00097F89C3D012B15D817D104F5A045D5F8DE
:101EF000003FE3B9D5F8043FCBB905230BE0022836
:101F000010D804F5804393F89C2D5AB1052283F82C
:101F10009C2D07E0013B87F89C3D04F5BA500C303E
:101F200011F016F82046BDE8F04109F02FBD114B25
:101F30001B68D86A03685B68984780460028ECD124
:101F400094F81414B02303FB0161DC31204605F042
:101F5000D7F8D5F8E43E0FCB05F6E86605F6087528
:101F600086E80F0085E80F0087F89C8DD5E700BF55
:101F7000882C0020942C0020FFF79ABF10B500F5A4
:101F8000A04300F5805493F8AB231AB1002384F8E2
:101F900019360AE0D3F8F833042B07D100F5BB401B
:101FA000503081F0D3F884F8190610BD0123EEE714
:101FB00010B500F5804400F59A43D4F8741D083339
:101FC000994200F5A04308D000F59A424C32914264
:101FD0001CBF4FF0FF32C3F86423074AC3F85423F1
:101FE000064AC3F85823FFF7C9FFD4F8740D0368F5
:101FF000BDE810401B6918470000C8420000C8C275
:10200000FFF7D6BFF7B500F5A0460446D6F8F8337B
:102010008B420D463ED00B1F00F5BB47594207F1DE
:10202000500759413846019180F080FF01993846A8
:1020300080F07CFF042D02D117486CF065FDD6F8C6
:10204000F833012B18D1032D16D104F5C04004300C
:102050007BF098F940B1204607F07EF820B104F5F6
:102060002D502C306CF04AFD2046C6F8F85303B0D2
:10207000BDE8F04002F05CBC072DF5D1D6F8742322
:102080006423052192FBF3F304F54E50034A54F008
:1020900093F9E9E703B0F0BD04580020EC370C08D1
:1020A00038B500F580450446D5F8740D03689B6B80
:1020B000984700283FD004F5A04393F8F023D2BB03
:1020C000D5F8741D04F59A420832914235D193F83F
:1020D000A4232AB901212046BDE83840FFF792BF6A
:1020E000B3F85A24152A26D193F8D41D11F0010112
:1020F0001FD1D3F8F823072A1BD093F94A3E0BB916
:102100000421E8E720460AF009FCDFED0F7AB4EE7F
:10211000E70AF1EE10FAF3DB04F5BB40503080F033
:1021200055FF0028ECD0094A062104F54E5054F022
:1021300043F90721CFE70321CDE704F59A434C3358
:102140009942F8D138BD00BF0000B44210380C08E5
:1021500038B5214CD4F8742D04F608539A422DED6D
:10216000028BB0EE408A03D00020BDEC028B38BD5C
:1021700004F58055D5F8F833042B23D194F89D3D10
:1021800033B11649A1F6DC202DF036F80028ECD149
:102190009FED137AF0EEC87AF4EEC77AF1EE10FAFA
:1021A00007D49FED100A28EE008ABDEEC88A85ED9F
:1021B000DD8A0D4880F00AFF0028D5D0002385F87D
:1021C000A733D2E7B5F85A14A4F5804006F090F989
:1021D0000028D3D1C8E700BF986C0020908B002066
:1021E000000000340000C842688A002010B52DEDC0
:1021F000028B00F5A0430446D3F8F823042A0BD140
:1022000004F06CF92046B0EE408A04F037FA38EE5C
:10221000400ABDEC028B10BD03F6347393ED000A47
:10222000F7E700002DE9F0412DED028B00F58C65FC
:102230008AB00446284612F045F804F59850002369
:1022400007A910300793089309930FF013FB002898
:1022500000F087809DED090ADFED597A04F5A0456D
:1022600095EDE17A20EE270ADFED567AA7EE270AF0
:1022700004F5AA40143004F5804685EDE10A65F0C6
:10228000D1FF2046FFF70CFFD6F8740D03689B6B57
:10229000984795F8AB33002B5ED100285CD095F8B9
:1022A000F033002B58D1D5F8F833042B70D09FEDC4
:1022B000468A204604F004FA04F5C04204F59A4325
:1022C000C2F8BC00D6F8741D203399421CD195F891
:1022D000783FCBB904F50053B3F9A43B002B04DCE1
:1022E0003A49D1F8641BC9060ED5D5F8E47ED5F875
:1022F000EC1E7F680A33C91B64277B438142ACBF55
:102300005B181B18C2F8BC30D5F8F833D2F8BC10F3
:10231000D6F8A02D05912046049203930CF0A2FA62
:10232000B6F9AE6D07462046FFF760FFCDE90076AF
:1023300004F50050D0EDEC1A059905F2144504F5AA
:102340003150F0EE400ADDE9033295ED001AB0EEAF
:10235000480A303080F000F90AB0BDEC028BBDE8CD
:10236000F08104F59070FFF7DDFB02280AD994F89C
:102370001434B02202FB034393F8402212B193EDD0
:102380008B0A69E7284611F037FEB1EE400A63E791
:1023900004F5BD4704F5BE48783708F1080804F590
:1023A000BD4142466831384615F094FF00283FF49D
:1023B0007EAF4146384616F021F8B0EE408A78E705
:1023C000CDCC4C3ECDCC4C3F00000000984C0020C2
:1023D000FFF728BF00F5804200F59A43D2F8742D2C
:1023E00044339A421FBF00F5A040D0F88C330B60F5
:1023F000012008BF0020704710B500F5804200F5AD
:102400009A43D2F8742D44339A420C4612D000F508
:102410004050D0F8A80503681B69984707EE900A5A
:102420009FED057AF8EEE77A012067EE877AC4ED32
:10243000007A10BD0020FCE70AD7233C10B500F558
:10244000804200F59A43D2F8742D44339A420C46E8
:102450000AD000F54050D0F8A80503685B6998479A
:10246000012084ED000A10BD0020FCE730B50546D0
:102470000FC985B06C4684E80F0040F279322146DE
:10248000284604F0D1FC0C4B03F55362D3F8743D9D
:1024900093420ED19DF8001011F0040102D12046A4
:1024A00015F014FD0548214604F078FD012005B023
:1024B00030BD0020FBE700BF986C0020982C002066
:1024C00000F58040D0F8740D03689B6C184700003D
:1024D00000F58040D0F8740D0368DB6C18470000ED
:1024E00010B500F5805303F5A36403F21453246878
:1024F00014601B680B6000F50050D0F8643B9B052E
:1025000009D4D0EDEC6AD2ED007A9FED037AE6EEC5
:10251000C77AC2ED007A10BD35FA8E3C38B50D4D44
:10252000044629460C480FF0F3F804F5804305F102
:102530003C0183F89D0D04F5985010300EF080FF9B
:1025400004F5BE40D0ED0D7AF1EE677AC0ED0D7A5C
:1025500038BD00BF908B0020A83F002010B5044676
:1025600000F590701FF01CF92046BDE81040FFF701
:10257000D5BF0000FFF7F2BF00F50050D0F8643B74
:10258000194214BF012000207047000038B5054BE8
:102590001C6823680A461D68034B01462046A8476D
:1025A000002038BD942C0020982C002070B52DED13
:1025B000028B0446036804F500559B6D9847D5F8D7
:1025C000643B1B0618D5B5F91433B5F91613CA1AAE
:1025D0000B4402EBD27203EBD37352105B1000EE8C
:1025E000902A00EE103A04F59850F8EEE00AB8EEA2
:1025F000C00A10300EF0E2FC5A4BB5F846231A70B0
:1026000004F5C0455EF0FEFB04355EF04DF8002198
:102610002846FEF7F3FF544E0123B0712846F371AC
:102620007AF0A6FE28B928467BF0AAFFB0FA80F01F
:1026300040093071042120460BF0B2FE20B104F5B0
:10264000AA4034304EF0D2F828467AF091FEE8B92C
:1026500094F8143404F5A04504EB031341F28832D6
:10266000D3F8C461D5F87C3FF31A93420ED904F530
:102670009070FFF757FA022808D9C5F87C6F2046FA
:1026800005F55D6504F0CAFC00232B60B4F9A430A5
:102690001BB9B4F8A230A4F8A430B4F8A430DFED2C
:1026A000338A07EE903AF8EEE77AB7EE008A88EEC2
:1026B000270AD4ED2B7AF0EEE77AF4EEE87AF1EE21
:1026C00010FA09D5B4F9A23007EE903AF8EEE77A9D
:1026D00088EE277A84ED2B7AD4ED2B0A26F0E8FDDC
:1026E00020BB4EF095FF40F27D124FF480114EF06A
:1026F00047FF4CF01BFC4CF083F804F53C502C30A9
:10270000B0EE408A73F082FF04F54250B0EE480A02
:10271000083073F07BFFB0EE480ABDEC028B04F585
:1027200046503C30BDE8704073F070BFD4ED2B7A5A
:1027300094ED460AF0EEE77AF4EEE87AF1EE10FA5C
:1027400009D5B4F9A23007EE903AF8EEE77A88EEB0
:10275000277A84ED2B7AD4ED2B0A26F0A9FD0028E8
:10276000BFD0C6E7A0230020058E00200000003463
:10277000FFF71CBF70B500F5A046044696F9483E29
:10278000002B27DD06F0E8FC20BB04F5C04504352E
:1027900028467BF0F5FEE8B128467AF0E9FDC8B19D
:1027A00082F046FDD6F89433C01A96F9483E4FF4AD
:1027B0007A72534398420DD301221C212846FFF719
:1027C000E7F838B104F54E50034ABDE870400621E1
:1027D00053F0F2BD70BD00BF30380C0830B52DEDA0
:1027E000028B044683B000F5985001A910300FF019
:1027F00013F8002871D004F5A04595EDDF7ADDEDE2
:10280000017AB4EEE77AF1EE10FA08D504F5C0408B
:1028100004307AF0B7FD10B1019BC5F87C3304F5A4
:102820000054D4EDDA6AB4F91433052BB8BF05238C
:1028300007EE903AB4F9163307EE103AB8EEC77ABD
:10284000F8EEE77A37EE077A1820C6EE870AB6EE7A
:10285000007AF4EE470AF1EE10FAC8BFF0EE470A2C
:102860009FED2D7A67EE877A9FED2C7A86EEA71A78
:10287000F0EE007AB4EE671AF1EE10FA48BFB0EE4F
:10288000671ADDED017AF4EEC77AF1EE10FACCBFEB
:1028900086EEA70AB0EE410A26F01CFEB0EE408A92
:1028A0001F480DF0C3FF90B91E484021FFF764FE9A
:1028B00068B11D4BD3F8F833012B08D1F7EE007A3D
:1028C000B4EEE78AF1EE10FA58BFB0EE678AB0EEC8
:1028D000480A03B0BDEC028B30BD04F5C0400430A3
:1028E0007AF050FDB7EE008A0028D9D046205DF07E
:1028F0002BFDB4EEC80ADFED0D7AF1EE10FAD8BF69
:10290000B0EE480A87EE800AAAF03EFB2F209FED2A
:10291000081ADFED080ABFE73333333F17B7D13862
:10292000A83F0020982C0020987C00200000344212
:102930008FC2D53F9A99193FF8B504465CF0FAF872
:102940000368DB689847054610B900252846F8BD9E
:10295000204606F091FA04F580460746D6F8740D35
:1029600003689B6B984780B10E4BD3F8740D0368D6
:102970005B6B984748B104F5005494F9BD33002BC4
:10298000E3D0032BE1D03D46E0E796F8883D002BED
:10299000DCD004F5005494F98053023D18BF0125A2
:1029A000D4E700BF986C002073B500F5804202F6B2
:1029B000BC5393ED000AD2F8742D00F599432433EB
:1029C0009A422BD100F50053D3F8BC3BB3F9084031
:1029D000003C18BF012400F5A04300F53B5500F56D
:1029E0008050D3F80C64D0F8082593F808343435B7
:1029F000B61A5BB10A488DED010A4FF40061FFF78A
:102A0000BBFD9DED010A80F00100C3B222463146B4
:102A1000284602B0BDE870407CF060BC0024DAE7D4
:102A2000982C002010B5044605F054FE98B104F52A
:102A3000A042D2F80C3403F58C415031C2F80C148A
:102A400004F58051D1F808150029BEBFA3F58C43C9
:102A5000503BC2F80C342046FFF7A6FFBDE81040FB
:102A600004205DF05DBC00002DE9F0412DED048BEC
:102A700000F5005696EDEC8ADFED388A28EE288ABC
:102A800000F58048BDEEC88A00F5A04708F6BC53A3
:102A900093ED009AD7F8103418EE102A1A4408EE75
:102AA000102A054646205DF04FFCB8EEC88AD6EDE8
:102AB000D67AD8F8740DA0EE278A05F59943243309
:102AC0009842FDEEC87A17EE904A44D1D6F8C03B42
:102AD000B3F90860003E18BF012603685B69984798
:102AE000D0B9D8F8740D03689B6B9847A0B905F569
:102AF000C043D3F8B430022B0ED1284609F062FD52
:102B000050B107F62863D3ED007A67EEA87AFDEEA0
:102B1000E77A17EE903A1CB205F5415805F5805555
:102B200008F10C08D5F80C35E41A97F808343BB1D5
:102B30000B484FF40061FFF71FFD80F00100C3B2A6
:102B4000B0EE490ABDEC048B324621464046BDE852
:102B5000F0417CF0FFB80026BFE700BF0000C8428C
:102B6000982C002010B504460BF0BEFF68B100B2EF
:102B700000EB4000C0EB001300EE103AB8EEC00AC4
:102B8000BDE8104013205DF0CBBB2046FFF76CFF83
:102B9000F6E7000010B50E48FFF7CEFEB0B10D4CC1
:102BA00004205DF0D1FBD4F8BC0B5CF033FA0420B8
:102BB0005DF0B6FB13205DF0C7FBD4F8C00B5CF0F2
:102BC00029FABDE8104013205DF0AABB10BD00BF7C
:102BD000982C0020984C0020F8B52DED028B04466F
:102BE000FFF7AAFE002800F0828004F5804704F574
:102BF0009942D7F8743D3432934278D004F5994223
:102C00005C32934273D004F59A4293426FD004F53C
:102C10009942643293426AD004F599426C329342ED
:102C200065D004F599422C32934260D004F50055EA
:102C3000F6EE008AD5F8BC0B5CF0ACF8B4EEE80A0E
:102C4000F1EE10FA40DDB0EE087AFFEE007AE0EE29
:102C5000077AB0EE670AD5F8D42B04F5A04607EE44
:102C6000902AD6F80C34B8EEE77A07EE903AF8EEF0
:102C7000E77A5142E7EE007AFDEEE77A17EE900A26
:102C8000C6F80C0426F0C6FCC6F80C04D7F8742D60
:102C900004F59A4328339A4222D0D5F8C00B5CF051
:102CA00079F8B4EEE80AF1EE10FAB0EE408A21DCD1
:102CB000FEEE007AB4EEE70AF1EE10FA22D5B0EE9D
:102CC000087AF7EE007A19E0FEEE007AB4EEE70A31
:102CD000F1EE10FABFD5B0EE087AF7EE007AB6E75B
:102CE00024484FF48051FFF747FC0028D5D0BDECB5
:102CF000028BF8BDB0EE087AFFEE007AE8EE077AB4
:102D0000B0EE678A204605F0E5FC08B1B1EE488ACE
:102D1000D6F81034D5EDCB6A9FED176A05F6D83595
:102D200095ED007AB5EEC08A07EE903AF1EE10FA12
:102D3000CCBF28EE268A27EE488AF8EEE77A66EEC0
:102D4000866AE8EE067A27EE067AFDEEE77AFDEE71
:102D5000E66A17EE903ABDEEC77A16EE902A17EEA5
:102D6000101A17EE900AC6F8103426F053FCC6F875
:102D70001004BCE7982C00200000C84270B504463F
:102D800004F5804582F054FAD5F8843DC31AB3F5B2
:102D9000FA6F064603D9D5F8740D06F073FE2E4B74
:102DA000C5F8846DD3F8740D026813689847002144
:102DB000204609F0B3FDDFED297AB0EEC00AB4EE8B
:102DC000E70AF1EE10FA45D504F5BE43D3ED0D7ACE
:102DD000B1EE047AF0EEE77AF4EEC77AF1EE10FA8B
:102DE00038D504F58C6011F007F9F6EE007AB0EEF4
:102DF000C00AB4EEE70AF1EE10FA2BD504F5B85587
:102E000095ED057AF0EE087AB4EEE77AF1EE10FA75
:102E100005F114051ED504F53B5034307CF0CEFA94
:102E200004F541500C307CF045F804F54650243050
:102E30007CF072FF95ED007AF7EE007AB4EEE77A57
:102E4000F1EE10FA06D504F54C501830BDE870408C
:102E50007CF0B8BC70BD00BF986C0020000000344E
:102E600000F5005090F90B33012BC3BF00F547600C
:102E700090ED290ADFED047A9FED040AC8BF20EE29
:102E8000270A46205DF04CBA0000C842000000004E
:102E90002DE9F8432DED028B00F5804909F6BC536E
:102EA000D3ED008A054609F0AFF98046D9F8740DD4
:102EB00003681B6A984705F54656243698B14F4C6F
:102EC000D4F8D033002B0EDD82F0B2F9D4F8D03331
:102ED000C01A40F6B733984205D8B4F9C443304617
:102EE0007CF026FF7AE005F5C04305F5005793F81E
:102EF000A93043B1B7F99C33002B04DD05F54053ED
:102F000093F9BA3103BBD9F8743D05F599452435D9
:102F1000AB426DD00021B0EE680A30467CF0A0FCD8
:102F2000054604205DF010FA2BB207EE903A97EDBB
:102F3000D47AF8EEE77AE0EE077AFDEEE77A17EE5C
:102F4000904A444424B2CAE72846012109F030FBE4
:102F50009FED2B7AB7F99C33C0EE077A05F5A045B3
:102F600005F5836508EE103A55F80C3C9FED250AEF
:102F7000B8EEC88A28EE278A07EE903AF8EEE77A8C
:102F800067EE807A9FED200A27EE800AA9F020FEE6
:102F9000B7F91433DFED1D7A95ED007A20EE270A9C
:102FA00007EE903AF8EEE77A0021B4EEE77AF1EE18
:102FB00010FA58BFF0EE477A80EE277A3046DFED00
:102FC000147AB0EE480AA7EE270AF0EE680A7CF001
:102FD000A3FDBDEEC00A10EE103A1CB2BDEC028B90
:102FE00020460C49BDE8F84341F2941226F022BB7A
:102FF000B8F1000118BF01218DE700BF987C0020C7
:1030000000A08C450AD7233C35FA8E3C0AE81C41C7
:10301000E02E65426CEEFFFF38B500F540530546E3
:10302000D3F8A8050368DB689847014605F54C50BE
:1030300018307CF0A9FB04B22846FFF77DFC70B184
:1030400007EE904A05F50055B8EEE70AD5F8C80B2B
:103050005BF0E0FFBDEEC00A10EE103A1CB2204655
:103060000349BDE8384041F2941226F0E3BA00BFAC
:103070006CEEFFFF38B590F81434B02202FB030366
:1030800093ED837AF7EE007AB4EEE77AF1EE10FA78
:10309000044600F5A0451CD5002109F03FFCDFEDFA
:1030A000407AB0EEC00AB4EEE70AF1EE10FA10D59D
:1030B000D5F8F833012B0CD0072B0AD0002385F864
:1030C00068330023C5F86C332046BDE8384009F06A
:1030D0009BB882F0ADF8D5F87033C5F87003C31A09
:1030E000B3F57A7F84BF002385F86833204609F062
:1030F0008BF8D5F8F833012B07EE100A2DD0072BEB
:103100002BD0B8EEC77ADFED276AC7EE267A04F532
:103110000052B2F9602300EE102AB8EEC00A27EE82
:10312000800ADFED1F7AB0EEC07AB4EEE77AF1EEF6
:1031300010FA14D4002385F8683395F8683304F541
:103140004C501830D3B97CF007FABDE83840164926
:1031500000B241F2941226F06DBA9FED140A95F870
:103160006823002AE9D10122934285F86823E4D03C
:10317000072B1CBF0023C5F86C33DEE795EDDB7A27
:10318000DFED0B7A67EEC77A9FED0A7A67EE877AF2
:10319000FDEEE77A17EE901A7CF0F6FAD5E700BF5D
:1031A0000000003400A08C456CEEFFFF0000000022
:1031B000E02E65420000C84270B52DED028B00F58F
:1031C000BB46503682B0054630467FF02FFE04469F
:1031D000D8B905F50052D2F8BC3BB3F9083073B941
:1031E00005F5BE43D3ED0D7A92EDD77AF0EEE77A8E
:1031F000F4EEC77AF1EE10FA4CBF012400243046F9
:103200007FF028FE002808BF002430467FF00EFE25
:1032100028BB05F5A043D3F86433013319D0F4B9C2
:103220009FED1A8A2846FFF733FE07EE900AB8EEA4
:10323000E70A8DED010AD4B915205DF071F89DED16
:10324000010A1A2002B0BDEC028BBDE870405DF0AF
:1032500067B8002CE4D02846FFF70CFF02E02846B0
:10326000FFF7DAFE07EE900AB8EEE78ADAE71A20EF
:103270005DF0F8FA9DED010A08B9B0EE480A152094
:103280005DF04EF8B0EE480ADBE700BF000000003A
:1032900010B500F5005303F6D832D3EDCB6ADFED5D
:1032A000127A92ED007A9FED116A03F5476366EE9C
:1032B000A76A27EE277AD3ED2A7A67EE867AFDEEA3
:1032C000E66ABDEEC77AFDEEE77A044616EE902A6E
:1032D00017EE101A17EE900A26F09CF904F5A04498
:1032E000C4F8100410BD00BF0000C842A00CB345D4
:1032F00010B504460BF058F8031E2ADB04F5005104
:1033000091F90B239A4224DD04F5A040D0F8F8434C
:10331000022C1ED0D1EDD97ADFED0E6AD31A66EEFB
:10332000E76A07EE102A07EE903AB8EEC77AF8EE91
:10333000E77AD0F8103487EE876A07EE903AF8EE15
:10334000E77AE6EE867AFDEEE77A17EE903AC0F875
:10335000103410BD0000C842F8B52DED028B00F509
:10336000A0459FED440AD5F80C349FED437A07EE53
:10337000903AF8EEE77A044667EE807A9FED3F0ACE
:10338000F0EEE76AF4EE476AF1EE10FAC8BFF0EE2D
:10339000477A27EE800AA9F05BFA25F0BDFFB7EE69
:1033A000008AC8EE007A05F2144704F50056C7ED0E
:1033B000007A96F93C3353B3204605F08BF930BBC5
:1033C000B6F91433012BB8BF012307EE903A05F587
:1033D0008362F8EEE77AD2ED006A86EEA77AB4EE61
:1033E000C87AF1EE10FA15D840F6C4122449D5F87F
:1033F0000C0426F00FF9C5F80C04D6F8D42B40F6CF
:10340000C4139A42D4BFC6F8D42BC6F8D43BBDEC43
:10341000028BF8BDD7ED007AB4EEE77AF1EE10FA40
:10342000F5D588EE070A20EE000AA9F0FBFBDFEDD8
:10343000157AD5F80C0420EE270ADFED137A20EE7A
:10344000270A40F6C413FDEEC07A17EE904A9C425C
:10345000B8BF1C462246614226F0DCF8C5F80C04D1
:10346000D6F8D43BA342D4BFC6F8D43BC6F8D44B5D
:10347000CDE700BF0AD7233C0000AA4235FA8E3CB4
:103480003CF6FFFFE02E65420000C84210B500F593
:1034900040530446D3F8A80503681B68984704F511
:1034A0000053D3F8D42B514226F0B4F804F5A043CE
:1034B000C3F80C042046BDE81040FFF74DBF0000E4
:1034C00070470000012070470820704701207047B6
:1034D00070470000014B93F848037047984C002058
:1034E000034B93F9580B003818BF0120704700BFF9
:1034F000984C0020014B93F94A037047984C0020E8
:1035000013B5064BD3F8740D4B690468009308316A
:103510000EC9646CA04702B010BD00BF986C0020BB
:1035200070470000002070477047000038B5254DF7
:10353000D5F8740D03685B6898470F2834D80F28B6
:1035400039D8DFE800F00836080808080808083805
:1035500036363636363610241B4B93F8792312B1A3
:1035600093F878330BB944F01004184BD5F8742D48
:103570009A42A3F1080303D09A4218BF44F0100402
:10358000134991F9BD13C1B19A4218D0032902D150
:10359000104B9A4201D144F040040F4879F0E8FE04
:1035A00068B144F080040AE0182814BF01241824EC
:1035B000D2E71824D0E70124CEE79A42EDD144F0B7
:1035C000010038BD986C0020985C0020DC79002058
:1035D000984C0020A07900209C8C002008B504485D
:1035E00005F0BAFD00280CBF0120022008BD00BF75
:1035F000982C0020F0B52DED028B8BB005460EF017
:1036000027FB4FF48071D0F8047290ED828AD0F8D5
:103610000C6204461448FEF7AFFF30B9134BDFEDE0
:10362000147A93EDEC7AA7EE678A2D7C81F000FE88
:10363000D4F81823D4F81C33D4F81413089209933F
:1036400027221C23CDE900320390079103AA1E21F3
:10365000284604978DED058A069653F0E1FE0BB0DF
:10366000BDEC028BF0BD00BF982C0020984C0020D0
:1036700035FA8E3C2DE9F0432DED068B414ED6F800
:10368000742D06F644539A428BB075D006F58059D6
:10369000A6F5805390F81080D3F8A875D9F80C34AB
:1036A0009FED399A07EE903AD9F81034B8EEE7AAB0
:1036B00007EE903A3B6838469B68F8EEE79A9847E1
:1036C00007EE900AF8EEE77A384667EE897A2AEE36
:1036D00009AAFDEEE77A69EE899A17EE903A1DB2D3
:1036E0003B681B69984707EE900AF8EEE77AD9ED38
:1036F000E38A67EE897AA6F58040FDEEE77A06F662
:10370000A85617EE903ADFED217AF4EEE78AF1EE53
:1037100010FA58BFF0EE678A1CB202F035FE3B6823
:10372000D6ED00AADFED1A7A5B6908EE100A38467A
:103730006AEEA7AA9847FCEEE88AB8EEC88A18EEA7
:10374000903AB72228EE098AADF824301A23CDE941
:1037500000323E2103AA40468DED03AACDED049A26
:103760008DED058ACDED06AA8DED070AADF8205046
:10377000ADF8224053F054FE0BB0BDEC068BBDE813
:10378000F08300BF986C00200AD7233C00FF7F47DE
:103790000000C84208B502480AF006FE00B208BDA3
:1037A000982C002055F0FEB837B50D46134840F26E
:1037B000EF2203F039FB2C7814F004040AD0696876
:1037C00003220F4814F0BEFA0C4803B0BDE83040A5
:1037D00002F0ECBC01AA2146284614F087FB002821
:1037E000F2D0DDED017A9FED077A67EE877A224607
:1037F000FDEEE77A17EE901AE3E700BF982C002061
:10380000A08B00200000C84210B5054C012384F8AD
:103810007B3355F007FB002384F87B3310BD00BFDA
:10382000985C002058F0A2BD2DE9F0412DED028BEF
:103830004FF0000882B0CDE900281E4F9FED1E8A90
:103840000C461546B0EE480AB1F90220D7F8BC1B69
:103850004FF47A73064659F071F80123CDE900530D
:10386000B4F90020D7F8C01BB0EE480A30464FF438
:103870007A7359F063F8B4F90420D7F8C41B9FEDAC
:103880000F0A43463046CDE9005859F057F8CDE9C4
:103890000058B4F90620D7F8C81BB0EE480A4FF418
:1038A0007A73304659F04AF802B0BDEC028BBDE89D
:1038B000F08100BF984C00200000FA4400007A44D8
:1038C00038B5C5780B46352D044628BF3525352239
:1038D00000211846ABF004FC2A4604F10C01BDE8B7
:1038E0003840ABF0B3BB000010B5074B93F934255B
:1038F00040F24D3440F24D13002A08BF1C4655F0EB
:10390000D9F8204310BD00BF987C002010B50446B4
:1039100014F01CFE204610BD10B50C4C002384F89A
:10392000A73355F079FFA4F58052A4F53E73D2F881
:10393000742D9A4208D194F820342BB904F21C401B
:10394000BDE810402BF0B2BB10BD00BF987C00203A
:1039500013B5124C94F84611A4F108000BF0D6FEF2
:1039600078B194F84611A4F108000CF03DF940B18B
:1039700094F84611A4F1080002B0BDE810400CF024
:1039800075B90EF065F901A90DF046FF18B19DED6E
:10399000010A02B010BD9FED020AFAE7984C002020
:1039A0000000000008B51248D0F8742D00F63C5312
:1039B0009A4216D0B0F98C3DABB900F5805393F81C
:1039C000312382B990F8892D6AB993F8E13363B94C
:1039D000A0F5804005F0C0FB00280CBF03200420A8
:1039E00008BD0220FCE70520FAE70620F8E700BF43
:1039F000986C002010B5224B03F64452D3F8743D66
:103A0000934290B0044638D000231E48029314F02D
:103A100083F9014618B91B4802AA14F0C9F9247C9D
:103A200081F006FC184BDDED027AD3F8102FD3F8A5
:103A3000143F05930023F8EEE77A9FED147A07937D
:103A4000089309930A930B930C930D930E934FF6DF
:103A5000F853ADF83C300023CDE9030267EE877AD6
:103A600096228DF83E303323CDE90032572103AA48
:103A70002046CDED067A53F0D3FC10B010BD00BF48
:103A8000986C0020A08B0020987C00200AD7233C53
:103A900010B555F009FA044688B90A48A0F58052D5
:103AA000A0F53E73D2F8742D80F8A7439A4206D150
:103AB00090F820341BB900F21C402BF0F7FA204696
:103AC00010BD00BF987C00200120704708B5034B53
:103AD000D3F8740D03685B68984708BD986C0020A4
:103AE00030B587B005460EF0B3F804462D7C81F062
:103AF00093FBD4F88422D4F88832049205930021F1
:103B00001023CD22CDE900320290039102AA42F6A1
:103B10000C31284653F084FC07B030BD30B52DED94
:103B2000028B89B005460EF093F800F55A7393E8BE
:103B3000070002AC84E80700DDED020A9DED030AF0
:103B40002D7CF1EE600AB1EE400AA9F0D3F82046D0
:103B5000B0EE408A28F062FBDFED0B7A049B0793FE
:103B600028EE278A0C230122CDE90032A82105AADC
:103B700028468DED058A8DED060A53F051FC09B0FB
:103B8000BDEC028B30BD00BFE02E6542282938B560
:103B9000054623D007D824292BD0272911D01B294B
:103BA00008D1012413E0432937D008D84029F8D0A0
:103BB000422928D02846BDE8384059F01BB853297F
:103BC000EEE7122152F02AFE044610B900242046E6
:103BD00038BD297C13484BF049FDF8E7162152F017
:103BE0001DFE04460028F1D0297C0E484BF018FE3B
:103BF000EDE70C2152F012FE04460028E6D02846DC
:103C0000FFF78CFFE3E7102152F008FE044600287E
:103C1000DCD02846FFF764FFD9E7017C02487FF03B
:103C200003F9BEE7CC810020688A0020F0B52DEDB5
:103C3000028B05468DB01646B0EE408A0C46002930
:103C400030D0007C53F082FB0746287C54F082FA87
:103C500000F121039F4207D2287C0DB0BDEC028BFE
:103C6000BDE8F04052F0C8BD63690893636A2269F9
:103C7000CDF82530236AA069E1680792CDF8293094
:103C80006222212327680590CDE900320691287C25
:103C90000397192303AAC2218DED048A8DF82460AD
:103CA00053F0BEFB0DB0BDEC028BF0BD70B52E49DC
:103CB000D1F8742D01F644539A42044652D0A1F52E
:103CC0000055B5F8EE33DE0708D5A1F5805393ED26
:103CD000080A0122A1F6E471FFF7A8FFB5F8EE3358
:103CE000980708D52149022291ED5F0A204601F587
:103CF000BC71FFF79BFFB5F8EE33590708D51B4998
:103D0000032291EDBC0A204601F53B71FFF78EFFBF
:103D1000B5F8EE331A0708D51449052291EDD30AF8
:103D2000204601F55271FFF781FFB5F8EE33DB064F
:103D300018D50F4ED6F8F833042B13D10DF088FFA9
:103D4000054606F55D607FF09FF895EDC70ADFED4B
:103D5000097A014620EE270A20460622BDE8704077
:103D6000FFF764BF70BD00BF986C0020985C002016
:103D7000987C0020E02E654270B504460E461DF08A
:103D80004DFD90F8F412B02303FB0101DC31204615
:103D900003F0B6F9054698B13EB10DF059FF90F821
:103DA0007C3243F0020380F87C3204F5804304F552
:103DB0009A44D3F8740D2034A04201D105F0B0FD2F
:103DC000284670BD73B51646019104460DF040FFBC
:103DD00001990DF08BFB054698B13EB10DF038FF0F
:103DE00090F87C3243F0020380F87C3204F5804383
:103DF000D3F8740D04F59A432033984201D105F0AD
:103E00008FFD284602B070BD30B5054685B00C4622
:103E1000D1E9040125F0EAFD40B1684613F08CFFBA
:103E20006A462146284658F0F9FC08B9022067E0A6
:103E3000344840F24F32694602F0F6FFD4ED037A7F
:103E4000F4EE677AF1EE10FA22D69FED2F7AF0EEBB
:103E5000E77AF4EEC77AF1EE10FA54BF012200229D
:103E60009DF80030294962F3410368468DF800301F
:103E700014F0CCF80028D9D12548694668F0E4FE52
:103E800040B94FF0EBF9052216214EF09FFFCDE728
:103E90000022E5E7D4ED017AFDEEE77A17EE903ADD
:103EA000DB0706D41B4B03F55362D3F8743D9342F2
:103EB00025D11949134802220AF088F89DF800100C
:103EC00011F0040102D1684614F000F80D4869466B
:103ED00003F064F894ED020AB4EE400AF1EE10FA31
:103EE0000BD6B5EEC00AF1EE10FA06DD9DF8001013
:103EF0000948C1F3400106F071FD002000E00420F4
:103F000005B030BD982C002000000034908B0020BC
:103F1000484E0020986C0020C879002010B52DED87
:103F2000028BD1ED017A91ED008AFCEEE77A8AB03E
:103F3000CDED037A9DF80C1005AA044658F058FC04
:103F4000C8B1DFED0E7A059B009368EE277A002258
:103F5000FDEEE77A114617EE903A06A813F00CFF33
:103F600023682046D3F8CC3006A9984700200AB031
:103F7000BDEC028B10BD0220F9E700BF0000C84273
:103F800037B5124DD5F8740D03681B6A0C46984777
:103F900040B9D5F8742D05F608539A4202D0042092
:103FA00003B030BDD4ED007AD4ED020A94ED010ADD
:103FB0000748FCEEE77ACDED017A9DF8041003F096
:103FC0003FFE0028EBD00020EAE700BF986C0020FD
:103FD000982C002008B5D1ED007A9FED087A0848AA
:103FE000F0EEE77AF4EEC77AF1EE10FA54BF012151
:103FF000002104F069FB002008BD00BF0000003470
:10400000982C002010B5D1ED007AFCEEE77A17EE7F
:10401000903A9CB2012C02D0022C06D084B91148EF
:10402000214664F06DF8002010BD0F4890F8283547
:104030005B0707D559F08CF80C4A052152F0BCF902
:104040000420F1E790F914351BB959F081F8084ABA
:10405000F3E7A0F5A04007F099FF002814BF002067
:104060000420E1E7AC810020987C0020043E0C088D
:104070001F3E0C0838B58B8BC02B05460C4631D83B
:10408000B12B0BD8112B00F09680142B00F09680EA
:1040900021462846BDE8384059F09EBEB23B0E2B63
:1040A000F6D801A151F823F0174101089140010809
:1040B0009140010891400108914001089140010898
:1040C00091400108914001080D410108914001080B
:1040D000314101086D410108914001082141010869
:1040E00003410108D42B08D0B3F5967F49D0D02BDB
:1040F000CED1BDE83840FFF785BFBDE83840FFF7B7
:1041000069BF2146BDE83840FFF77EBE2146BDE8C5
:104110003840FFF703BF2146BDE83840FFF730BF06
:1041200094ED000A2848FEF713F8E8B100201CE0DF
:10413000264C94F89D3DBBB12549A1F6DC202BF01F
:10414000B3F888B104F58053012283F8552404F6AE
:1041500008510222A4F5804009F038FF0028E5D17B
:104160001C4B002283F85524042038BD174C94F8CA
:104170009D3D002BF8D01649A1F6DC202BF018F855
:10418000DFE7D1ED007A9FED147AF0EEE77AF4EEF6
:10419000C77AF1EE10FA14D5D1ED017AF0EEE77A94
:1041A000F4EEC77AF1EE10FA0BD50C49022206485C
:1041B00009F00CFFBAE70A490222F8E7094902228E
:1041C000F5E70220D1E700BF982C0020986C002072
:1041D000908B0020987C002000000034A079002003
:1041E000C0790020B879002070B53F4B03F55362C9
:1041F000D3F8743D93428EB00C4673D1CD78272D01
:1042000028BF27252722002104A8AAF069FF2A46F3
:1042100004F10C0104A8AAF019FF059B9DF8364093
:104220000093069B0193E443079B0293E4B2089B2F
:1042300003938DF8364080F0FBFF14F0810F04F0FB
:104240008705064601D1802D11D1684626F064FF0E
:10425000DFED267A264B20EE270ADFED267AC3F81B
:10426000C86320EE270ABDEEC00A83EDEF0A14F002
:10427000820F01D1802D11D1684626F067FFDFED56
:104280001B7A1B4B20EE270ADFED1A7AC3F8CC63AA
:1042900020EE270ABDEEC00A83EDF00A14F0840F69
:1042A00001D1802D11D1684626F060FFDFED0F7A35
:1042B0000F4B20EE270ADFED0F7AC3F8D06320EE14
:1042C000270ABDEEC00A83EDF10A63060AD5DDEDCB
:1042D0000C7A9FED087A064B67EE877AC3F8D863AD
:1042E000C3EDF57A0EB070BD986C0020E02E6542EB
:1042F000987C00200000C84230B5214C91B008469F
:1043000002A9FFF7DDFAD4F8742D04F553639A423D
:1043100033D19DF83C30072B2FD104F58054DDEDCF
:10432000056AD4F80C3F9FED177A07EE903AF8EE45
:10433000E77AE6EEC77AFDEEE77A17EE903AC4F830
:104340000C3F58F005FFD4F8E42ED4F80C3F526827
:104350009FED0D7A9B1A07EE903AF8EEE77A054644
:1043600067EE877A17EE900AFCF7CEF8074ACDE998
:1043700000010621284652F01FF811B030BD00BFE1
:10438000986C00200000C8420AD7233C383E0C0835
:1043900010B51D4B03F55362D3F8743D93420446A8
:1043A00096B008460FD108A9FFF78AFA9DF8541075
:1043B00003AA204658F01CFA38B958F0C9FE134A2F
:1043C000042151F0F9FF16B010BDBDF8503023F0B4
:1043D00004039BB2002BF6D0DDED0B7A9FED0C7A37
:1043E000039B009367EE877A0022FDEEE77A114681
:1043F00017EE903A04A813F0BFFC236804A9D3F881
:10440000CC3020469847DEE7986C00204C3E0C08E4
:104410000000C84230B48D7A4B7A43EA0523CD7A46
:1044200043EA0543562B04460A461BD008D8522BB4
:1044300012D0542B13D02046114630BC58F0A8BEE1
:1044400003F18073863B23F07F43012BF3D8017C7B
:10445000064830BC4BF0ACBA30BCFFF7C5BE30BC30
:10446000FFF74ABF30BCFFF793BF00BFCC810020ED
:1044700000207047C8207047012070470020704717
:104480000020704790F89C308B4286BF283150F84E
:10449000210000207047000090F89C308B4286BFBE
:1044A000283150F821000020704700000320704799
:1044B000014B93F846037047984C002070B50446B2
:1044C0004C4808F025FA18B1E36A43F40003E362AC
:1044D000484808F01DFA88B146205BF035FFDFED53
:1044E000467AB4EEE70AF1EE10FA07D8236B43F4EC
:1044F00000032363636B43F400036363E36A43F4E1
:10450000F843E3623D4BD3F8740D03685B6898474A
:104510000138172814D8DFE800F03A420C44424230
:104520004242133A3A3A3A3A3A1313131313131313
:10453000133A334A92F878338BB392F879238AB3DB
:10454000304B93F8CC3D012B3DD0022B44D02E4B69
:104550001D68DDB12D4E284696F8B21B47F0E0F8F5
:10456000A0B1E36A43F48073E36296F9EC331BB1C4
:10457000236B43F48073236396F8B21B284647F0FD
:1045800007F918B1636B43F48073636370BDD4E9BA
:104590000C2342F4E04243F4E043226363630123CB
:1045A00000E00023216B41F480622263626B42F4DD
:1045B00080606063002BC3D041F4406142F44062EC
:1045C00021636263BCE7E36A43F48003E362236B25
:1045D00043F480032363BAE7E36A43F48003E362AE
:1045E000236B43F480032363636B43F480036363AF
:1045F000ADE700BF982C0020000000B4986C0020AC
:10460000985C0020987C0020B88E0020984C0020F8
:1046100013B54FF44470CDE9002113F08FFF044629
:1046200028B1DDE9002158F0D3FF024B236020467A
:1046300002B010BD4C400C080020704700207047AD
:10464000002070470020704700F50E50283070475A
:1046500000487047D4650C0800F58040D0F8740D10
:1046600003685B681847000000F5804300F59A4036
:10467000D3F8743D08301B1A584258417047000067
:104680009B20704730B500F5A04303F5826353F8D3
:10469000042CDFED296A07EE902AB8EEE77AD3ED15
:1046A000007AF8EEE77A85B0044627EE267A67EEC0
:1046B000A67A00F59850002301A9103003938DEDE0
:1046C000017ACDED027A04F57F650BF0A3FC04F5C9
:1046D00040521C32692128464DF078FC04F54552C1
:1046E00038326A2128464DF071FC04F5405393F9A5
:1046F000BA2132B9D3ED6C7AF5EEC07AF1EE10FA48
:1047000006DD04F54B522C326B2128464DF05EFC41
:1047100004F54C54183420467BF058F828B104F1C5
:1047200030026D2128464DF051FC0DF091FA0CF04D
:10473000D9FF05B030BD00BF0AD7233C10B54FF4F8
:104740008011044609F02CFE10B12046FFF79AFFB5
:104750004FF48001204609F023FE28B124F082F9AD
:10476000BDE8104022F042BB10BD000030B500F59E
:10477000985591B000231035029302A900230446F6
:104780000DF1070228468DF807300DF04BF803A90C
:1047900028460CF09BF808B92D4B039330220021DA
:1047A00004A8AAF09DFCA3238DF8103095238DF862
:1047B000113080F045FD04F5A042CDF81300D2F889
:1047C0000C34ADF81B3004F58053D2F81024CDF82A
:1047D00017104620D3F80815D3F80C35ADF81D1086
:1047E000ADF81F20ADF821305BF0AEFD10EE103AB1
:1047F0001520CDF823305BF0A7FD10EE103ACDF870
:10480000273004F531539FED137AD3ED357A67EEF7
:10481000877A284617EE903ACDF82B30029BCDF8D8
:104820002F309DF807308DF83330039B0D930DF03A
:10483000FFF904F580433022D3F8B03D8DED0E0A28
:1048400004A904F57F600F934DF014FD11B030BD45
:104850002292CA7F0000C84270B58EB0352204464D
:1048600000216846AAF03CFCA3238DF80030952374
:104870008DF8013001238DF8023080F0E1FC04F561
:10488000A04504F54056D5F88C33CDF80300D6F892
:10489000A805CDF80710CDF80B3003681B699847C1
:1048A000ADF80F00D6F8A80503689B689847ADF8E7
:1048B00011001E4801F068FDADF81300D6F8A805F8
:1048C00003685B69984710EE103AD6F8A805CDF852
:1048D000153003689B69984710EE103ACDF81930EF
:1048E00004F5804303F6A85135220968CDF81D1060
:1048F000D5F8101FCDF82110D5F8141FCDF82510CC
:10490000D5F80C1FCDF8291004F5C041D3F8A03D0F
:10491000D1F8BC10CDF82D1004F57F606946CDF8B4
:1049200031304DF0A7FC0EB070BD00BF982C0020B8
:1049300030B587B01622044600216846AAF0D0FBA5
:10494000A3238DF8003095238DF8013002238DF8D4
:10495000023080F075FC04F5A045CDF80300204638
:10496000CDF8071004F0F8FBD5F8FC330393144B93
:104970008DF80B001B68D86A90F89C308DF81030C9
:104980000368DB69984795F8E1338DF812308DF8AC
:10499000110024F067F823F0B5F9D5F8F8338DF855
:1049A00013008DF81430162295F8E2338DF8153087
:1049B000694604F57F604DF05DFC07B030BD00BF77
:1049C000942C002010B58AB02722044600216846A6
:1049D000AAF086FBA3238DF8003095238DF80130D3
:1049E00009238DF8023080F02BFCCDF80300042061
:1049F000CDF807105BF0A8FC10EE103A1320CDF8AC
:104A00000B305BF0A1FC10EE103A4620CDF80F30D1
:104A10005BF09AFC10EE103A1520CDF813305BF0E5
:104A200093FC10EE103A0320CDF817305BF09CFC9D
:104A300010EE103A1A20CDF81B305BF085FC10EE1A
:104A4000103ACDF81F3004F59B433C3327221B68F6
:104A5000CDF82330694604F57F604DF00BFC0AB0B9
:104A600010BD000013B5044600F57F6001904CF0C6
:104A70001BFF01984CF0B2FF04F58053019893F9A5
:104A800020310BB14DF052F8204602B0BDE8104085
:104A9000FFF798BF7047000010B500F5804304464B
:104AA000D3F8740D03685B68984704F5005301461A
:104AB00093F8C82204F57F604DF09CFD04F59850F2
:104AC00010300DF011FB04F59070BDE810401BF0A4
:104AD0000FBF00009FED020A002245F0EFB900BFB2
:104AE0000AD7233C184B70B5044640F8043B59F0F4
:104AF000A1FE164E164B6360542560195AF050F80B
:104B000066513035B5F5557FF7D104F555705CF039
:104B10000FF804F27C75FF2384F88C3784F89437FF
:104B20000C49284645F0DAFB0B4B1A6812B10B48CA
:104B300080F04CFB1D6001232046094984F8C137F1
:104B400045F0CCFB204670BD083900206C900C0865
:104B500080900C08F8C90D0884980020447D0C084A
:104B600068800C082DE9F04100F50D519AB00D2236
:104B7000043104464BF050FF0022BF48BF4E2721AE
:104B800045F014F9042100205BF0ACFF1321012053
:104B90005BF0A8FF462102205BF0A4FF1521032053
:104BA0005BF0A0FF5BF00AFD45F09EFDB44A138860
:104BB00043F0040313804FF000080AAF00211022D5
:104BC0003846AAF08DFA01238DF830303388ADF8DD
:104BD000283005A973680B93384644F0EFFFC8B13D
:104BE0009DF91430002B15DD59F0A4FF9DF8141029
:104BF000036801391B68C9B2984758B1051D28469A
:104C000044F026FF30B9B368ADF8183006A928463D
:104C100046F008FA08F10608B8F12A0F06F10C066A
:104C2000CCD1984800220DF10B0144F0F9FC06ADFF
:104C3000064620B344F00CFF08BB934B0FCB85E82E
:104C40000F0004A9284644F0B9FF002840F03C8139
:104C50004FF004088D4B0FCB87E80F0005A93846AD
:104C600044F0ACFF28B105A844F0F2FE08B148F0CA
:104C7000010803A930468DF80C8046F081F9844B79
:104C80000FCB85E80F0003A9284644F097FF0028C2
:104C900046D00998002204A944F0C2FC0646002828
:104CA0003ED044F0D5FE0546002839D19DF80C30A1
:104CB000013BDBB2032B96BF764A0346D35C8DF8EB
:104CC00028303046394646F05BF97348002205A982
:104CD00044F0A6FC064668F0F9F978B168F0F4F9FA
:104CE00090F8302090F8281090F84830114490F84F
:104CF00040200A44D34214BF0125002586B1304626
:104D00009DF90C8044F0A4FE50B91DB1B8F1000526
:104D100018BF0125394630468DF8285046F030F945
:104D200004F50F500022B7EE000A0121203045F0B3
:104D3000C5F804F50D500022B7EE000A02213C3000
:104D400045F0BCF8012304F5FF510093534A0023BA
:104D500018318E2045F02EF894F9A4C9BCF1000F4B
:104D60001AD14F4E0FCE3D460FC50FCE0FC50FCEF9
:104D70000FC596E80F0085E80F006246042138460B
:104D800045F014F89FED470A474845F047FE47486D
:104D9000B7EE000A45F042FE012504F50651444AEB
:104DA00000950023303140F2051045F003F804F57A
:104DB0000E5002213030FFF78DFE04F50C50032118
:104DC0001830FFF787FE04F50C5003212030FFF761
:104DD00081FE04F50E5003212C30FFF77BFE04F515
:104DE0000E5002213430FFF775FE04F50C500221FD
:104DF0002C30FFF76FFE04F50C5002213030FFF726
:104E000069FE04F50C5002212830FFF763FE04F51B
:104E1000BB4050307EF09EF9264A1368D90709D46A
:104E20002549156004F5055318330B6004F58853C4
:104E30000433CB6004F50F501F49022230300125A6
:104E400045F00AF81D4A0095002304F57F61FD2016
:104E500044F0B0FF1A4B1A68D20705D4194A1D60F6
:104E600004F59154143414601648012145F010F8EB
:104E70001AB0BDE8F08100BFA47D0C0814800C08B6
:104E8000948E0020687D0C080C330C081C330C0831
:104E90002C330C08A07D0C08737D0C0860A40C0852
:104EA0003C330C0800000000807D0C088F7D0C084E
:104EB0002CC50D088C2C0020002200208C350D08FC
:104EC000902C00201822002004A844F0C1FD0028E6
:104ED0003FF4BEAE4FF00C08BCE600BF00207047A8
:104EE0000020704700207047002070470020704766
:104EF00070470000002070470020704784B001A870
:104F000080E80E0004B000207047000000207047C9
:104F1000704700001020704700487047908C0C08C4
:104F200000487047A08C0C080020704770470000B4
:104F30000120704701207047002070470023436024
:104F40008360C36003614361002303767047000000
:104F500010B50446FFF7F2FF0023637610BD000092
:104F6000027E531CDBB2042B037600EB820288BF67
:104F7000002382ED010A88BF0376704710B504460E
:104F8000FFF7EEFFD4ED017A9FED107A94ED020A5F
:104F9000637E77EE877A042B77EE807A94ED030AAE
:104FA00094BF0133052377EE807A94ED040A63768B
:104FB00077EE807A637E94ED050A77EE807A00EED4
:104FC000103AB8EEC00A87EE800A10BD000000005B
:104FD00003F000BE03F026B803F070BA03F030B857
:104FE00001F090BC01F018B801F0B6B901F0FCB9BD
:104FF000FDF7C0BBFDF754B870B51F4B036000F55B
:1050000040530446D3F83C051C4AC3F8802308B13A
:1050100013F0A0FA1A4B236004F5805393F8942FF1
:1050200042B9D3F8905F2DB1284620F067FF28469B
:1050300013F08CFA04F59050183077F0F5FB04F576
:1050400089505CF0F3FF04F6F44504F69446B5424B
:1050500004D0183D284620F0A7FBF8E7094BC4F818
:10506000C83804F6C41050F091FA04F5136050F0FB
:105070008DFA204670BD00BFCC730C0898500D0807
:10508000802E0D0818F70C0838B54C4B044640F834
:10509000043B61F01FFA04F1100010F0A1FA04F1D2
:1050A000680049F01BFC04F590701AF0DBFF04F572
:1050B0008C600EF077FF04F2845013F04DFA04F682
:1050C000C80021F07FFF04F5476060F0E1FF04F5C0
:1050D000546046F04BFA04F57F604CF0FFFF04F596
:1050E0008850043066F02CFF04F589505CF086FF90
:1050F00004F58A501C3011F0D3FF04F5905018309D
:1051000077F07EFB04F59150143049F0A9FF04F5C7
:105110009450083062F0BCFB04F580530025284A07
:1051200083F8AC5204F5955004F595530C331C30BC
:10513000136041F057FA04F59850294610300BF0EF
:10514000ADF804F5CB5071F067FC04F5F150043074
:1051500074F076FB04F5F9501C3076F0ABFC04F5E6
:10516000FD5077F0E1F804F5FF5018300AF0FAF836
:1051700004F50550183072F031F904F5065030305E
:1051800067F07AFA04F50950303077F0D5FE04F56F
:10519000005304F50B5083F8C8520A4D203077F0C5
:1051A000EDFF2B6813B1084880F010F8204607493E
:1051B00045F094F82C60204638BD00BF802E0D08C5
:1051C000EC970020F08E0020A88C0C08882D0D088C
:1051D0002DE9F04F2DED028B04469FB0FFF754FFF1
:1051E000E44B236004F50F503030FFF77BFC04F5EF
:1051F0002E50343004F5005779F074FB04F50E534B
:105200000E33C7F8DC3B04F53050062387F8E03B4B
:1052100008305CF005FB04F5BB435033C7F8883C0D
:105220000E934FF40063C7F88C3C5A2387F80C3D6B
:1052300004F50C5807F5476304F5985608F108087B
:10524000CD4ADFEDCE8AC7F8848C1036C7F8806C63
:10525000B7EE008AC3F8602104F53950C84AC3F894
:105260006821C3F8CC2183ED578AC3ED598A0C30ED
:1052700050F0ACFC04F5395004F5315A183050F0B8
:10528000A5FC4FF00009BF4BC7F8683E0AF1300A91
:1052900087F8809E0AF5FC70FFF750FEBA4BBB49B9
:1052A000C7F8683E87F8819E504645F017F8B84B1E
:1052B000C7F8883E07F688630022C7F88C6EC7F8E7
:1052C00090AE04F53A555A63DA6304F53B50012376
:1052D00087F8CC3E0835203012F02EFD87F8F09E7E
:1052E000AC49284644F0FAFF04F53B5041463430BF
:1052F00079F0AEFE04F5415041460C3079F00CFBDC
:1053000004F54650414604F5405724307AF06AFAD5
:105310002C22494607F55270A9F0E2FE04F54C50E4
:105320009D49183044F0DAFF04F54E599B4BC7F8FD
:10533000803309F114007EF097FE04F5505309F113
:10534000380B1C3358460F9355F038FA0F9B0BF16E
:10535000140B5B45F6D10723C7F840350023A7F8A7
:1053600044354FF4CB7013F0EFF8C7F83C0504F563
:10537000555008307EF078FE04F556500C307EF023
:1053800073FE874B1A680AB9C3F80090854BC7F8BB
:10539000803304F556504FF48051C7F8A8552C308F
:1053A00010F020FA04F558502C3042F095FC04F52A
:1053B00059502C3045F0ECFE04F55A5069F0AAFB28
:1053C00004F5994004F580451C3004F08BFA764BC7
:1053D000C5F89C3C04F59940243004F083FA734BE3
:1053E000C5F8A43C04F599402C3004F07BFA704BCE
:1053F000C5F8AC3C04F59940343004F073FA6D4BB9
:10540000C5F8B43C05F6C843002204F59940DA60BB
:105410009A605A6083ED008A5C3004F063FA664B50
:10542000C5F8DC3C04F59940643004F05BFA634B4A
:10543000C5F8E43C04F599406C3004F053FA604B35
:10544000C5F8EC3C04F59A4004F04CFA5D4BC5F805
:10545000003D04F59A40083004F044FA5A4BC5F870
:10546000083D04F59A40203004F03CFA574BC5F84B
:10547000203D04F59A40283004F034FA544BC5F826
:10548000283D04F59A40303004F59A4904F02AFA90
:1054900009F13C094F4BC5F8303D484604F022FA6B
:1054A0004D4BC5F83C3D04F59A40443004F01AFADF
:1054B0004A4BC5F8443D04F59A404C3005F0AEFF28
:1054C000FE2385F8803D052385F89C3D4FF0FF3B8A
:1054D000434BC5F8749DC5F8789DC5F8A4BD1193DC
:1054E00005F6BC553F4B85ED008A04F59B402246EE
:1054F0004FF4007100934030394B109404F5A045EF
:105500000FF04CFB0023C5E9EF33C5E9F133C5E9E2
:10551000F3330323C5F8F83305F21443C5F864B335
:10552000C5EDE08A83ED008A2F4BC5F83C342F4B44
:10553000C5F8443404F5A8402D4BC5F84C34C5F8E3
:105540003844C5F84044C5F84844603012F0F4FBD4
:1055500004F5A8407C3012F0EFFB04F5A94004F5F7
:10556000A849183012F0E8FB09F11C09214BC5F8D5
:10557000AC3441E0CC730C08000080BF0000B442A2
:105580000000B4C2148D0C08248D0C084C060E08C3
:10559000C0030E0868030E0804FE0D0898500D089D
:1055A0003892002028410C08D0960C08B49A0C08B8
:1055B0009C9C0C0824950C08D8970C085C980C0847
:1055C00044970C0854960C08D4950C083C9A0C0887
:1055D0004C990C08D8980C084C8D0C08C8990C08EC
:1055E000D14F0108FC3D0C08D54F0108D94F0108E7
:1055F000DD4F01080000FFFFA5F8B0B409F19800E5
:1056000012F09AFB6F4B7049C5F810B54846C3F8C5
:10561000009044F063FE4FF6FF73A5F8583404F58C
:10562000AA406A4B6A49A5F874B41430186044F073
:1056300055FE04F5AA4034304AF0E2FD654BD7F838
:10564000A8251294CDE91334634BCDE91534634B8F
:10565000CDE91734624BCDE91934624BCDE91B34E7
:10566000614B1D931EA911E903000CAB83E80300F5
:10567000DDE91A010AAB83E80300DDE9180108AB94
:1056800083E80300DDE9160106AB83E80300DDE9EA
:10569000140104AB83E80300DDE9120102AB83E8E7
:1056A0000300CDE900284946324653460E9804F5DA
:1056B000BC487DF057FB08F15C084C4BC5F85C3EDC
:1056C00008F13C0012F038FB4949404644F006FE20
:1056D000484B1F6817B148487FF078FDC3F8008039
:1056E00006F51B76454BC5F85C3E04F5BD40C5F894
:1056F000E46E85F8607E85F8657E85F8897E683081
:1057000012F01AFB04F5BD40783012F015FB04F5D9
:10571000BE40083012F010FB04F5C0481C22394688
:1057200005F61870A9F0DCFC08F1040804F5BF4088
:105730005CF0B2FD04F5C046404677F0D9FD304B31
:1057400030497360404644F0C9FD2F4A2F4911602B
:1057500033463C334FF0140CB8B20CFB0012013747
:10576000127C002AF8D12A4A10802A4A17680FB101
:105770002948B1E704F5C0404030136077F0A2FD3E
:10578000264B3364264B3365642386F85430254B0F
:10579000C6F8883004F5C040234BC6F88C30234946
:1057A000503044F09BFD224B336520460123C6F860
:1057B000B07086F8B87085F8A4331FB0BDEC028BCA
:1057C000BDE8F08FD48D002074040D08F4970020FC
:1057D000E0660D08E14F0108E54F0108E94F0108B7
:1057E000ED4F0108F14F0108F54F0108FC8C0C0842
:1057F000E4010E0808A00020BC8C0C08A4900C0842
:10580000A4370C087C370C08A88E002018820C08DE
:10581000A48E0020608E0020D88C0C08E4370C0881
:10582000348D0C08ACA00C0804A10C0804580D0819
:1058300084A20C0810B57FF001F8064C064B1860E6
:105840002046FFF7C5FC2046044A0549BDE8104044
:10585000A6F0D8BE982C0020942C002050F00020F8
:10586000F94F01080069C0F3401070470F299DBF30
:10587000302303FB0100503000207047014B93F9A7
:105880008D037047984C0020014BD3F8C80B70472C
:10589000984C002008B503689B68984730B9044BC2
:1058A00093F88E0DB0FA80F0400908BD0020FCE7A7
:1058B000986C002008B5044806F0C0FD10B9034BF1
:1058C00093F8880D08BD00BF982C0020986C00202C
:1058D000022A10B50C4605D1BDE810400948352212
:1058E00008F04EBC084BD3F8740D03685B6898470A
:1058F000A04205D159F01EF9BDE8104059F0A4B8F6
:1059000010BD00BF982C0020986C0020012910B514
:105910000C4614D0022907D0D1B90E4BC3F8B010F1
:1059200057F016FC0C4A05E00A4BC3F8B01057F0CC
:105930000FFC0A4ABDE81040062150F03DBD57F06B
:1059400007FC074A062150F037FD024BC3F8B04070
:1059500010BD00BF988C0020638E0C08388E0C0898
:105960004C8E0C08012902D0022900D011B9024B3B
:10597000C3F8B410704700BF988C0020622910B49F
:1059800000F3888047291ADC402900F0958008DC64
:10599000162951DC032904DD4F4B01248C402340A0
:1059A00053B95DF8044B59F097BFA1F19604012358
:1059B000A3404A4C2342F4D05DF8044B7047A1F158
:1059C00048031A2BEDD801A454F823F0B959010863
:1059D000A3590108A3590108A3590108A3590108B3
:1059E000B9590108A3590108A3590108A35901088D
:1059F000A3590108A3590108A3590108A359010893
:105A0000A3590108AF5A0108AF5A0108AF5A01085B
:105A1000B9590108A3590108AF5A0108B959010839
:105A2000A3590108A3590108B9590108B959010836
:105A3000A3590108B9590108A1F12703112BB0D8C6
:105A4000112BAED801A454F823F000BFB9590108B6
:105A5000A3590108A3590108A3590108B95901081C
:105A6000A3590108A3590108A3590108A359010822
:105A7000A3590108A3590108A3590108B9590108FC
:105A8000B9590108A3590108A3590108B9590108D6
:105A9000B9590108B02904DC952986DC6B2980D12D
:105AA0008AE7A1F1D003022B3FF67BAF84E75DF8D4
:105AB000044B002359F0E2BE094B012283F8AC20CD
:105AC000A3F58043D3F8C40B00283FF475AF5DF80D
:105AD000044B642159F074B810004100A100800407
:105AE000988C002038B50B46622B0446114600F313
:105AF0009580472B13DC382B7ADC262B4CDC102BC3
:105B000000F0B680162B00F00781042B00F0C78050
:105B10000A4620461946BDE8384059F01BBCA3F19F
:105B200048021A2AF4D801A050F822F0795C010842
:105B3000115B0108115B0108115B0108115B010891
:105B4000A35C0108115B0108115B0108115B0108EE
:105B5000115B0108115B0108115B0108115B010871
:105B6000115B0108AF5C0108EF5C0108115B0108E3
:105B7000115D0108115B0108F75C0108A95C0108CF
:105B8000115B0108115B01085F5C0108255D0108DC
:105B9000115B0108875C0108A3F12702112AB7D81D
:105BA00001A050F822F000BF5F5C0108115B010802
:105BB000115B0108115B0108635C0108115B0108BE
:105BC000115B0108115B0108115B0108115B010801
:105BD000115B0108115B0108995C0108815C0108F7
:105BE000115B0108115B0108935C01088D5C0108E1
:105BF000402B8DD1931E5942644C594184F8AB100F
:105C000057F0A6FA624A94F8AB10624B002908BF1D
:105C10001346614A062150F0CFFB20E09B2B00F099
:105C20008E8007DC6B2B00F09480962B7FF470AF96
:105C300007211EE0AD2B7AD00CDC9D2B7FF468AFE2
:105C40000124002A00F08180022A5BD14F4B83F8A7
:105C5000AA4057E0A3F1D002022A3FF659AF01242F
:105C600050E08A1E4D4B5142514183F8811DF6E7A9
:105C70000A21FFF72DFEF2E70A4601212046F8E748
:105C80000A460421FAE70A460321F7E70A460C21EF
:105C9000F4E70A460F21F1E70A460021EEE70B215F
:105CA000E7E70A460D21E9E70A460521E6E7374C12
:105CB000D1B102290DD1012384F8A830A4F50053F5
:105CC000D3F8740D03685B6A984710B1344800F04C
:105CD000A5FD57F03DFA334A94F8A810324B00293D
:105CE00008BF1346314A95E784F8A810E6E7204636
:105CF000FFF70CFEB3E7012431B1022902D12C4B8E
:105D000083F84441204638BD294B83F84411F9E714
:105D10002046FFF727FEA2E7022AA0D1204806F07E
:105D200035F99CE758F006FF58F08EFE97E7022AF7
:105D300095D19FED200A1A48FCF70AFA8FE7022A4C
:105D40008DD1174806F08AFA89E7104B83F8AA200C
:105D5000D8E7022A14D1114DD5F8740D0368DB6B16
:105D60009847044628B10121A5F5804002F0ACFC1B
:105D7000C8E757F0EDF9104A042150F01DFB6EE71B
:105D80000748002102F0A0FC69E700BF988C0020C2
:105D9000788E0C085F760C08808E0C08986C0020BA
:105DA000982C0020BB610C081C9B0C08908E0C08E2
:105DB000984C002000000000A38E0C0810B5084C81
:105DC000D4F8740D03689B6B984738B9D4F8740DF8
:105DD00004F64454001B18BF012010BD0220FCE74C
:105DE000986C002008B5022103205AF0C5FD02215D
:105DF00008465AF0C1FD012104205AF0BDFD0221E0
:105E000015205AF0B9FD132002215AF0B5FD1248B1
:105E100006F07EFDA8B1002146205AF0ADFD00211C
:105E200049205AF0A9FD00214A205AF0A5FD002181
:105E300001205AF0A1FD0021BDE8084008465AF0B3
:105E40009BBD012146205AF097FD012149205AF0BF
:105E500093FD0121E8E700BF982C00200249034888
:105E6000052208F0B3B800BFA0790020982C0020CC
:105E700038B5304B01241C7090F90A302B2B0CD113
:105E80002D487DF065F92D4807F07EFEBDE83840CD
:105E90002B4801220921FBF77BBD284D9FED290AE4
:105EA000D5ED460A642103205AF030FBD5ED460AB1
:105EB0009FED240A642102205AF028FB9FED220A5C
:105EC00003205AF02DFA9FED200A02205AF028FAFA
:105ED0009FED1E0A04205AF023FA9FED1C0A15209C
:105EE0005AF01EFA13209FED190A5AF019FA2846A3
:105EF00006F00EFDA0B1002146205AF06BFD0021F6
:105F000049205AF067FD00214A205AF063FD002124
:105F100001205AF05FFD002108465AF05BFDB2E710
:105F2000214646205AF056FD214649205AF052FD9E
:105F30002146E9E798920020688A0020982C0020EA
:105F40009C8C0020000000000000C84200A08C458E
:105F500000F58040D0F8740D03681B6C18470000F2
:105F600000F5005393EDEB7A00F5A040B5EEC07A52
:105F7000F1EE10FA5DBFD0F8E43EDFED086AD3ED34
:105F8000017AD0F8FC0E5FBFF8EEE77AE7EE267AEA
:105F9000FDEEE77A17EE900A704700BF0000C84296
:105FA00000F5005090F8EC0328B141F001010842DF
:105FB00014BF01200020704713B50346FFF7F0FF20
:105FC00058B103F5005191F8E41BC90705D503F555
:105FD000305393ED000A02B010BD03F5A04422B97E
:105FE00004F6347494ED000AF5E794F8CC2D022AF7
:105FF000F6D103F5AA40012201A934304AF086FA0D
:106000000028EDD09DED010AE5E7000000F5A04372
:1060100093F8202FFFF7D0BF10B54B68516800F5FB
:10602000A0448B42D8BF0A46D4F8180FCCBF1A46FA
:10603000194623F0EFFAC4F8180F10BD10B5044646
:10604000564866F075FC10F0080217BF544BDFEDA0
:10605000557A93ED6F7AD3ED717A1FBF77EE877A19
:106060009FED517A012267EE877A10F0010317BF86
:106070004B4B9FED4C7AD3ED716A93ED6E7A1CBF5A
:1060800037EE667ADFED486A04F5005118BF27EE57
:10609000267AD1EDED6AF5EEC06A18BF0123F1EE64
:1060A00010FA3CDD3E4A9FED406AD2EDED6A66EEA5
:1060B000866A0122F4EE676AF1EE10FA58BFF0EE3C
:1060C000667A04F5A04090F8201F69B393B1D0F828
:1060D000243F06EE903AF8EEE66AF4EEC76AF1EE77
:1060E00010FA58BFF0EE476AFDEEE66A16EE903AF7
:1060F000C0F8243FBAB1D0F8243F07EE103AB8EE0A
:10610000C77AB4EEE77AF1EE10FAD8BFB0EE677A4C
:10611000BDEEC77A17EE103AC0F8243F03E0002A1C
:10612000CFD1002BCDD110BDD3B1D0F8E43ED3ED0B
:10613000016AD0F8183FF8EEE66A76EE876A07EE55
:10614000103AB8EEC77AF4EEC76AF1EE10FAD8BF8B
:10615000B0EE667ABDEEC77A17EE103AC0F8183F77
:10616000002AE0D0D0F8E43E93ED017AD0F8183F51
:10617000B8EEC77A77EE277A07EE103AB8EEC77A0C
:10618000F4EEC77AF1EE10FA58BFB0EE677ABDEEC2
:10619000C77A17EE103AC0F8183FC4E7484E0020FF
:1061A000984C0020000000000000C84200F5A0400C
:1061B0000023C0F81C3F704773B516460546002300
:1061C0006A463046009311F0A5FE48B1DDED007A35
:1061D0009FED287A67EE877AFDEEE77A17EE900A50
:1061E00005F5A044C4F81C0F33785B071CD594F860
:1061F000203FCBB105F5AA40012201A934304AF075
:1062000085F988B1D4F8243FDDED016A9FED197A54
:1062100007EE903AF8EEE77AE6EEC77AFDEEE77A17
:1062200017EE903AC4F81C3FD4F8F833042B1FD073
:1062300005F50055B5F9E623002A16DDD4F81C3F14
:106240009FED0D7A83EAE371A1EBE37107EE901AFB
:10625000F8EEE77A67EE877A07EE102AB8EEC77A8B
:10626000F4EEC77AF1EE10FA02D50023C4F81C3F11
:1062700002B070BD0000C8420AD7233C37B50B7886
:106280005A0704460D461DD500F5AA40012201A972
:1062900034304AF03BF9A8B1D5ED017A2B78DFED27
:1062A0001C6AF8EEE77ADB0767EEA67A1BD59DED50
:1062B000017AB4EEE77AF1EE10FACCBF01200020AB
:1062C00003B030BD2B78D5ED017A13F0010FF8EE55
:1062D000E77A04F5A04411D104F6FC6393ED007A4B
:1062E000B8EEC77AE5E704F5A044D4F8E43E93EDB0
:1062F000017AB8EEC77AE7EE667AD8E7D4F8E43EDA
:1063000093ED017AB8EEC77A77EE877AE4E700BFBB
:106310000AD7233C00F5005300F58042B3F99633C9
:10632000D2F8742D00EE103A00F59A4308339A42E1
:10633000B8EEC00A0ED100F5A040D0F8F833042B17
:1063400002D090F8A5332BB100F55D60D0ED007A56
:1063500030EE270A70470000014608B501F5A0415C
:10636000FFF7D8FF01F6FC63D3ED007A9FED057AC5
:10637000F8EEE77AE0EE477AFDEEE77A17EE900A5C
:1063800008BD00BF0000C84237B500F5A04504466F
:1063900095F8203FFBB100F5AA40012201A9343055
:1063A0004AF0B4F8B8B105F62472D2ED007A9FED48
:1063B0000D7A05F62873D3ED006AF8EEE77AE6EE7B
:1063C000877ADDED016AE6EEC77AFDEEE77A17EE31
:1063D000900A03B030BD2046FFF7BEFFD5F8183F46
:1063E000181AF6E70000C842014608B5FFF792FF09
:1063F00001F5BE40D0ED0D7A37EEC00ADFED047A2C
:1064000020EE270AFDEEC07A17EE900A08BD00BF05
:106410000000C8422DE9F04100F5BD4800F5BE4539
:1064200008F17808083504462946404611F0E6FF91
:1064300004F5BD4604F5A04768362A463146404675
:1064400087EDE30A11F010FFDFED220A87EDE40A81
:10645000B7EE001A762023F03DF804F5315383EDB2
:106460007D0A2046FBF71CFE04F58043D3F8740D2B
:1064700003685B6898470B280BD006D80A280FD012
:106480000023C7F81C3FBDE8F0810E38C0B20128D8
:10649000F6D829462046FFF7F1FE0028F0D011E09B
:1064A00029462046FFF7EAFE30B90B484FF48041F9
:1064B000FCF762F80028E3D12046FFF795FFB0F51E
:1064C000FA6FE6DD2A4631462046BDE8F041FFF787
:1064D00073BE00BF00000000982C002010B52DED09
:1064E000028B00F5A043DFED1F8AD3F80C2F93F841
:1064F000083F07EE902ADA0758BF00F5AC52B8EE15
:10650000E78A58BFD2ED007A28EE288A58BFF8EE05
:10651000E77A82B058BFA7EEE88A5B0704460FD53A
:1065200000F5AA40012201A9343049F0EFFF38B14B
:106530009DED010A30EE480A02B0BDEC028B10BDA1
:106540002046FFF709FF04F5AC5393ED000A07EE70
:10655000900AB8EEC00AF8EEE77A28EEC00AA7EE75
:10656000A80AE7E70AD7233C38B52DED028B00F5E2
:10657000804200F59943D2F8742D64339A42044660
:106580004DD100F58053D3F8105500F50053B3F901
:10659000E433002B66DD04F5B85292ED057AF7EE90
:1065A000007AB4EEE77AF1EE10FA5BD404F53252D9
:1065B000D2ED067AF6EE006A67EEA67A87EE871AC3
:1065C000B5EEC01AF1EE10FA4CD907EE905A9FEDD5
:1065D000288AB8EEE70A07EE903A04F5AA4004F5D7
:1065E000A044F8EEE70A20EE080A34304AF09AF8A0
:1065F000D4F81C3F9FED1F1ADFED1F0A002BBCBF14
:1066000007EE903AF8EEE77A4FF42970B8BFA7EE9C
:10661000880ABDEC028BBDE8384022F05BBF05F074
:1066200053FBF8B904F54053D3F8A80503681B6978
:10663000984704F50053DFED100AB3F9E43301EE97
:10664000103A04F5A04393EDE30AB8EEC11A0546EB
:1066500040F27F2022F03EFFBDEEC00A10EE103A5D
:106660001BB296E7BDEC028B9FED030A38BD00BF5D
:106670000AD7233C00007A440000000010B504460D
:106680007EF0D6FD04F50053D3F8F82B801A41F2C2
:10669000883290420FD802212046FFF781FC50B18A
:1066A00004F5A044D4F8F823042A04D103F6EC330B
:1066B00093ED000A10BD9FED010AFBE7000000000A
:1066C00030B52DED028B00F5A045DFED298A95F858
:1066D000203F83B004467BB3D5F8243F9FED250AC5
:1066E00007EE903AF8EEE77A00F5AA4027EE800A26
:1066F000012201A9343049F041FFE8B12046FFF7FB
:1067000033FFDDED017A05F6287585ED000A37EED9
:10671000800A20468DED010AFFF7B0FFDDED017A1A
:1067200030EE270A20EE280ABDEEC00A10EE100A4D
:1067300003B0BDEC028B30BDD5F8E42ED5F8183F80
:1067400052689B1A08EE103A2046FFF7E3FDB8EEB8
:10675000C88A2046A0EE288AFFF790FFBDEEC88ABF
:10676000B8EEC88AA0EE288ABDEEC80ADEE700BFF0
:106770000000C8420AD7233C10B500F58043044608
:10678000D3F8740D03685B6A984718B104F5C044E8
:1067900094F8A80010BD000038B500F5A0440D46DF
:1067A000D4F8183F0B44C4F8183F94F8203F3BB18D
:1067B000FFF7E2FF20B9D4F8241F2944C4F8241FAE
:1067C00038BD000030B500F50050D0F8E023D30705
:1067D0000FD4094B08201D785C688D4204D12242F9
:1067E00014BF0120002030BD013803F10803F2D1AD
:1067F000F9E70120F7E700BFF4900C0810B500F5A9
:1068000080430446D3F8740D03685B6898470146DB
:106810002046BDE81040FFF7D5BF000037B500F5B2
:10682000A0440546D4F8FC3EC4F8183F0023C4F841
:106830001C3FFFF7E3FFE0B105F5AA40012201A9E3
:10684000343049F063FEA0B12846FFF795FF80B9C8
:10685000DDED017A9FED097A67EE877A0123FDEE7F
:10686000E77A84F8203F17EE903AC4F8243F03B04B
:1068700030BD002384F8203FF9E700BF0000C84284
:1068800038B504460D46FFF7B9FF30B1032128465D
:1068900011F01CFB80F00103D8B204F5A04484F889
:1068A000210F38BD73B500F5A0444A68C4F8182F0D
:1068B0000B780D46D90741BFD4F8E43E5B689B18BE
:1068C000C4F8183F94F8213F064623B100F5BE41B5
:1068D0000831FFF7D5FF2B785B070FD506F5AA40E7
:1068E000012201A9343049F011FE38B1012384F8A6
:1068F000203F6B68C4F8243F02B070BD002384F8C9
:10690000203FF9E7F0B52DED028B044683B004F586
:10691000A0450E468DED010AFFF7C4FFDFED360AF4
:106920009DED010A40F24310B7EE001A22F0D2FDAD
:10693000D5F81C3F5B4207EE903AF8EEE77A204626
:1069400067EE807A04F50057FDEEE77AB0EE408AF4
:1069500017EE901AFFF720FFD7EDFA7AF5EEC07A1E
:10696000F1EE10FA43DDD5F81C3F002B3FDD204649
:10697000FFF70AFD07EE900ADFED206AB8EEE77A2E
:10698000D7EDFA7A67EEA67AB4EEE77AF1EE10FA6E
:106990002DD531462046FFF785FF04F5BD4132462F
:1069A00078312046FFF708FCD5F81C3F5B4207EE24
:1069B000903AF8EEE77A204667EE887AFDEEE77ABD
:1069C00017EE901AFFF7E8FEB5EEC08AF1EE10FA66
:1069D0000DDDD5F81C3F07EE903AB8EEE77AC7EE2A
:1069E000087AFDEEE77A17EE903AC5F81C3F03B03F
:1069F000BDEC028BF0BD00BF000000000000C8C26B
:106A0000F0B500F5A04487B094F8083F03F0050303
:106A1000052B07460BD04AF0FBFD4FF4AE724FF446
:106A200080114AF0ADFD0025284607B0F0BD1E4894
:106A30006A46032111F05AFA0028F4D01B4801AA33
:106A4000032111F053FA05460028ECD0184BDFED76
:106A5000190A93EDE40A40F26D10B7EE001A22F025
:106A600039FD04F608730FCBB0EE401A02AEDFED2D
:106A7000111ADDED010A9DED000AB7EE002A86E845
:106A80000F0022F059FCDFED0C7A20EE270A304689
:106A9000FDEEC07A032217EE901A11F053F9314639
:106AA0003846FFF7FFFEBFE7808B0020A08B002059
:106AB000987C0020000000000000C842F7B50D4699
:106AC00002210446FFF76CFA60B304F5A047D7F83B
:106AD000F833042B26D12046FFF790FE10B304F5BF
:106AE000AA46343604F5BD4101236A467831304662
:106AF00049F0F6FBB0B104F5BE41012301AA08310B
:106B0000304649F0EDFB68B19DED017ADDED007A8C
:106B100077EEC77A95ED007A37EE277A85ED007A21
:106B2000C7EDEC7A03B0F0BDF0B52DED048B00F5A8
:106B3000005489B000F5546794F8B21B03910546E0
:106B4000384644F0E3FD03990646384644F0F0FD2C
:106B5000042E0399B0EE408A20D1002305A88DEDC4
:106B6000050A0693079325F045F805F5B15005A9E8
:106B7000103022F061FFDFED957A8DED050AB4EE5D
:106B8000E71AF1EE10FACDED060A8DED071A05DBD6
:106B900005F5805393F88C35DE070CD494F8E43B6C
:106BA000002262F3000384F8FC2B84F8E43B09B074
:106BB000BDEC048BF0BD94F8E43B98075CBF43F058
:106BC000020384F8E43B05F530565CBF04F6E83375
:106BD00083ED008A314686ED001A2846FFF76EFFE6
:106BE00094F8FC3B092B00F2878004F60443D3EDB4
:106BF000000A9FED779AB0EE480A22F059FB00BBDD
:106C000004F6E83394F8B21BD3ED008A384644F01A
:106C1000ADFD07EE900A9FED6F7AF8EEE77A78EE19
:106C2000C88A67EE877AF0EEE88A67EE897AF4EE32
:106C3000E78AF1EE10FAC2BF94F8FC3B013384F806
:106C4000FC3B04F6044394F8B21BD3ED008A3846AB
:106C500044F08CFD07EE900AF8EEE77A9FED5E7A3D
:106C600067EE897A78EEC88A67EE877AF0EEE88A6E
:106C7000F4EEE78AF1EE10FA02DD002384F8FC3B23
:106C800004F6044383ED008A94F8E43BDA078ED5DA
:106C9000284605F5A047FFF721FC96ED008A97F8F6
:106CA000203F30EE488A002B4BD005F5AA40012248
:106CB00005A9343049F02AFC002848D17EF0B8FA02
:106CC000D4F8F82B41F28831821A8A42034604F63E
:106CD000EC3204F53F6141D982ED008A284681ED0E
:106CE000008A0221FFF75CF918B107F55D67FA68C1
:106CF000BA60C4F8F83B5AE794F8E43B43F0010368
:106D0000590784F8E43BBBD405F5A042D2F8F82338
:106D1000042AB5D102212846FFF742F90028AFD056
:106D200043F0040384F8E43B3068F9F7EDFB05F524
:106D30004E57CDE90001294A062138464FF03CFB69
:106D40009EE72846FFF75AFD0028AED1B6E796ED3C
:106D5000000A9DED058A38EE408AAFE79FED1E0AD6
:106D600092ED007ADFED1E7A28EE008AA7EE278AE0
:106D700082ED008AC4F8F80BD1ED007A38EE678A0C
:106D8000F3EE0E7AB0EEC88AB4EEE78AF1EE10FAAE
:106D90007FF70DAF94F8E43B5B070BD53068F9F74C
:106DA000B3FB05F54E54CDE900010E4A06212046FD
:106DB0004FF002FB242205F52F500021104409B0AA
:106DC000BDEC048BBDE8F040A8F08AB900000034A7
:106DD0000AD7233CCDCC4C3DCDCC4C3EB4900C08D6
:106DE000CDCC4C3FD1900C0838B52DED028B0D4623
:106DF0000446FFF773FB002320462B70B0EE408A59
:106E0000FFF73CFC0221204638EE400AFFF7C8F8A5
:106E100028B104F5005494F8E40B00F00100BDEC37
:106E2000028B287038BD000070B50B7803F00503A5
:106E3000042B05460C46164615D105F5A0454AF02B
:106E4000E7FBB2B24FF480114AF09AFBD5F8E42E7A
:106E5000636852689B1A13F5FA7FC8BF6360237892
:106E600043F00103237070BDF8B500F5805300F5C1
:106E7000A047D3F88065D7F8B453B542044619D07B
:106E80000E4A1268D26A92F89C209AB100F5BE416F
:106E9000751B25220831FFF7C7FF07EE905AB8EEA1
:106EA000E70ADFED077A04F5315020EE270A30308B
:106EB0007BF0E0FCC7F8B463F8BD00BF942C002061
:106EC0000AD7233CF8B500F5A044054694F8A7C3BB
:106ED0000F4604F6E866BCF1000F53D004F60873C1
:106EE0000FCB86E80F00012384F8A83397E80F0042
:106EF00004F6087686E80F00D4F8103F05F5BE4684
:106F0000083693B9D4F8143F7BB9D4F8003FD4F8CD
:106F10000C2FC4F8103FD4F8043FC4F8143F22B932
:106F2000D4F8FC1E304610F00DFF314628222846CA
:106F3000FFF77AFF94F8081F11F0040102D13046E0
:106F400010F0C4FF05F5BD4105F5BD40324668317E
:106F5000783011F0BFF938B104F6E86604F6F86449
:106F600094E80F0086E80F00284604F045FB284609
:106F7000FFF750FA284604F06FFE2846BDE8F840B7
:106F8000FEF7E6BF04F6F8630FCB86E80F00012397
:106F900084F8A73384F8A8C3A8E70000F8B500F583
:106FA00000530446B3F93E33002B0E4633DB0B7817
:106FB00013F0020F14BF4FF0FF33012304F5A04577
:106FC00005F6E86785F8C03E05F6F8630FCB87E85D
:106FD0000F0096E80F0005F6087787E80F0004F524
:106FE000BE41572208312046FFF71EFF2046FFF71B
:106FF00015FC2046FFF70EFA204604F02DFE002374
:1070000085F8A833C5F8C43E85F8AD332046BDE801
:10701000F84004F0F1BA4FF0FF33CFE72DE9F04329
:10702000364B1B6885B00546D86AFAF78BFA0028FC
:1070300061D105F5005393F9603B5A1C54D0002BE5
:1070400005F58C6711DD95F87124242107EE903A3F
:1070500001FB027292ED0B7AF8EEE77AB0EEC77A96
:10706000B4EEE77AF1EE10FA3EDC05F5805305F553
:10707000985693F88C3513F0010406F1100629D0C8
:10708000C3F340089B0732D495F8141495F858447C
:107090004FF0B00909FB015191F8F1314CBB022BC3
:1070A00018D9684610F048FE694630460AF030FBB1
:1070B000044678B195F8143409FB03534246D3F8DB
:1070C0000012684610F03EFE0AF0C2FD69460AF062
:1070D0000DFA044638460DF039F830460AF024F926
:1070E0002846FBF71BFA204605B0BDE8F0830024D4
:1070F000F0E74446EEE70020F6E700BF942C0020BE
:1071000038B50C4B1B680546D86A0C46FAF71AFAD4
:1071100010B10024204638BD0AF09AFD21460AF03D
:10712000E5F904460028F4D005F5A8401C3025F008
:107130004FFBEFE7942C0020F0B500F5A0450023AD
:1071400085F8A73385F8A83305F6F863044600EE02
:10715000101A0FCB87B005F6E86686E80F0002AE7E
:1071600004F5BD42B8EEC00A30461749783244F003
:1071700017F996E80F0005F6087787E80F0004F581
:10718000BE4140F25712083120460191FFF74CFEF4
:1071900001992046FFF774FB01992046FFF782FB17
:1071A00004F500532046B3F93E33002BB4BF4FF033
:1071B000FF33012385F8C03EFFF72CF9204607B0C6
:1071C000BDE8F04004F048BD0463002010B5034959
:1071D000044644F0E5F8204610BD00BF04630020DB
:1071E000F8B500F5A04404F6F86305460E460FCB4B
:1071F00004F6E86787E80F0006F108012846FFF764
:1072000061FEB388D4F80C2F03EB830303EB8303F5
:107210009B001BB2002BD8BF4FF4C873A4F8A23355
:10722000D4F8E43E5968521AC4F874239A680A32B2
:10723000C4F8102FDB680A33C4F8143F0023C4F8E5
:10724000883384F8A43384F8B833C4F8783300233F
:10725000C4F86C334FF0FF33C4F8643395F87124ED
:1072600005F58C63242101FB0233DB6AC4F89C33EF
:10727000F8BD000070B50E4608310546FFF722FE46
:10728000B38805F5A0444BB3642213FB02F3C4F8A2
:107290007433B4F9A233002BD8BF4FF47A734FF094
:1072A000240205F52F50D8BFA4F8A23300211044C2
:1072B000A7F016FF04F6347305F5BB4093ED000A02
:1072C000314650307BF044FED4F8F833072B0CD114
:1072D00028460421BDE87040FAF794BED4F8743310
:1072E000002BD6DC40F6B833D1E770BD0B7A00F541
:1072F000A04013F0020F14BF4FF0FF33012380F8BA
:10730000C03E70477FB501F1080305460E460FCB1E
:107310006C4684E80F0005F5BD417831204610F039
:1073200075FE21462846FFF7CDFD31462846FFF77A
:10733000DDFF04B070BD00007FB501F10803044615
:107340000E460FCB6D4685E80F0004F5BD41783140
:10735000284610F05BFE29462046FFF7B3FD204685
:107360003146FFF7C3FF337907EE903A337E9B0730
:1073700048BF9FED0C7AF8EE677A04F5A04448BF49
:1073800067EE877A9FED087A67EE877AFCEEE77AF8
:1073900017EE903AC4F8B83E0123C4F8D83E04B0C2
:1073A00070BD00BF0000803B00A00C477FB501F11D
:1073B000080304460E460FCB6D4685E80F0004F522
:1073C000BD417831284610F021FE29462046FFF7BE
:1073D00079FD20463146FFF789FFB38804F5A044C4
:1073E0004FF47A725343C4F8D03E0123C4F8D83E18
:1073F00004B070BD2DE9F34100F5BE4504460835E3
:1074000000F5BD400E466830294610F0BFFD04F57A
:10741000A047C0B94FF0FF33C7F8643306F108083E
:10742000404610F0B9FC032802463AD1F1682846DC
:1074300010F088FCB388C7F8D83E204602B0BDE8FB
:10744000F041FEF7B3BE1AF0E9F9FAF76BFB012839
:1074500012D94FF0FF33C7F864331AF0DFF990F810
:10746000F432DFED150AB02202FB030090ED3C0A76
:10747000284611F039F8D1E704F58058D8F81005FE
:1074800021F0FCFF08F5A263C7F86403D3ED007A8E
:107490009FED0A0ADFED080AF8EEE77A27EE800A88
:1074A000E6E701AA0021404610F082FC0028C1D086
:1074B00001990022BBE700BF00007A440AD7233CB1
:1074C0007FB501F1080304460E460FCB6D4685E8F3
:1074D0000F0004F5BD417831284610F097FD29468C
:1074E0002046FFF7EFFC20463146FFF7FFFE04F58C
:1074F000A0440023C4F8D83E04B070BD37B504469C
:107500000D467DF095FEE060D5ED027AF5EEC07A8D
:10751000F1EE10FA15DD9FED127A67EE877AFCEE38
:10752000E77AC4ED027A55F013FEA2684FF47A733D
:10753000B2FBF3F30B4A062103B0BDE830404EF036
:107540003BBF65F043F80023009395F90D2095F9B2
:107550000E3095F90C1064F0D5FFA060E3E700BF92
:1075600000007A4434910C082DE9F0412DED028B96
:1075700084B004460AF06CFB09F0BCFC04F58053AF
:1075800004F5A04593F808380BB9002874D0D5F855
:107590006433013370D1D5F88833002B48D07DF0A7
:1075A00047FED5F88833C01AB0F5FA6F64D394F863
:1075B0001424DFED5D7A9FED5D8A4FF0B00808FB83
:1075C000024292ED840A20EE270A21F06FFFD5EDEA
:1075D000DB7A30EE670A21F069FFDFED557A20EEA5
:1075E000080A04F54E5720EE270A21F007FFFDEEAA
:1075F000C07A17EE906AC5EDD97AD5EDDB7A67EEE1
:10760000887A17EE900AF8F77FFFCDE9020194F827
:10761000143408FB0343D3F80C02F8F775FF454A0E
:10762000CDE900013346062138464EF0C5FE23E081
:1076300004F59070FAF776FA02281DD994F81434FC
:10764000B02202FB034393ED837AF1EE047AB4EEA9
:10765000E77AF1EE10FA0FDD374B1B68D86A036842
:10766000DB699847012803D07DF0E2FDC5F8880367
:10767000D5F88833002B92D104F54053D5F8641324
:10768000D3F8A8054A1C036845D01B6B98472B48C4
:1076900007F098FA20B104F5A8401C3027F034FB1D
:1076A0002046FEF7A1FED5F874338342064635DA4C
:1076B00007EE906A9FED227AF8EEE77A04F54E54D1
:1076C00067EE877A05F6E86617EE900AF8F71CFF72
:1076D0001C4ACDE90001204606214EF06DFE012432
:1076E0004FF0FF33C5F8643385F8A44305F6F8631B
:1076F0000FCB05F6087786E80F0087E80F001248E1
:1077000065F0E0F8002385F8A733204604B0BDEC0F
:10771000028BBDE8F0815B6B9847B8E7074807F03C
:1077200031FA0028C4D1F1E735FA8E3CE02E6542EB
:107730000000C84244910C08942C0020982C002092
:107740000AD7233C68910C08484E00202DE9F047E9
:1077500000F5A0462DED028B4FF0FF33C6F86433E1
:1077600006F608738C4607460FCBBCF804509CF80D
:10777000049088B004AC2D0A84E80F0020D007F5EF
:10778000BD4808F168082146404610F037FE214602
:107790004046B0EE408A10F001FDDFED557AB4EEC0
:1077A000E78AF1EE10FA0BDBEBB200EE903ADFED78
:1077B000517AF8EE600A20EE270A204610F094FE77
:1077C00007F5405A96F8A823DAF8A8059FED4A0A6B
:1077D000036807F5BD489B6A08F1780822B307F5EE
:1077E000BD4122466831984707F50052B2F96E3321
:1077F000002B1CDD07EE903A96EDE37AF8EEE77A7F
:10780000B4EEE77AF1EE10FA11DD07F5BD4122463C
:107810006831404610F05EFDF0B90025284608B0FA
:10782000BDEC028BBDE8F08722464146DBE7B9F1AB
:10783000000F1CD1002D3BD1B2F96C33DAF8A8054A
:10784000D6EDE00A00EE103A0368B8EEC00A1B6AF3
:107850009847B0EE408A0EE0002DDED106F6E864CF
:1078600006F6F86696E80F0084E80F00D6E707EE04
:10787000909AB8EE678A2146404610F0BFFDB4EEFC
:10788000C08AF1EE10FA16DBB6F85834039321469D
:10789000404610F0B3FDBCEEC00A039B174A8DEDC5
:1078A000000A062107F54E504EF086FD0125B5E78A
:1078B0009FED118ADFE707F5BD412246683140465A
:1078C00010F008FD05460028A7D0B6F858340393F9
:1078D0002146404610F092FDBCEEC00A039B084AC8
:1078E0008DED000A062107F54E504EF065FD95E737
:1078F00000000034E02E65420000000084910C0876
:10790000A2910C0870B500F5005500F5A046B5F938
:1079100070130029ACBF01234FF0FF330029B8BF1B
:10792000494286F8C03E89B2044604F0B1FAB5F97E
:107930006C3396EDE37A002BCABF07EE903ADFED89
:107940000D7AF8EEE77AFCEEE77AF8EE677AB4EEB5
:10795000E77AF1EE10FA07D804F54E50064A0621F0
:107960004EF02AFD012070BD204604F0ADF900283C
:10797000F2D1F8E700000000C0910C082DE9F041B9
:1079800000F5BD4700F5BE45683708350446294671
:10799000384610F0FBFA04F5A04604F5405830B321
:1079A000D6F864134B1C22D0D8F8A80503681B6BCB
:1079B0009847D6F8D83E012B47D0D6F8D83E022BB0
:1079C00006D12046FEF7C8FCD6F80C3F984243DDAE
:1079D0002046FEF7C1FCD6F80C3FC01A0028B8BFFD
:1079E0004042B0F5FA7FCCBF0020012035E004F51D
:1079F000BD402946783010F001FDDFED197AB4EE74
:107A0000E70AF1EE10FA16D53846294610F0C6FB03
:107A10009FED147ADFED140AF6EE007AE0EE077AB5
:107A200028469FED120AFDEEE77AF8EEE77A27EE98
:107A3000800A10F059FDD8F8A8059FED0D0A0368DB
:107A40002A469B6A39469847B3E72046FEF784FCEE
:107A5000D6F80C3F9842B0DB0120BDE8F08100BFB2
:107A600000004843A00CB345000096430AD7233CCE
:107A700000000000F7B5374FD1ED026AD7F8FC3EA1
:107A80009FED357A07EE903AF8EEE77A0546D7EEA5
:107A9000876A0E46F5EEC06AF1EE10FA08DD55F081
:107AA00057FB2E4A06214EF087FC012003B0F0BDA3
:107AB000D1ED037A97EDE16AF5EEC07AF1EE10FAB6
:107AC00013DDF4EEC67AF1EE10FA0ED555F040FB58
:107AD0000446D7F88403F8F717FD214ACDE90001E1
:107AE000062120464EF068FCDFE7DFED1E7A337C8E
:107AF000B4EEE76AF1EE10FA54BFB0EE677AB0EE7A
:107B0000467A0BB90020D1E7B5EEC06AF1EE10FA63
:107B10000CDC86EE876A03EB830307EE903AF8EEFF
:107B2000E77AF4EEC67AF1EE10FAEBD52C7C002C55
:107B3000E8D17DF07DFB6B69C01A337C4FF47A721B
:107B400053439842DED901232B747DF071FB6861A9
:107B50002046ABE7987C00200AD7233CD8910C083C
:107B6000E9910C080AD723BC38B5054676F0B4FE77
:107B700075F008FC044640B97DF05AFBEB68C01A6A
:107B8000AB68984284BFAC600124204638BD000039
:107B900038B504460D467DF04BFB04F5A0439FED40
:107BA000077AC3F8DC0ED5ED027A67EE877AFDEE30
:107BB000E77A17EE902AC3F8D82E38BD00007A4431
:107BC00010B504467DF034FB04F5A043D3F8DC2E59
:107BD000801AD3F8D82E90424FF0000084BFC3F82B
:107BE000D80E012010BD000000F5A04393EDE37A0C
:107BF000D3F8D82E22EAE27207EE902AF8EEE77A5E
:107C00000020B4EEE77AF1EE10FA44BFC3F8D80EC4
:107C10000120704710B500F5005300F5A040B3F9FE
:107C20003E33002BB4BF4FF0FF33012380F8C03E3A
:107C300000F6087400F6F8600FC884E80F0010BD65
:107C400038B504462DED028BF0EE408AB0EE608A26
:107C500001B301295CD0B5EEC08AF1EE10FA66DD01
:107C6000DFED347AB4EEE78AF1EE10FA5FD8FCEE7D
:107C7000C87A04F54E5017EE903A2F4A06214EF07E
:107C80009BFBFDEEC87A04F5005417EE903A84F899
:107C90000B333BE0F8EE000A21F00AFB40B104F59B
:107CA00080444FF0FF33C4F8A43DBDEC028B38BDD7
:107CB00004F50053B3F9142307EE902AF8EEE77A9F
:107CC000F4EEE87AF1EE10FAC5D8B3F9163307EE00
:107CD000903AF8EEE77AF4EEE87AF1EE10FABADBD1
:107CE000DFED147A68EEA77A04F58043FDEEE77ABB
:107CF000062117EE902AFCEEE87AC3F8A42D04F5CD
:107D00004E5017EE903A0D4A4EF056FB0120CCE74C
:107D1000FCEEC07A0A4A17EE903A062100F54E5062
:107D200004F500544EF048FBC4EDC88AEEE700208D
:107D3000BBE700BF0000C8422F920C0808920C0855
:107D40001C920C08D1F80D3000EE903AD1F80930B1
:107D5000097A00EE103AFFF773BF000070B58B8808
:107D6000012B04460D4611D100F590763046F9F707
:107D7000D9FE02280AD994F81414B02303FB016138
:107D80002046DC31BDE87040FFF7BAB909F060FF6A
:107D900005F10801BDE8704009F0A8BBF0B500F599
:107DA000A04600279D4B86F8AD7389B0044608466F
:107DB0000D4683F8217F24F01DFB40B3012386F894
:107DC000A43304F54053D3F8A8050368DB6B984748
:107DD00086F8AB73C6F8C47E03A80FF0ADFFB6F803
:107DE00058144FF6FF73994208BF3946013104F524
:107DF000A84001AA89B21C3026F008FB28B1BDF8C2
:107E00000600A0F115035842584186F8A5036B8877
:107E10005D2B00F0FC8032D81F2B29D80F2B01D806
:107E200000202AE0103B0F2BFAD801A252F823F0D1
:107E3000237F0108397F0108437F01084D7F010836
:107E4000617F01082F7F0108117F0108217E010851
:107E5000217E0108217E0108217E0108217E010882
:107E6000217E0108217E0108717F0108577F0108EA
:107E7000532BD5D1012086F8AB0309B0F0BDBD2B43
:107E800018D8BB2B4BD8B22B7CD00CD8702B74D00D
:107E9000722BC5D1D5ED027AFDEEE77A17EE903A56
:107EA000C6F8D83E3BE0B32BBAD129462046FFF7AF
:107EB00055FF34E0C33B9AB2112AB1D8112BAFD889
:107EC00001A252F823F000BFBD7F0108217E010806
:107ED000BD7F0108217E0108217E0108217E010865
:107EE000BD7F0108217E0108217E0108217E010855
:107EF000F37F0108217E0108217E0108217E01080F
:107F0000217E01088F7F0108217E0108AD7F0108D5
:107F1000002386F8E13329462046FFF761F9012066
:107F2000ABE705F108012046FEF7CCFFF7E729464D
:107F30002046FFF79FF9F2E729462046FFF7E2F9CE
:107F4000EDE729462046FFF7F7F9E8E729462046FE
:107F5000FFF72CFAE3E729462046FFF7B1FADEE700
:107F600004F59A4129222031204606F02FF8D6E761
:107F700029462046FFF73EFAD1E729462046FFF77B
:107F800007FECCE729462046FFF7DCFEC7E7AB88B3
:107F9000012BC4D803F0010386F8A633AB88204A2E
:107FA000062104F54E504EF007FAB8E7A9880039CB
:107FB00018BF0121204600F087FBB0E7EB6896F878
:107FC000F91F04F5BF4473B92B6963B96B6953B9E1
:107FD00020465AF08FF90428A1D196F8F91F2046BF
:107FE0005AF092F99BE705F1080220465AF0CAFAC6
:107FF00095E795ED041AD5ED020A95ED030A96F87A
:10800000F91F002204F5BF405AF0A0F987E704F5F4
:108010009A4029460830FFF771FA80E7987C0020E3
:1080200040920C0800F5804200F59A43D2F8742D76
:1080300008339A4201D1FFF7B1BE0120704700001A
:1080400010B500F5804200F59A43D2F8742D08333C
:108050009A4204460DD100F59A410822203105F0DC
:10806000B5FF04F54E50034ABDE8104006214EF01E
:10807000A3B910BD50920C08F0B506468FB009ADFB
:1080800006F5A04428460F460FF056FEB4F85834C3
:108090004FF6FF72934208BF0023013306F5A84054
:1080A00007AA99B21C3026F0B1F9A0B117B100238C
:1080B000C4F8BC3E95E80F0001AE86E80F00D4F886
:1080C000143F009304F6087494E80E00034802F08D
:1080D00039FD0FB0F0BD0120FBE700BFC0790020E3
:1080E00070B5064606F5A045002103F0D1FED5F88F
:1080F000C44E7CB9304603F0E7FD10B90024204699
:1081000070BDD5F8BC3E012BF8DD7DF091F8C5F8C7
:10811000C40EF4E7D5F8D81E61B17DF089F8D5F822
:10812000C43EC01AD5F8D03E9842E7D90023C5F81E
:10813000D83E01213046FFF79FFF04460028DDD0DE
:10814000044A062106F54E504EF036F9002385F814
:10815000AD33D4E778920C0870B50A468B88190ABB
:10816000137E0546DB0748BF01EB810105F5A044FE
:1081700048BF4900002603F08BFE84F8AD63284613
:1081800003F0A2FD10B90024204670BDD4F8D81E1B
:1081900051B1D4F8BC3ED4F8B82E9342F3DD012B94
:1081A000F1DDC4F8D86E01212846FFF765FF0446CB
:1081B0000028E8D0034A062105F54E504EF0FCF8A1
:1081C000E2E700BF90920C0838B5054605F5A044DB
:1081D000898803F05DFED4F8D83E73BBD4F8BC3E6A
:1081E000002BB8BF5B42012B02DC0024204638BDC7
:1081F00094F8C12E94F8C23E6AB9002BF5D0D4F899
:10820000FC2E6423062192FBF3F305F54E500C4A35
:108210004EF0D2F801E0002BF1D10121C4F8D81EB4
:108220002846FFF729FF04460028DED0054A06212C
:1082300005F54E504EF0C0F8D8E70021F0E700BF3A
:10824000A8920C08C6920C082DE9F0474B881F2B0A
:108250008AB004460A462FD80F2B06D8954A042127
:1082600004F54E504EF0A8F887E0A3F110010F2955
:10827000F4D801A050F821F08B8301084D84010847
:1082800059840108678401088184010899830108E1
:108290007F8301085D8201085D8201085D8201081B
:1082A0005D8201085D8201085D8201085D8201082E
:1082B0008D84010873840108702B00F0F5800CD8C0
:1082C000532B00F0E9805D2BC8D100F59A400830AF
:1082D0000AB0BDE8F047FFF747BCB32B08D8B12B75
:1082E0004BD8722BBAD10AB0BDE8F047FFF77CBC7F
:1082F000D42B3BD8BB2BB1D9A3F1BC02182AADD8E3
:1083000001A151F822F000BF7B8301087B830108A3
:108310005D8201085D8201085D8201085D820108BD
:108320005D8201087B8301085D8201087B8301086F
:108330005D8201085D8201085D8201087B8301087E
:108340005D8201085D8201085D8201087B8301086E
:108350007B8301087B8301085D8201085D8201083F
:108360007B8301085D8201087B830108DF2B04D039
:1083700040F6B83293427FF471AF01202FE02046DF
:108380000AB0BDE8F047FFF7EFB8114620460AB043
:10839000BDE8F047FFF7DAB904F5A04504F5BB46A0
:1083A000D5F8F83304F5BD4704F5BE4804F5BD49DA
:1083B000072B06F1500607F1680708F1080809F1D4
:1083C00078090FD104F5A74470340194D5F87433BB
:1083D000009342464B46394630467AF07DFE0AB05D
:1083E000BDE8F08700230DF1270133488DF82730D1
:1083F000FEF7FAFCD5EDEC7AD5EDE10A95EDE41A3D
:10840000D5F894A3CDED060A30EE670A04F5C04016
:1084100004308DED070A8DED051A74F0A9FF0546AD
:10842000204600F099FE9DF827309DED051ADDED00
:10843000060A9DED070ACDE90203CDE900A54B46EA
:108440004246394630467AF09DFDC8E7204691887D
:1084500003F01EFD0020C2E7114620460AB0BDE829
:10846000F047FFF779BE20460AB0BDE8F047FFF7B6
:1084700037BE114620460AB0BDE8F047FFF7A4BE5C
:1084800020460AB0BDE8F047FFF73CBA20460AB0E4
:10849000BDE8F047FFF772BA00F59A4008300AB01D
:1084A000BDE8F047FFF7E6BA0AB0BDE8F047FFF7CE
:1084B00087BB00BFE0920C08982C002070B500F537
:1084C000804200F59A43D2F8742D08339A4205464B
:1084D0000E4602D00024204670BDFFF7B5FE0446CC
:1084E0000028F7D0318805F54E5052F049F9F2E7EF
:1084F00021F04003152B04D0A1F15E0358425841EE
:108500007047012070470000102945D8DFE801F0CE
:10851000090D1115191D212529442C3034403838F6
:108520003C0000F59A404430704700F599401C30FB
:10853000704700F599402430704700F599402C3081
:10854000704700F599403430704700F599405C3031
:10855000704700F599406430704700F599406C30E1
:10856000704700F59A40704700F59A400830704710
:1085700000F59A402030704700F59A402830704747
:1085800000F59A403030704700F59A403C30704713
:1085900000F59A404C3070470020704700290DDBF1
:1085A000074890F8E02BCBB29A4207D3D0F8DC3BD7
:1085B0000122595CA0F5005005F0E2BD704700BFF4
:1085C000984C00202DE9F34100F50053044693F840
:1085D000B03B03F0010603F0020803F004075B0759
:1085E00000F54E5535D01F4A062128464DF0E4FED1
:1085F00026B104F53B50343076F07CFFB8F1000F23
:1086000004D004F541500C3076F0F0FC27B104F5AD
:108610004650243077F098FB04F5C044012384F8D9
:10862000A930114A114B1249B8F1000F08BF1A4680
:10863000002F08BF1946CDE900210E4A0621002E61
:1086400018BF134628460C4A4DF0B6FE02B0BDE8EE
:10865000F0810A4A0621284602B0BDE8F0414DF0FB
:10866000ABBE00BF0D930C0802930C08146D0D08EF
:1086700009930C08FC920C081E930C0830930C080C
:1086800010B5044600F53B50343076F05FFF04F53A
:1086900041500C3076F0D6FC04F54650243077F08B
:1086A0008DFB04F5C04393F8A92052B1002283F852
:1086B000A92004F54E50034ABDE8104006214DF0B4
:1086C0007BBE10BD50930C0809B1FFF77BBFFFF7CD
:1086D000D7BF000000F580430A4AD3F8741D9142C9
:1086E0000DD093F8813D43B900F59A42083291428A
:1086F00003D100F5A04090F8A63318467047002338
:10870000FBE700BFDC79002010B504467CF090FD4B
:10871000054BD3F8943DC01A642804D82046BDE820
:10872000104056F081B910BD986C002010B500F5CE
:108730002E54D4ED087AF5EEC07AF1EE10FA8AB034
:108740004FF0000304F1200445D9079308930993DF
:1087500006AB019300F5985007AB009303AA05AB55
:1087600004A9103008F048FF30B3DDED080A9DED94
:10877000070AA4F0F3F8DDED090AA4F0EFF8D4ED50
:10878000007A9DED047A77EEA76AB4EEE70AF1EE7F
:1087900010FAF4EEC76AACBF01200020F1EE10FA27
:1087A0000CD802309DED037AF4EEC77AF1EE10FAA0
:1087B0000CD8003818BF01200AB010BDF4EEC77AFB
:1087C000F1EE10FA9CBF0130C0B2EBE7012894BF74
:1087D00000200120F0E70020EEE7000010B5074B75
:1087E0001A7A4AB901241C724AF038FD2246112136
:1087F000BDE810404AF0EABA10BD00BF588D002015
:1088000010B5074B1A7A4AB100241C724AF026FDB3
:1088100022461121BDE810404AF0D8BA10BD00BF71
:10882000588D0020F0B5054685B005F59856684688
:1088300010360FF081FA6946304609F00FF8A0B102
:108840003248334C334F74F093FD40B105F52E534D
:10885000D3ED087AF5EEC07AF1EE10FA07D80023CE
:1088600028462380FB73FFF7CBFF05B0F0BD2846F9
:10887000FFF75CFF98B3637873BB23780133DBB2F7
:10888000082B237002D1304608F022FF2378092BF1
:1088900002D1304608F014FF2378092B1CD94FF47D
:1088A000857323804AF0DAFC022210214AF08EFA06
:1088B0007CF0BEFC6368C01A47F23053984208D976
:1088C000154A022105F54E504DF076FD7CF0B0FCC6
:1088D00060602846FFF782FF6378FB73C5E7267860
:1088E000002EF9D0013E6378F6B22670002BF3D04B
:1088F000002EF1D166704AF0B1FC324610214AF0E8
:1089000065FA2846FFF77CFFE6E700BF9C8C002055
:10891000588D0020058E002064930C0800F5A040BF
:10892000D0F8F833042B14BF90F8240401207047CA
:1089300073B500F580450192A5F88C1D04467CF0C6
:1089400077FCC5F8900DD5F8740D03685B689847FF
:1089500085F88A0DD5F8740D03685B6898470F2871
:10896000019A0BD80F2827D8DFE800F01C261C1C22
:108970001C1C1C1C1C264C260A260A0A18281BD163
:1089800004F50056019296F98033ABB1D5F8740D19
:1089900003685B68984785F88A0D96F98033019AD9
:1089A000022B27E01E4B93F8AA30F3B104F599414E
:1089B0005C31204605F00AFBD5F8740D95F88A6DF8
:1089C00003685B689847864204F54E5420D0D5F87A
:1089D000740D03689B689847124A03460421204699
:1089E00002B0BDE870404DF0E7BC04F5005393F9C8
:1089F0008033022BDAD004F59941042B0CBF64318B
:108A00001C31D6E72046FFF789FF0028D4D1B7E70D
:108A1000054A0421204602B0BDE870404DF0CCBCB0
:108A2000988C002074930C0896930C08F0B50446BB
:108A300004F5804685B00F46154655F07BFFD6F805
:108A4000740DA6F88C7D03685B68984718281ED8BB
:108A5000DFE800F00D0D0D0D0D0D0D0D0D1D526813
:108A60000D0D57571D1D1D1D1D1D1D1D0D00314BCD
:108A7000D3F8F823012A20D104F5005393F8813369
:108A8000023B012B19D904F5405383F87C23D6F817
:108A9000740D294A294B052D18BF1346026803930C
:108AA0009268904704F54E540090039B244A042199
:108AB00020464DF081FC05B0F0BD224B93F8AA3062
:108AC0003BB104F599412A465C31204605F07EFA17
:108AD000DDE704F5005393F98133032B03D12046DE
:108AE00003F030FAD3E7022BEBD0042B15D104F5B9
:108AF0009A412A460831E8E72046FFF70FFF002891
:108B0000C5D104F5005393F98133032BE7D0022B31
:108B1000D7D0042BEBD0012BB9D104F59A412A46CA
:108B20002031D2E704F5005393F98133042BAED101
:108B3000DDE700BF987C0020AC930C08E3770C08BD
:108B4000B4930C08988C002070B5044600F54E567E
:108B5000114A0421304604F580454DF02DFC0023D8
:108B6000A5F88C3D04F5005393F8C832032B12D1BD
:108B700095F88A1D3022204605F002FBD5F8740DC9
:108B800003689B689847054A034606213046BDE8BE
:108B900070404DF011BC70BDC8930C08DF930C08F9
:108BA00000F5405310B500220529044683F87C23C4
:108BB00000F54E500CBF054A054A042104F58044D7
:108BC0004DF0FAFB0023A4F88C3D10BDF8930C087F
:108BD00009940C0830B50B4687B00446052A18D80E
:108BE000DFE802F0172A0350175D00F5A043D3F821
:108BF000F833042B20D02C4D95F89D3DE3B12B4943
:108C0000A1F6DC2025F0D4FF28B1294B012283F8FE
:108C1000242407B030BD2549A1F6DC2026F0C8FA8F
:108C200050B104F59A4104220831A5F5804007B0FF
:108C3000BDE8304005F0CAB904F5A043D3F8F833D5
:108C4000042BE6D004F5005393F94B33022B0AD1E1
:108C5000154B93F89D3D33B11449A1F6DC2025F066
:108C6000A7FF0028D1D104F59A41042220312046E3
:108C700005F0ACF904F50C500B3007B0BDE83040FE
:108C800041F002BC0B4A112101A87BF087FB04F5DF
:108C9000BC4001AA01215C3077F042F9B9E707B086
:108CA000BDE8304003F04EB9986C0020908B002056
:108CB000987C002024940C0870B52DED048B04469C
:108CC0007CF0AAFA4F4BB4F8BE101A884E4E8A4276
:108CD00005464E4A06D01980002330601370BDEC63
:108CE000048B70BD33684A49C31A8B4276D901237D
:108CF000137055F01FFF55F0D7FD356055F01AFF82
:108D000055F0D2FD04F5405393F87B3323B104F5BD
:108D1000BC405C3077F058F855F0EEFD0428DED901
:108D200055F008FE0021204603F02EFC00212046CD
:108D3000F0EE409A03F032FC01212046B0EE409A5A
:108D400003F0ECFD00212046B0EE408A03F030FC39
:108D500004F5C0400430F0EE408A74F013FBDFED00
:108D60002D7A0028B0EE690A4FF0040008BFB0EE7B
:108D7000678A57F0D5FAB0EE490A132057F0D0FAB7
:108D8000B0EE680A152057F0CBFA04F5BC45B0EEFA
:108D9000680A1A2057F0C4FA5C354620B0EE480A3B
:108DA00057F0BEFA284677F09DF808BB0121084627
:108DB00057F0B8FD9FED170A022057F0B1FA9FED6A
:108DC000150A032057F0ACFA204603F0C7FFBDECAC
:108DD000048B2046BDE8704004F0D6BE1278002A0D
:108DE0003FF47DAF44F6206293427FF678AF80E790
:108DF0002846FDF73DF804F5A04393F9663E2B2B7A
:108E0000D4D06CE7648D0020688D0020668D002032
:108E1000400D03000000000000F5804200F59A4379
:108E2000D2F8742D08339A4204D100F5A04090F88E
:108E30002404E8B10F4B93F8C80203F58043A0F176
:108E40002702012A93F8B8300FD92C2809D00A2814
:108E500009D0A0F13102504250410A2B18BF002026
:108E600070470120F9E7012070470A3B58425841FA
:108E7000704700BF984C002008B500F5005393F8E8
:108E8000B02142B193F8EC312BB1FFF7C5FF80F070
:108E90000100C0B208BD0120FCE700002DE9F04749
:108EA00000F50055A64F95F8EC81044600F5C0404A
:108EB0008AB0043074F05CFAD7F8F833042B064615
:108EC0004FD000284DD0B7F85A14A7F5A040FFF7AF
:108ED0000FFB014620B197F820144B1E594259410F
:108EE00004F50657DFF86CA23037384664F050F8C6
:108EF0009AF8B8300A2B814603D1A6BB00238AF822
:108F0000B83095F8B031002B39D195F9B6318D4D87
:108F1000012B03D0063BDBB2012B11D895F8C832E8
:108F20000A2B0DD104F58046D6F8740D03681B6A30
:108F3000984728B1D6F8781D2B22204605F046F830
:108F40009AF8B8300A2B04BF37238AF8B83095F85E
:108F5000C8320A2B02D1372385F8C8320AB0BDE8DF
:108F6000F0870121BCE740EA0803DBB2002BC8D13F
:108F7000AAF5C04000F0F0F80028BFD0C1E7002EED
:108F8000ECD004F5BB40503079F072FF0028E5D1F9
:108F90002046FFF741FF0028E0D1B9F1000F00F0B3
:108FA000BF8069494A46384663F0CAFB95F9B681E5
:108FB000B8F1010F07D040F38780A8F10603DBB2B8
:108FC000012B00F281805FFA88F8B8F1010F4ED1D1
:108FD00004F5804204F59A43D2F8742D08339A427E
:108FE00009D104F5A04393F8243423B195F84B3309
:108FF000013B012BB2D904F59A410A2220312046C7
:1090000006AE04F0E3FF30460EF096FE95F9C92156
:1090100092BBB8F1010F2FD004F5A048B5F9CA31C1
:10902000D8F8E41EDFED495AD1ED017A002BF8EEB5
:10903000E77A52DD07EE103AF8EEC76AE6EEA57A57
:109040003046FDEEE77A17EE901A0EF07BFE002315
:109050003846CDE9043364F037F804A964F094FD90
:10906000002857D0049B0893059B099317E004F54B
:109070009A410A223031C2E72046FCF771FF07EE21
:10908000900A6F4604F5BD42783221463846B8EE64
:10909000E70AFEF79BF897E80F0086E80F0095F9BE
:1090A000B631012B10D031462046FDF7E9FB3146A1
:1090B0002046FDF773FF95F9B631072B04D104F56F
:1090C0004054012384F87A334AF0C8F84A4609210B
:1090D0000AB0BDE8F04749F079BED5ED6E6A95ED6E
:1090E000715A95ED6F7A35EE076A36EEC57AB4EEB1
:1090F000C67AF1EE10FA89BF37EE067A95EDEB7A73
:1091000027EE257AF6EE006A94BFE7EE257AE7EEC1
:10911000267A95E7D8F8E43E9A680892DB68A4E7D7
:10912000B8F1000F3FF41AAF95F8EC31002B7FF443
:1091300015AF074A052104F54E504DF03DF9C3E740
:10914000987C0020984C002030940C080000C84205
:1091500039940C08988C002010B5044600F5C040E6
:10916000043074F00FF904F5A04494EDFF7A48B18F
:10917000DFED067AB4EEE77AF1EE10FAACBF01202B
:10918000002010BDDFED027AF4E700BFCDCCCC3D6E
:109190006666663F00F58043D3F8741D00F59A4378
:1091A0004C33994204D100F5A04393F8F0239AB9C7
:1091B00000F59A430833994210D100F5A04393F883
:1091C000F0234AB1D3F8F823032A07D1B3F85A247D
:1091D000A2F116035A425A41104670470022FBE79B
:1091E0002DE9F84F00F5804200F59A43D2F8742D2E
:1091F00008339A42054600F5A04704D100F500580F
:1092000098F9243333B90023C7F8E43387F8E133FE
:10921000BDE8F88F7CF00CF8D7F89843814634B15C
:10922000041B40F6C3139C4294BF0024012428462B
:10923000FFF792FF834620B1002487F8E043002621
:109240003FE005F5C040043074F092F882460028F3
:10925000F2D005F5BB465036304679F009FE0028BD
:1092600040D097F8E063C6BB44B305F5805141F2A6
:109270007072D1F80835002BB8BF5B42934206DC10
:10928000D1F80C35002BB8BF5B42934228DD05F5C1
:10929000A84105F5BD40603178300FF0AFF8DFED43
:1092A000467AC7F8E493B4EEE70AF1EE10FA4FF00D
:1092B00000034CBF01260026C7F8E833012387F8D6
:1092C000E03305F59070F8F72DFC022833D9002C17
:1092D00046D10023C7F8E4339AE75C465E46EDE7E3
:1092E0003446EBE7304679F0ABFD064638B1002C4A
:1092F000A5D04FF4FA73C7F8E83354469FE7D7F880
:10930000F833012B03D0032B0DD03446D9E7D8ED29
:10931000F17AF5EEC07AF1EE10FAF6DD97F8F03357
:10932000002BF2D1E5E72846FFF734FF0028ECD107
:10933000002CDED1C5E705F5FF5A05F5005B0AF103
:10934000180A9BF84611504606F056FB0028C0D07C
:109350009BF84611504606F047FC0028B7D1B8E705
:10936000D7F8E43313B9C7F8E49351E7D7F8E82303
:10937000A9EB03039342FFF44BAF97F8E133002BC3
:109380007FF446AF012287F8E12398F82433DB0706
:1093900005D505F5C0400C210430F8F7F9FA05F5BC
:1093A0004E502EB1054A0221BDE8F84F4DF004B8E9
:1093B000034A3146F8E700BF0000964250940C087B
:1093C00066940C082DE9F04F2DED028B054685B013
:1093D000002305F5005803937BF02AFFD8EDC87AE7
:1093E000F5EEC07AF1EE10FAC4BF9FEDBD7A67EEDC
:1093F000877A05F5907BC8BFFCEEE77A07465846AA
:10940000CCBF17EE906A9626F8F78CFB022840F244
:10941000FC8095F814349FEDB37AB02202FB03531D
:10942000D3ED837A67EE877AFCEEE77A17EE903A0F
:109430009E428CBF00260126B8F91433022BB8BF18
:10944000022307EE903A05F59850B8EEE78A03A993
:10945000F6EE087A103028EE278A08F0DDF9044687
:1094600040B1DDED037AF4EEC87AF1EE10FAACBF4C
:10947000012400245846F8F755FB05F5C04901289A
:1094800009F1040905F5A04A16D8484673F070FFA3
:1094900090B18CB99AEDFF7ADFED937AB4EEE77A6A
:1094A000F1EE10FA08DDDDED037AF4EEC87AF1EEA4
:1094B00010FAACBF01240024484673F059FF009015
:1094C000002800F0FA8095F8142405EB0212D2F877
:1094D000C02172B158460192F8F724FB012800F22E
:1094E0009680019A41F28731BA1A8A428CBF0022D3
:1094F0000122DAF8941301B11AB9002C40F08980E6
:10950000344605F5804105F59A42D1F8741D0832BC
:1095100091421AD198F94C23002A40F0828000220F
:109520008AF8E223DAF8F823042A00F0A880072A50
:1095300000F0B980032A08D12846FFF72BFE20B19E
:1095400000248AF8E143CAF898439AF8E22302B16A
:109550007CB907EE904A9FED657ADAEDFF6AF8EE86
:10956000677A67EE877A9FED627AE6EE877ACAEDD0
:10957000FF7A2846FFF7F0FD0446A8B19AF80004E8
:10958000CAF8947308B9CAF8047405F5804105F562
:109590009A42D1F8741D0832914205D1DAF8982325
:1095A00002B108B9CAF898739AF828258AF80044D5
:1095B00064F3C3028AF828256EF014F821466DF092
:1095C000EDFF4C4A28465471FFF70AFE2846FBF788
:1095D000AFF934B198F8CA221AB97BF029FEC8F85D
:1095E000CC0288F8CA422846FFF7B6FD002875D19C
:1095F000484673F0C7FE80F00100C0B28AF8080444
:1096000005B0BDEC028BBDE8F08F002614E7002208
:109610006FE71FF027FA1EF075FB00287FF470AF8C
:109620006FE7524207EE902A05F6C802F8EEE77A95
:1096300092EDDB7AF4EEC77AF1EE10FA11DDDFED90
:109640002E7A9AEDFF7ACAF8EC73B4EEE77A01222B
:10965000F1EE10FA8AF8E2237FF764AFCAEDFF7AE1
:1096600060E79AF8E223002A3FF45CAFDAF8EC23D3
:1096700040F6B831BA1A8A423FF651AF52E705F5C3
:10968000BB40503079F0DCFB00283FF45EAF9AED30
:10969000E17ADFED197AB4EEE77AF1EE10FA7FF7AE
:1096A00054AF009C51E79AEDE17AFEEE007AB4EEF9
:1096B000E77AF1EE10FAF4D447E7DAF8F823002C51
:1096C00018BF3446012A07D005F5BB40503079F069
:1096D000ADFB00283FF439AF002436E700208DE7CA
:1096E0000000B4420000C8429A99993E9A99193EE6
:1096F0009A99593F058E0020CDCC4C3E00207047F2
:1097000000207047012070470020704701207047FB
:10971000034BD3F8F803431E58425841704700BF2B
:10972000987C002030B587B002A80EF005FB3048C9
:1097300079F07CFB20B12F492F48FDF7B3F81FE0EB
:109740002B4879F07DFBE8B12C4C04F1240523462D
:1097500004F11002A4F11001A4F59470009579F0C1
:1097600095FBCDE90045A4F6F86292EDE30A2449A1
:1097700004F11003A4F11002A4F5947079F048FBF1
:1097800007B030BD1A4802A979F098FB08B102A9C8
:10979000D2E7194802F098FA0028CCD1194C94F875
:1097A000083F5B071DD4D4F81C3F002BC3D0114ADF
:1097B000A2F12001A2F110000EF08CFD0028BAD118
:1097C000D4EDE47A0B490C48B7EE000A30EE670A94
:1097D000FDF798F80C4A084802F12001FCF71CFC40
:1097E000CEE7A4F5A040FDF70BF90028C8D1DAE7D1
:1097F000688A0020A08B0020982C0020908B0020ED
:109800007C580020987C0020808B002008B50A48F6
:1098100090F8BD33013B012B03D8A0F50050F9F7B8
:10982000DBF90648F9F7FEF80448F9F79BF9BDE8BB
:1098300008400248F9F7C0BC984C0020982C002042
:10984000124A904208B50ED002F1080188420AD0AF
:1098500002F11001884206D002F13801884202D09C
:109860005C32904206D10A4B93F97503B0FA80F04E
:10987000400908BD03681B6A984728B1054B93F857
:109880007A0380F00100F4E70120F2E73C79002040
:10989000984C0020985C0020104A904208B518D0DF
:1098A00002F10801884214D002F11001884210D060
:1098B00002F1380188420CD05C32904209D0036832
:1098C0001B6A984738B1064B93F87A0380F0010081
:1098D00008BD0020FCE70120FAE700BF3C7900202A
:1098E000985C0020024A0260024A4260704700BF52
:1098F000B8940C08A83F002008B50368DB6D9847B2
:109900000648D0F8742D00F550639A4205D0BDE8A2
:109910000840A0F58040FEF7B3BE08BD986C00205B
:109920002DE9F041464CA4F53E730025C11A4B4287
:10993000C4E9F355A4F500584B41002284F8505374
:10994000A4F8A65384F8AA53C4F86C2384F8685387
:1099500084F8E15384F8E253C4F8C853C4F8D853E8
:10996000C4F87C2388F81C364368D3F8FC31A4F88B
:10997000A03304F6F86306460FCB04F6E86787E8E1
:109980000F0084F8A95384F8B853C4F8C45E7BF080
:109990004FFCA4F58057C7F87C0D336830465B69EF
:1099A00098474FF0FF3384F8AC0384F8AD5388F840
:1099B0007C5384F8215F84F8AB53C7F8A43D336827
:1099C00030469B6D98470546002835D033683046B1
:1099D0009B6B984784F8F003D8F8A8050368DB6B05
:1099E0009847A7F6E84075F0EDFEA4F5A04002F018
:1099F00039FDA8F5656063F031FB94F82434C3B1F8
:109A0000A4F5A040FFF7A8FB98B90E4873F0BAFC84
:109A100078B9D7F8740D03685B6B984748B953F071
:109A200097FB094A06214CF0C7FC04F21C4025F0C4
:109A30006BF90648F8F734FB2846BDE8F08100BF13
:109A4000987C00209C8C002078940C08982C002096
:109A500070B503681B6E0E4615469847044650B90C
:109A600095F900303BB90548054B00683246C06A9D
:109A700029461CF0DDF9204670BD00BF942C002063
:109A80009C940C0810B50D4C204675F097FC04F51D
:109A9000AC7075F00FFA04F52C7076F03DF9084BB8
:109AA00003F5A042002182F8681303F5005300215A
:109AB000C2F86C13012283F8402E10BD8C5B00208D
:109AC000982C002008B52DED028B1520B0EE408AB1
:109AD00056F026FCB0EE480ABDEC028B1A20BDE819
:109AE000084056F01DBC000008B5084890F97533D1
:109AF0000121A0F5005033B102F010FFBDE808408D
:109B0000462056F00DBC02F031FFF7E7984C0020DC
:109B1000042070470048704782D40D080048704701
:109B200082D40D08037A73B1D0ED037AFDEEE77AA3
:109B300017EE903A084AC2F80C34437A3BB10369F5
:109B4000C2F8103470474368D3F8F831F2E743683D
:109B5000D3F8FC31F4E700BF987C002008B500235F
:109B6000038100F11401406807F06CFE012008BD7C
:109B700070B56E4E2DED048B06F59B430446012116
:109B8000304693ED0F9ADFED6A9A02F0FDFC012159
:109B9000B0EE408A304602F001FDC8EE297A06F5A3
:109BA00000556068B5F9983304F1140108EE903A55
:109BB000F8EEE88AB5F99A3368EEA78AC0EE297AFA
:109BC00008EE103AB8EEC88A28EE278A07F03AFE67
:109BD00095F99E3363B39FED577AF0EEE87AF4EE91
:109BE000C77AF1EE10FA23D5227A6368002A55D19C
:109BF000012222720022E26094ED037ADFED4E7AB8
:109C0000D3F8F8314D4A4E4867EEC77A9FED4D7A4A
:109C100067EE877AB0EE490AFDEEE77A17EE901A02
:109C20000B44C2F80C340023012275F057FB08E006
:109C3000002343482372F0EE490AB0EE680A75F03B
:109C400049FB042056F06CFB95F99E3343B19FED20
:109C5000397AF0EEC87AF4EEC77AF1EE10FA28D429
:109C6000002339486372F0EE490AB0EE480A74F0F6
:109C70008BFF132056F054FBB5F99C33002B03DD0A
:109C8000324E96F9BA3163BB28482021F8F774FCAC
:109C9000002843D1254802F0B7FA42E0D3EDC56A67
:109CA00096ED467AD4ED037AE6EE877AC4ED037A30
:109CB000A2E7637A2BB9012363726368D3F8FC319E
:109CC00023611E4B2169C3F810146368D3F8FC01AB
:109CD0000023091A1A461C48B0EE490A75F03AF8F2
:109CE000C7E70121A6F5405002F062FC80EE297A18
:109CF000B5F99C33002106F5D27007EE903AF8EEE4
:109D0000E77AF0EE490A27EE870A75F005FFBDEC09
:109D1000048B2046BDE87040FFF7D4BE0348F9F736
:109D2000B7F807EE900AB8EEE70AF0E7982C0020A3
:109D300000A08C4500000034E02E6542987C002095
:109D40008C5B00200000C842E45C0020985C00208E
:109D50002DE9F04F2DED0C8BDFF8A8A39FEDDEDA97
:109D60009FEDDE9A97B00AF59B4300F11405044677
:109D70000121504693ED0FBA02F006FC0121504636
:109D8000F0EE408A02F00AFC01215046B0EE408A13
:109D900002F00EFCDFEDD27A88EEA77A0AF50056C3
:109DA00001A8B6F998330AF5A04B0AEE903AF8EEFE
:109DB000EAAAB6F99A33DFEDCB8A6AEE87AA88EE73
:109DC000277A0AEE103AB8EECAAAB6F99C339FED8C
:109DD000C68A2AEE07AA80EE277A09EE903AF8EEB4
:109DE000E99A6AEE8D7A69EE879AF0EEEACAF4EEA5
:109DF000C8CACDED017AB0EECACA6AEE0D7AF1EEAC
:109E000010FAF0EEE9BAB4EEC8CACDED027A58BF46
:109E10004FF0010969EE8D7A48BF4FF00009F1EE6D
:109E200010FAF4EEC8BA9AED460ACDED037A54BFA3
:109E30004FF001084FF00008F1EE10FA54BF01276F
:109E4000002721F0DDFD01A9284621F0F9F8284678
:109E500021F0E8F9284621F05FF920EE090A2846AA
:109E600020EE280ABDEEC00A10EE103ACBF80C34F2
:109E700021F06CF920EE090A20EE280ADFED9B8A1A
:109E8000BDEEC00ACDED0D8A10EE103ACBF81034BD
:109E90000DF1280B4FF07E53594660680A93CDEDC3
:109EA0000C8ACDED0B8A07F0CDFC0021504602F064
:109EB00035FDB0EEC00AB4EEC80AF1EE10FA16D5C0
:109EC0005046FFF749F990B9F4EEC8CAF1EE10FA1E
:109ED0000DD5B4EEC8CAF1EE10FA08D5F4EEC8BA42
:109EE000F1EE10FA44BF9BE80F0085E80F000AA8C6
:109EF00021F0FCF9294612A88DED141A8DED120AF5
:109F0000CDED130ACDED151A21F002FA0DF1100A6C
:109F100051460EA88DED101ACDED048ACDED058ABF
:109F2000CDED068A8DED0E0ACDED0F0ACDED111A9D
:109F300020F0C0FFB6F99833DFED6D7A01EE103AEC
:109F4000B6F99A3309EE103AB6F99C3308EE903A16
:109F5000B8EEC11AB8EEC99AF8EEE88A21EE271ACF
:109F600029EE279A68EEA78AF4EEC8CAF1EE10FA35
:109F700021EE0D1A29EE0D9A68EE8D8A07D594F818
:109F80002430DFED5A7A002B18BFB0EE671AB4EE1A
:109F9000C8CAF1EE10FA07D594F82530DFED537AF0
:109FA000002B18BFB0EE679AF4EEC8BAF1EE10FAC3
:109FB00007D594F82630DFED4D7A002B18BFF0EE70
:109FC000678A9AE807000DF11C0B8BE80700F1EE99
:109FD000410AC2209DED070A1FF07CFAC3208DEDD7
:109FE000070AB0EE491AF1EE490A9DED080A1FF082
:109FF00071FAB0EE681AF1EE680A8DED080AC42015
:10A000009DED090A1FF066FA514658468DED090A82
:10A0100021F08CFC12A928468DED120ACDED130A11
:10A020008DED141A06F6F86621F00AF8284621F09C
:10A03000F9F8DDED076A96ED007A2E4B9FED270AC1
:10A04000C6EE877A5846DDED086ACDED077AD3ED86
:10A05000147A86EEA77ADDED096A8DED087A86EE30
:10A06000A77A8DED097A21F0CBFCB9F1000F01D070
:10A07000CDED07AAB8F1000F01D08DED08AA0FB100
:10A08000CDED099AF0EE4B0A9DED070A1A4875F0DE
:10A0900021F9042056F044F9F0EE4B0A9DED080A30
:10A0A000164874F071FD132056F03AF90021F0EED5
:10A0B0004B0A9DED090A124875F02EFD2046FFF768
:10A0C00001FD84F8249084F8258084F8267017B068
:10A0D000BDEC0C8BBDE8F08F35FA8E3CE02E65426E
:10A0E00000A08C450000C8420000003400000000C1
:10A0F000CDCC4C3E985C00208C5B0020E45C0020C2
:10A100003C5E0020982C002010B50446FFF7ECFCC4
:10A110000B4B93F99E23022A0DD1B3F99C23002AFD
:10A1200009DD03F5805393F9BA3123B12046BDE828
:10A130001040FFF70DBE2046BDE81040FFF718BDE8
:10A14000984C00200A20704700487047459F0C0833
:10A1500000487047459F0C08012070470120704758
:10A16000012070470120704701207047034BD3F84E
:10A17000F803031F58425841704700BF987C0020E5
:10A18000F8B5194D05F6F8630FCB05F6E86405F64A
:10A19000087684E80F0086E80F00002705F21C40CF
:10A1A00085F8AC7324F0F0FF104B1C68E66A336846
:10A1B00030465B689847A8B196F84D3093B1E36A92
:10A1C0009B8F7BB152F0C4FFE36A094A9B8F062143
:10A1D0004CF0F2F8E36A05F21C40998F24F0C0FDC0
:10A1E000E36A9F870120F8BD987C0020942C002012
:10A1F00088950C0810B50A4C94F82034012B0BD12B
:10A2000004F21C4022F06AF8B4F85A34152B03D13A
:10A2100004F55D6078F0EAFE0023C4F8983310BDC1
:10A22000987C002008B507F013FD90F87C32DB071E
:10A2300004D5BDE80840024824F042BE08BD00BF76
:10A24000B480002010B5304C94F82034012B0ED08F
:10A25000A4F538710822A4F5A04003F0B7FE52F02F
:10A2600077FFBDE81040294A06214CF0A5B8B4F8A4
:10A270005A34162B05D0152B36D1D4F8F833072BCA
:10A280000AD1234804F01EFA214804F055FBBDE82A
:10A2900010401F4804F074BAA4F5A040F9F7F6F88E
:10A2A000A4F5A040F8F7F4FFA4F54053D4F80C143B
:10A2B00093F9DC2364235A4304F55D6078F0F2FDE2
:10A2C000C4F80C0404F55D6078F02EFF30B1BDE8F1
:10A2D00010409FED100A462056F022B8A4F5A04089
:10A2E000BDE81040F8F7BCBD1E2B18BF4FF0FF3380
:10A2F000074818BFC4F86433F9F7C8F80448F8F7FA
:10A30000C7FF0348ECE700BF987C0020A0950C082D
:10A31000982C00200000000010B5144BB3F85A34FC
:10A32000532B04461ED102F0EFFE9FED110A46208A
:10A3300055F0F6FF9FED0E0A492055F0F1FF9FED15
:10A340000C0A4A2055F0ECFF462056F0C9F8492087
:10A3500056F0C6F84A2056F0C3F82046BDE8104033
:10A36000FFF790BBBDE81040FFF750BA987C002083
:10A3700000000000082070470048704738960C081D
:10A380000048704744960C080120704708B5024801
:10A39000FEF718F9012008BD982C0020014800F0B4
:10A3A00059B900BF7479002010B50446FFF72EFAA2
:10A3B0002046BDE81040FFF797BB00000120704722
:10A3C00000487047B8960C0800487047C0960C08C3
:10A3D000012070470120704710B5054B03F6087443
:10A3E00003F6F8630FCB84E80F00012010BD00BF17
:10A3F000987C002008B50B4800F5A04200F50053FA
:10A400000321D3F8D43B93FBF1F3C2F80C34F8F7F3
:10A41000A3FF0448F8F73CFFBDE808400148F8F7FF
:10A420001FBD00BF982C00200720704700487047D0
:10A43000A0790C080048704734970C080120704739
:10A4400001207047012070477047000008B50023C5
:10A45000037203610248FCF7E1F9012008BD00BF67
:10A46000982C002010B5194CD4F8BC3BB3F9083037
:10A4700023B9D4F8C83BB3F90830F3B10023037211
:10A480000361D4F8BC0B54F045FC04F6D433D3ED8F
:10A49000007A0F48F8EEE77A27EE800ABDEEC00A90
:10A4A00010EE103AC0F80C34A0F5A040F8F754FFB5
:10A4B000BDE81040074801F025BB037A002BE0D02F
:10A4C000A4F50050F8F7E2FFF2E700BF984C002037
:10A4D000987C0020982C002070B54E4DDFED4E7A10
:10A4E00095F814349FED4D7A2DED048BB02606FBC4
:10A4F000035393ED848A9FED4A9A28EE278A05F547
:10A50000A853BDEEC88A93ED070AF8EEC87A044650
:10A5100067EE897A97EE870A1EF0C8FF237AF0EE7D
:10A52000408A002B62D105F50053D3F8BC3BB3F948
:10A530000830002B5AD1284601F066FE002855D17C
:10A5400095F8143495F8581406FB035393F8F12149
:10A5500000294BD1012A49D993ED837AF0EE087A8C
:10A56000B4EEE77AF1EE10FA40DBDFED2E7AB0EED2
:10A57000E80AB4EEE70AF1EE10FA37D5236993B38F
:10A580007AF056FE2369C01AB0F5FA7F32D8237AE2
:10A59000002B3CD0244DA5F1200696E80F0085E85D
:10A5A0000F0094ED038AA5F110013046B8EEC88A79
:10A5B0000DF024FF28EE098ADFED1C0A284670EE14
:10A5C000200AB0EE480A0DF08FFF194B9FED190AD3
:10A5D000D3F8A805BDEC048B03682A4631469B6A74
:10A5E000BDE8704018477AF023FE20612369002BF4
:10A5F000CDD0C5E7104D84ED038A012323720023DB
:10A60000236105F110030FCB85E80F00BFE7BDEC18
:10A61000048B70BD982C00200000C84235FA8E3C97
:10A620000AD7233CDB0FC93FA08B002000007A44EF
:10A63000985C002000000000808B002005207047FF
:10A6400000487047A8970C0800487047B8970C0856
:10A650000120704738B54A4D2DED028BD5F8BC0B63
:10A660009FED488A54F056FBD5F8D43B07EE903A5C
:10A67000F8EEE77A05F5405427EE800AA5F500507C
:10A68000BDEEC00A10EE103AC4F80C34F8F764FEC0
:10A69000D5F8C00B54F03EFBB5EEC00AF1EE10FA4F
:10A6A000DABF05F6D833D3ED007AD5EDCB7A36484C
:10A6B000CBBF20EE270A20EE270A20EE080A28EE5C
:10A6C000400ABDEEC00A10EE103AC4F81034F8F794
:10A6D0000FFE95EDCB7AD4F8100405F6D83327EEAB
:10A6E000087AD3ED007A27EE888AFDEEC77A17EE56
:10A6F000902AFDEEC87A17EE901A1EF08BFFC4F870
:10A7000010042148FDF7E6FF20B1D4F810345B4275
:10A71000C4F810341D4B93F8883D63B195F980332C
:10A72000022B08D1002301214620C4F80C34C4F8C0
:10A73000103456F04FF954F0FDF95F2155F0A2FAAC
:10A74000D8B155F06FFA022817D194F8A933A3B9FC
:10A7500094EDDF7AD5EDF37AB4EEE77AF1EE10FA04
:10A760000BD5012384F8A933BDEC028B084A0948B4
:10A77000BDE8384004214BF01FBEBDEC028B38BD54
:10A78000984C00200000C842982C0020986C0020B3
:10A79000C0970C081860002010B50446FFF736F883
:10A7A0002046BDE81040FFF79FB900000620704723
:10A7B000004870473C980C08004870474C980C08BB
:10A7C0000120704701207047012070470120704729
:10A7D0007047000008B50248FCF720F8012008BDCA
:10A7E000982C002038B50F4C04F50055D5F8BC0B5B
:10A7F00054F090FA05F6D432D2ED007AF8EEE77A0A
:10A8000004F5A04327EE800A2046BDEEC00A10EEF4
:10A81000102AC3F80C24F8F79FFD2046BDE8384005
:10A8200001F070B9982C00200F2070470048704745
:10A83000C0980C0800487047C8980C080120704761
:10A8400001207047012070470120704701207047A8
:10A850007FB50B4D05F54053002283F87A2305F5AB
:10A86000BD43783306460FCB6C4684E80F000023C7
:10A870002846B3602146FCF791FB012004B070BD6F
:10A88000982C002010B53B4CD4F8C833002B2CDD9D
:10A890007AF0CEFCD4F8C833C01A40F6B7339842E9
:10A8A00023D8A4F54053D4F8BC03D3F8D42B514299
:10A8B0001EF0B0FEC4F80C04A4F5A040F8F74CFD5F
:10A8C000D4F8CC33002B14DC2B48F8F7E1FC2B48F0
:10A8D00090F87A3393B30121A0F5405002F01EF8AE
:10A8E000BDE81040462055F01BBD2348F8F7CEFDCB
:10A8F000E6E77AF09DFCD4F8CC33C01A40F6B733C3
:10A900009842E1D81E4BDFED1F6A93EDCB7AD4F865
:10A91000C00303F6D833D3ED007A27EE267A67EE2C
:10A92000A67ABDEEC77AFDEEE77A17EE102A17EE8B
:10A93000901A1EF06FFEC4F81004C8E7A0F580500E
:10A9400090F90B33012B04DCBDE810400A48F8F7FE
:10A9500087BAD4F8D833002BF6D07AF069FCD4F853
:10A96000D833C01A40F6B7339842EDD894EDF50AC3
:10A97000B6E700BF987C0020982C0020985C00204F
:10A98000984C00200000C842D0ED027A0348FCEE4B
:10A99000E77A17EE903A99B201F07ABA982C002033
:10A9A00084B010B503AC84E80E000B4821466F223A
:10A9B000FCF73AFA9DF80C1011F0040102D1204680
:10A9C0000DF084FA04482146FCF7E8FABDE810408F
:10A9D000012004B0704700BF982C0020B0EEC00AE0
:10A9E000FDEEC07A38B54FF6FF7205460C4617EEFD
:10A9F000900A00211EF00EFE07EE900A002CF8EEE1
:10AA0000E77A054BC5ED027A14BF4FF0FF32012201
:10AA100083F8C02E38BD00BF987C0020FEF782BEB0
:10AA20000C207047004870473C990C08004870475C
:10AA300071D40D0801207047012070470120704734
:10AA4000012070470120704708B50C48FDF7E2F877
:10AA50000A480B49FBF714FF0848F7F76DFF40B1B0
:10AA600006484FF48051F7F787FD10B10348FBF714
:10AA7000D5FE024800F0C0FD012008BD982C002042
:10AA8000A08B002008B50D48F8F700FD0B48F7F73C
:10AA900053FF50B109484FF48051F7F76DFD20B1D5
:10AAA000BDE80840054801F02DB80448F8F7F0FB70
:10AAB000BDE808400148F8F7D3B900BF982C002042
:10AAC00008B50A484FF48051F7F756FD38B10848E9
:10AAD0000022D0F8181F00F608700DF033F9BDE819
:10AAE00008400248002101F0D3B900BF982C002093
:10AAF000987C0020881A10B51EF0B4FC104BD3F8D7
:10AB0000BC2E0028B8BF4042002AB8BF524248F6C7
:10AB1000A041B2FBF1F24FF47A7102FB01118842BD
:10AB20000CDC93F8082FD20606D503F6087403F65A
:10AB3000F8630FCB84E80F00012000E0002010BD77
:10AB4000987C002084B070B52DED048B86B00FADDD
:10AB500085E80E004E4CDFED4F8A0646D4F8A80576
:10AB600004F5005404F6D46393ED000A0368B0EED4
:10AB7000C00A5B6A9847B4EEE80AF1EE10FAB0EE4C
:10AB8000408A07DA012006B0BDEC048BBDE87040B6
:10AB900004B07047404928460DF03CFB02A8CDEDBB
:10ABA000030A8DED020A20F01FFE04A88DED040AB1
:10ABB000B0EE480ACDED050A20F010FD13A9284695
:10ABC0008DED000ACDED010A0DF024FB02A88DEDFC
:10ABD000020ACDED030A20F0ADFDB4EEE80AF1EE75
:10ABE00010FACFDBB4EEC08AF1EE10FA9FED2B9A8B
:10ABF000DFED2B8ADFED2B9A2BD802A8694620F0D7
:10AC0000DDFC04A88DED040ACDED050A20F048FD19
:10AC1000684620EE098A20F043FD94F9C03E07EE15
:10AC2000903AF8EEE77A28EE288AA7EEA90A1EF0F5
:10AC30003DFC20EE090ABDEEC88A20EE280A18EE77
:10AC4000101AFDEEC07A304617EE902AFFF752FF39
:10AC500099E738EE400A38EE088A80EE080AA2F03A
:10AC600015F802A8B0EE408A20F01AFD94F9C03E13
:10AC7000F0EE007AB0EE697AA8EE677A07EE903AC5
:10AC8000F8EEE77AA7EE270A1EF010FCC0E700BF37
:10AC9000985C002000000034908B0020E02E65427C
:10ACA0000000C842DB0FC93F10B504460848F7F75B
:10ACB00043FE20B92046BDE81040FEF733BD0448EE
:10ACC0004FF48051F7F758FC0028F3D010BD00BFB7
:10ACD000982C00200020704700487047B0990C085D
:10ACE00000487047B8990C08002070470020704752
:10ACF00038B5154C05460021204601F045FC0420DE
:10AD000055F00EFB0021204601F048FC132055F0C1
:10AD100007FB0021204601F04BFC2846FEF7D2FE3F
:10AD20002046012101F0FAFD462055F0F9FA6B6842
:10AD300004F5A044D3F8F831C4F80C346B68D3F8A8
:10AD4000FC31C4F8103438BD982C0020FEF79ABEB0
:10AD50000B2070470048704773920C0800487047FA
:10AD60002C9A0C0801207047012070470120704781
:10AD70000020704770B50B4E06F5A04505F6F86348
:10AD80000FCB05F6E86484E80F003046FBF7E8F8DF
:10AD900001463046FCF7D0F9002385F8783F0120C2
:10ADA00070BD00BF982C002038B53048F8F76EFB16
:10ADB0002E48F8F76DFA2D48F8F752F82B48102175
:10ADC000F7F7DAFBE0B12A4AD2F8FC3ED2F80C2FB2
:10ADD0009342D4BF00230123254C94F8782F72B9F5
:10ADE00073B304F6F8630FCB04F6E86585E80F004B
:10ADF000A4F5A040FBF70EFB012384F8783F38BD93
:10AE00001C4AB2F9A41B0029F9DD02F540529FED5E
:10AE10001A7AD2F8FC3ED2F8EC2E9B1A07EE903A42
:10AE2000F8EEE77A67EE877A07EE101AB8EEC77A7F
:10AE3000F4EEC77AF1EE10FACCBF01230023CBE782
:10AE4000A4F54053642193F9DC23D4F80C0412FBDD
:10AE500001F2D3F8D41B8A42A8BF0A465142C3F874
:10AE6000D42B1EF0D7FBC4F80C04C8E7982C0020A4
:10AE7000987C0020984C00200AD7233C38B52B4DF5
:10AE8000B5F9703383EAE371A1EBE37189B205F59B
:10AE9000405431B1002BB4BF4FF0FF33012384F88D
:10AEA000C03E234800F0F4FF94F8AA33F3B995F9B3
:10AEB0004B33022B1BD11F4D95F89D3D9BB11E4975
:10AEC000A1F6DC2024F074F968B1012384F855342C
:10AED000282205F60851A5F5804003F077F828B937
:10AEE000002384F85534012384F8AA3338BD012B9C
:10AEF0000CD10F4800F0E8FE40B10D48FBF744FAD2
:10AF00000028B8BF4042B0F57A7FD4DB95F94B33C7
:10AF1000042BEBD1074D95F89D3D002BE3D006495E
:10AF2000A1F6DC2024F0C0F9CEE700BF984C002049
:10AF3000982C0020986C0020908B002002207047F5
:10AF400000487047A09A0C080048704766D40D0866
:10AF5000034B0022C3F80C24C3F81024704700BF31
:10AF6000987C002038B5094D04462846F7F75AFD6D
:10AF70002846F7F7F7FD2046F7F70CFE2846F8F7C6
:10AF80001BF92046BDE83840FEF7AEBD982C0020E6
:10AF90000D20704700487047189B0C080048704708
:10AFA000209B0C080120704701207047012070474A
:10AFB0000023C37480F82430012070470148002129
:10AFC00000F066BF982C0020F0B5B54CD4F8042FE3
:10AFD000D4F8003F2DED088B1343D4F8FC2E134317
:10AFE00089B005460FD1AF48F8F750FAAD48F8F7E9
:10AFF0004FF99FEDAD0A462009B0BDEC088BBDE8C6
:10B00000F04055F08DB906F023FE90F87C32DB0756
:10B01000E9D5B5F90830E97C09EE103AB5F91030F8
:10B0200008EE903AB8EEC99AF8EEE88A002940F0A6
:10B03000D7809FED9EAA29EE0ABA0122FDEECB7AB7
:10B04000A4F5A040C4EDDD7AFAF7B6FF686800F514
:10B050007F700790B0EE408A20F022FBDFED947AFB
:10B0600020EE270A1EF0A0F90798F0EE409A20F093
:10B0700061FBA4F5A040F0EE40AAFEF76DF80028B1
:10B0800079D104F6F86696E80F0005F1140787E811
:10B090000F0096E80F0004F6E86787E80F0004F653
:10B0A000087787E80F00D4F80C3F824807EE903A03
:10B0B000F8EEE77AF0EE680A77EE8B7AB0EE690A7E
:10B0C000FDEEE77A17EE903AC4F80C3F0DF00CFA5B
:10B0D000002384F8E13395F91230724803EB8303BF
:10B0E00003EB83039B000121A4F8A233F6F78AFF48
:10B0F00094F8F073002F73D16F4B9FED707AB3F912
:10B10000143307EE903AF8EEE77A67EE877AF4EEBA
:10B11000E7AAF1EE10FA63DD52F01AF8064619EECE
:10B12000900AF5F7F1F9CDE9040118EE900AF5F768
:10B13000EBF9CDE9020119EE100AF5F7E5F9604ADD
:10B14000CDE90001062130464BF036F97AF070F86F
:10B15000C4F86073C4F84C037AF06AF80123C4F8A9
:10B160005C0329EE8A0AEB741EF048F9BDEEC00AB2
:10B1700084EDD90A34E07AF05BF8D4F80434C01ACC
:10B1800042F2107398427FF67CAFF0EE087AF4EE4C
:10B19000E7AAF1EE10FA7FF774AFBCEEC88A04F6A6
:10B1A000087718EE103A9BB208EE103AB8EEC88A4B
:10B1B00004F6F866B4EEC89AF1EE10FA46D851F0EB
:10B1C000C7FF404A06214BF0F7F896E80F0087E8E2
:10B1D0000F000123EB740321A4F5A040F6F712FF42
:10B1E000304803F0EFFC28B12E480321F6F70AFFA0
:10B1F0000023EB74D4F8F833012B40F0B480D4F87A
:10B20000FC3EAA699FED29AA9B1A07EE903AD4F852
:10B2100064330133F8EEE79A5CD0DFED2B7AE9EE88
:10B220000A7AF4EEE79AF1EE10FA0ADA274905F104
:10B2300014000DF0E3F8F4EEC08AF1EE10FA00F21B
:10B24000928018480321F6F7DDFE8CE051F080FF74
:10B250001F4A06214BF0B0F896E80F0005F1140CD8
:10B260008CE80F0096E80F0087E80F00D4F80C3F39
:10B2700007EE903A39EE488AF8EEE77AF0EE680A7F
:10B28000E8EE0A7A3846B0EE690AFDEEE77A17EE84
:10B29000903AC4F80C3F0DF027F90121E9749BE7BF
:10B2A000987C0020982C0020000000000000C8427C
:10B2B000E02E6542A08B0020984C00209A99993E80
:10B2C000699B0C08289B0C08000048C3908B002049
:10B2D000449B0C08B5F90A3007EE903AF8EEE77A8D
:10B2E00005F1140667EE8A7AF4EEE79AF1EE10FAA9
:10B2F00053DB434930460CF051FFDFED427AB6EEA6
:10B30000008AA0EE278A96E80F00BDEEC88A9FED5E
:10B310003E0AB8EEC88A04F6087728EE008A87E865
:10B320000F00F0EE680A3948B0EE480A0DF0DCF87C
:10B33000D4F80C3F07EE903AF8EEE77A28EE0A0AC6
:10B34000E9EE0A7AFDEEE77A17EE903AC4F80C3F80
:10B350001EF054F8BDEEC00A84EDD90AD4F8F833D3
:10B36000012B3FF45AAF2A4803F00CFC18B12848CF
:10B370000321F6F747FED4F8F833012B17D1244800
:10B3800003F0A0F9224803F0D7FA214809B0BDEC38
:10B39000088BBDE8F04003F0F3B9194930460DF0D1
:10B3A0002DF8F4EEC08AF1EE10FAA2D9D6E795F89E
:10B3B00024302BB9174861F085FA012385F8243031
:10B3C0001348F8F763F81248F7F762FF1048F7F7E9
:10B3D00047FD114890F87C336BB1002380F87C3333
:10B3E00033220221A0F5405009B0BDEC088BBDE826
:10B3F000F040FDF71BBB09B0BDEC088BF0BD00BFF2
:10B40000908B0020A00CB3450AD7233CA08B0020D2
:10B41000982C0020484E0020985C002010B504466F
:10B42000FEF760FA2046054B40F8143B0CF084FC14
:10B43000204603493EF052FF204610BD1C9C0C08DC
:10B44000B49B0C080320704700487047809C0C0890
:10B45000004870478C9C0C08F8B52A4D064600271A
:10B46000A5F54050A5F87873F7F776FF7368A5F552
:10B470008052D3F8F811D2F8D43B994205F5005424
:10B4800021DBC4F80C34736892EDCB7AD3ED7F6A7C
:10B490009FED1D6AF8EEE66A27EE067AF4EEC76ABB
:10B4A000F1EE10FA18DBBDEEC77A17EE103A174826
:10B4B000C4F81034FDF70EF920B1D4F810345B4213
:10B4C000C4F81034F8BD5B429942DADD012385F8F7
:10B4D0007833C4F80C74D6E702F6D832D2ED007A8D
:10B4E00067EE867AF4EEE76AF1EE10FA93BFFDEEAE
:10B4F000E77A012385F8793317EE903A88BF002365
:10B50000D5E700BF985C00200000C842982C0020BE
:10B5100070B500212DED028B04463448344D01F006
:10B5200033F832480021F0EE408A01F037F895F800
:10B530007833B0EE408AD3B1B0EE680A042054F0FC
:10B54000EFFE95F8793393B3B0EE480A132054F028
:10B55000E7FE2648002101F02BF82046FEF7B2FA5C
:10B56000BDEC028B2046BDE87040FEF7BDBA05F584
:10B570000056A5F54050F7F755FAD6F80C34002BD5
:10B580000CDCD6F80C34002BDBDA042054F0DCFEA3
:10B59000B4EEE80AF1EE10FACED4D2E7042054F06B
:10B5A000D3FEB4EEE80AF1EE10FAEADDC4E7114D7D
:10B5B0000E48F7F7D7FAD5F81034002B0CDCD5F885
:10B5C0001034002BC5DA132054F0BEFEB4EEC80AC6
:10B5D000F1EE10FAB8D4BCE7132054F0B5FEB4EE87
:10B5E000C80AF1EE10FAEADDAEE700BF982C0020A1
:10B5F000985C0020987C002000F5A0400023C0F853
:10B60000BC3EC0F8B83E80F8C13E80F8C23E7047EC
:10B6100000F58043D3F8A43D002BCBBF07EE903A52
:10B6200000F50050B8EEE70ADFED037ADCBF90EDDD
:10B63000C60A20EE270A70470000C8422DE9F041F3
:10B640002DED028B00F5985784B09FEDC98A103715
:10B65000054603A938468DED038A06F0DDF8B0B142
:10B660009FEDC47ADDED037A05F5A84367EE877A8E
:10B67000D3ED066A9FEDC07AE6EE877AF4EE487A5B
:10B68000F1EE10FA48BFF0EE487AC3ED067A28468C
:10B69000F7F7A4F805F58044B0EE408AF0EE000A12
:10B6A0009FEDB30A1DF0EEFF04F6BC53D3ED007A14
:10B6B00038EE678A05F50056E0EE087AC3ED007AA9
:10B6C00094F8883D002B40F09380D4F8742D05F554
:10B6D000994364339A4205D005F599436C339A42F5
:10B6E00040F0868008212846F6F746FF804630B1B4
:10B6F000D6EDC67A9FEDA17A67EE877A73E00221D4
:10B700002846F6F739FF0146002855D0D6F8C43B45
:10B710001B8B2846414608EE103A01F0FFF8D6F898
:10B72000C40B4369B8EE488AB0EE401A2BB3012B24
:10B7300028D0DFED937AF0EE671A96EDC60A9FEDFA
:10B740008F7AF4EEC17AF1EE10FA20EE070A4FF08C
:10B75000640124DBB6F8142312FB01F2B0EE672A71
:10B7600007EE902AF0EE400AB8EEE70A1DF0E4FD7D
:10B77000BDEEC00A10EE103AECE0DFED817AF1EE9A
:10B78000481ADAE78DED010A53F036FA07EE900A0F
:10B79000DFED7B1A9DED011AF8EEE77ACDE7B6F8FA
:10B7A000163313FB01F300EE903AB0EE482AF8EEA0
:10B7B000E00AF0EE671AD9E7B6F91423B6F91633A2
:10B7C0009B1A07EE903A2846B8EEE78A01F0A6F8F1
:10B7D000B6F81433642213FB02F307EE903AF8EE46
:10B7E000E77AE8EE007AFDEEE77A17EE903AB1E0FC
:10B7F00005F5A043D3F8F833042B40F0A08005F5FD
:10B80000BB40503077F05CFBC4F8A00DD4F8740D49
:10B8100003689B6B984700285ED094F8B43D002BDA
:10B820005AD0D4F8743D05F599451C35AB4253D038
:10B83000D4F8A03D9FED537A07EE903AD4F8B03D8E
:10B84000F8EEE77A384627EE878A07EE903AF8EE68
:10B85000E78A68EE878A06F0EBF9C8EE807A04F68C
:10B86000B8539DED037A77EE877AB6EE007AB4EEA0
:10B87000E78AF1EE10FA4CBF77EEC87ADFED407A36
:10B8800077EE877A93ED007AFDEEE77AF8EEE77AC5
:10B89000B4EEE77AF1EE10FA0ADD37EE676ADFED13
:10B8A0003A6AB4EE666AF1EE10FA48BFF0EE477AF3
:10B8B00004F6B853C3ED007AD4F8A03DDFED2F6A4B
:10B8C00007EE103AB8EEC77AA7EEA67ABDEEC77AB1
:10B8D00017EE103AC4F8A03DD4F8740D03681B6B42
:10B8E000984740B1B4F9AC2D002AC2BFD4F8A03DAE
:10B8F0009B18C4F8A03DB6F91623B6F91413D4F872
:10B90000A00D64235A4359431DF084FEC4F8A00DD2
:10B9100006F54763D6F8800C93ED4A8A06F088F95D
:10B92000C8EE007A04F6A8549DED037A77EEC77A44
:10B93000C4ED007A04B0BDEC028BBDE8F081D4F810
:10B94000742D05F59A4330339A4206D1D4F8A43DBC
:10B95000002B02DDC4F8A03D58E705F59A430833F3
:10B960009A427FF4C5AE2846FFF752FE00E700BFBB
:10B97000CDCCCC3DCDCC4C3ECDCC4C3F0000C842D4
:10B98000000000000AD7233C9A99993F30B500F592
:10B99000985587B010350023044628460393049336
:10B9A000059305F009F8002843D003A9284605F0BF
:10B9B00061FF00283DD004F5B15393ED047ADFED2B
:10B9C000216A8DED017AB0EEC77AD3ED077AB4EE35
:10B9D000E67AF1EE10FACDED027A06D5F0EEE77ACE
:10B9E000F4EEE67AF1EE10FA2AD401A81FF0F4FE84
:10B9F00003A901A81FF038FE04F5005393EDC87A9F
:10BA0000B5EEC07AF1EE10FAC4BFDFED0F7A27EE83
:10BA1000C00A04F58044C6BFA7EE270A012300230D
:10BA200084F8B43DCABFFDEEC07A002317EE903A09
:10BA300004E004F58044002384F8B43DC4F8B03D2C
:10BA400007B030BD000000340000C8422DE9F041CD
:10BA50002DED028B00F5A04607EE901AD6F8C43EF5
:10BA600000F5BE45B8EE678A0446083500F5405734
:10BA7000BBBB00F58043D3F8742D00F59A4308331F
:10BA80009A4204D000F59A4330339A4229D196F86D
:10BA9000A83333B304F5BD40294678300CF0AEFC32
:10BAA000D7F8A8050368F0EE408A5B6AB0EE480A52
:10BAB0009847F0EE087A60EE277AF4EEE78AF1EE26
:10BAC00010FA0EDDBDEC028BD7F8A8059FED0C0A2D
:10BAD000036804F5BD412A469B6ABDE8F041683120
:10BAE0001847B0EE480ABDEC028BD7F8A80596F9C6
:10BAF000C02E03682946DB6ABDE8F041184700BF45
:10BB00000000000070B504462DED028B04F5A04541
:10BB100079F082FBD5F8303F474AC31A9342064674
:10BB200072D907EE903AB8EE670ADFED447A9FEDDE
:10BB3000441ADFED440A20EE270A40F295101DF06A
:10BB4000C9FCC5F8306F04F50056DFED3F7AD6F832
:10BB5000C03BB3F9083008EE103A96F97233B8EEEC
:10BB6000C88AF0EE408A28EE278A0BB1B1EE488AE7
:10BB70009FED367ADFED367AB4EEC78AF1EE10FA31
:10BB800052DA05F62C73D3ED006AF4EEC76AF1EED3
:10BB900010FAB4EEE78AACBF01230023F1EE10FAED
:10BBA0003FD905F62C7292ED007AB4EEE77AF1EE09
:10BBB00010FA36D82046FAF731FE96F9733300EEC4
:10BBC000103A06F6984306F54A66D6ED000A93ED5C
:10BBD000001AB8EEC00A40F2A710F1EE600A20EE9B
:10BBE000080A1DF077FC28EE800ADFED1A8A20EEA5
:10BBF000280A2046FDEEC07A05F62C7517EE901A3D
:10BC0000FAF7CAFD85ED008A2046FAF717FA2046B2
:10BC1000F7F726F9BDEC028B2046BDE87040F7F738
:10BC200037BB002BC6D1C8E7B4EEE78AF1EE10FAB5
:10BC3000C3D90023B5E700BF9F860100BD37863515
:10BC40009A99193ECDCCCC3D53046939000000349B
:10BC5000000000B40000C84270B5044600F5A840DA
:10BC60004FF0FF311C3022F027FC431C054604F541
:10BC7000A04603D1114BC6F8803370BD04F5BE4118
:10BC800004F5BD40083168300CF088FA9FED0C7A5D
:10BC9000F6EE007AE0EE077AFDEEE77A17EE900A0C
:10BCA000281A1DF0DFFB07EE900A9FED067AF8EEEA
:10BCB000E77A67EE877AC6EDE07ADEE70000B44205
:10BCC000A00CB3450AD7233C00F54050D0F8A80596
:10BCD00003689B6B18470000F7B500F54053054615
:10BCE000D3F8A80503681B69984707462846FFF75D
:10BCF000EBFF05F5A0440646D4F8BC0E002862D13F
:10BD00003EB1D4F8FC3EC4F8C83E3E4BC4F8CC3E2D
:10BD10000120C4F8B47E1DF0A5FBD4F8BC3E94F914
:10BD2000C02E00FB0230C4F8BC0E3EB300230193CA
:10BD300094F8203F002B4AD094F8CC3D022B46D1FA
:10BD400005F5AA40012201A9343044F0DFFB0028A8
:10BD50003DD0D4F8243FDFED2C6A07EE903AB8EEE0
:10BD6000E77ADDED017AE7EE667AB1EE047AF0EE7D
:10BD7000E77AF4EEC77AF1EE10FA33D494F8C13EC4
:10BD8000002B3DD1D4F8BC3ED4F8CC2E002BB8BF4C
:10BD90005B42934234DBD4F8FC1ED4F8C83EC4F8AE
:10BDA000C81ECB1A03F2F31340F2E630834202F5C9
:10BDB000D2328CBF0023012302F5F07284F8C23E18
:10BDC000C4F8CC2E1CE0D4F8B43EF81AA1E7D4F89D
:10BDD000182FD4F8FC3E9B1A03F2F31340F2E6321C
:10BDE0009342CBD8012384F8C13E002384F8C23E9D
:10BDF000D4F8BC3E03F5D23303F5F073C4F8CC3E5F
:10BE000003B0F0BDE0A501000AD7233C2DE9F041C5
:10BE100000F58048044698F89D3DA3B300F5A04581
:10BE2000D5F8103F13B9D5F8143F63B304F5BD46F8
:10BE300004F5BE47204678360837FBF715F8394633
:10BE400030460CF0DBFA04F5BD413A466831304625
:10BE500085EDE30A0CF008FADFED0C0A85EDE40A43
:10BE60007620B7EE001A1DF035FB04F5315320465D
:10BE700083ED7D0AFFF730FFD8F8740D0368BDE845
:10BE8000F041DB6A1847BDE8F08100BF0000000008
:10BE9000012938B5044600F5A04512D800F5005335
:10BEA00095F8082FB3F93E3383EAE371A1EBE37110
:10BEB00089B2012998BF3C21920730D5FF2385F82C
:10BEC000C03E07EE901AF8EE677A05F6D463C3ED2C
:10BED000007A2046FFF7BAFDD5F8C43E2BBB2046BA
:10BEE000FFF7F2FE40B995EDE47AF7EE007AB4EE92
:10BEF000E77AF1EE10FA18DD79F09AF904F580434B
:10BF0000C5F8C40ED3F8740D03681B6A984760B176
:10BF100004F54E500021BDE838404EF031BC002BF6
:10BF2000B4BF4FF0FF330123C9E738BD10B500F5AA
:10BF3000AA44143420465CF021F92046BDE81040A4
:10BF40005CF08CB910B500F5A043044693F8283591
:10BF50009A0716D45B074FF002014CBF094A0A4A00
:10BF600000F54E504AF028FA04F5AA4014305CF06F
:10BF7000D9F804F52D500121BDE810402C3062F0B5
:10BF80007FBC10BD009D0C081A9D0C0870B500F513
:10BF9000A046054696F914459CB196F82835C3F39A
:10BFA00080045B0728D4B6F91A35002B0BDC284631
:10BFB000FFF7C8FF05F52D5001212C3062F060FC21
:10BFC0000124204670BD2146FAF720F8B6F91A354B
:10BFD00007EE903AF8EEE77AB4EEE70AF1EE10FADF
:10BFE000E5D5D6F89433002BE1D0044A042105F5B9
:10BFF0004E504AF0E1F9E4E70024E2E7309D0C08F6
:10C0000008B52DED028B08EE901A30B3F2B1B0F9FD
:10C01000083008EE103AB8EEC88AF8EEE88A9FEDCC
:10C02000100ADFED100A28EE800ADFED0F8A4FF4C8
:10C03000D470B7EE001A1DF04DFAC8EE280A1DF0B4
:10C04000A5F920EE280ABDEC028B08BD52F058FE7F
:10C0500007EE900AB8EEE78ADFE79FED020AF2E703
:10C060000AD7233C0000000000A08C4537B500F53E
:10C070000054054694F99F33002B52D052F05AFDDC
:10C0800052F04EFDC4F8BC0B52F054FD52F034FD9A
:10C09000C4F8C00B52F04EFD52F038FDC4F8C40B8A
:10C0A00052F048FD52F03CFD41F29411C4F8C80B27
:10C0B000D4F8BC0B52F088FDD4F8C00B41F29411B7
:10C0C00052F082FDD4F8C80B41F2941152F07CFD7D
:10C0D000284600F01DFC48BBD4F8C40B642152F084
:10C0E0006FFD52F027FDD02153F0CCFDC4F8CC0BEE
:10C0F00052F020FDD22153F0C5FDC4F8D00B05F558
:10C100001D5004304921019054F04AFB01984A2106
:10C1100054F046FB0198462103B0BDE8304054F08E
:10C120003FBB52F007FD52F0DDFCABE705F5C04325
:10C13000D4F8C40B93F8AC30642173B152F040FDD5
:10C140006421462054F024FA6421492054F020FA56
:10C1500064214A2054F01CFAC3E752F035FDEFE7A2
:10C1600010B500F500541E21D4F8BC0B52F030FD80
:10C17000D4F8C00B1E2152F02BFDD4F8C80B1E21A1
:10C1800052F026FDD4F8C40B1E21BDE8104052F039
:10C190001FBD000007B500F0BBFB014658B9019078
:10C1A000462054F017F90199492054F013F90199E8
:10C1B0004A2054F00FF90021042054F0DDFB002147
:10C1C000132054F0D9FB0021462054F0D5FB002168
:10C1D000492054F0D1FB00214A2054F0CDFB00212E
:10C1E000152003B05DF804EB54F0C6BB10B504464F
:10C1F00054F008FE54F058FA204601F0C5FCBDE8A2
:10C20000104054F007BD000038B500F50055044655
:10C2100095F99F330BB1002038BD0121F6F7ACF939
:10C2200090B104F58043D3F8742D04F59A43443358
:10C230009A4209D004F5994324339A4204D004F574
:10C24000994334339A42E6D12046F6F775FB00282D
:10C25000E1D0D5F8C83BB3F90800DDE738B52DEDDE
:10C26000028B00F5804393F8883D002B40F0B780A7
:10C270005C4A00F59A43D2F8742D44339A4200F593
:10C280004E5508D0584A0321BDEC028B2846BDE824
:10C2900038404AF091B800F500549FED546AD4F844
:10C2A000BC2BB2F90830002BB8BF5B429BB207EE43
:10C2B000903A138B06EE903AF8EEE66AF8EEE77ADB
:10C2C00066EE866AF4EEE67AF1EE10FA17DCD4F840
:10C2D000C02BB2F90830002BB8BF5B429BB207EE0F
:10C2E000903A138B07EE103AB8EEC77AF8EEE77A79
:10C2F00027EE067AF4EEC77AF1EE10FA01DD3C4A39
:10C30000C1E700F5B15004301FF088FFDFED397A46
:10C3100020EE270AF3EE0E7AB4EEE70AF1EE10FAF9
:10C3200001DD354AAFE7042054F0DEFA132054F063
:10C33000DBFA152054F0D8FA4D2054F0D5FA4E20EF
:10C3400054F0D2FA4F2054F0CFFA502054F0CCFAE7
:10C35000152053F0F9FF9FED298AB0EEC00AB4EE24
:10C36000C80AF1EE10FA0BD5102054F0BDFA562091
:10C3700054F0BAFA112054F0B7FA572054F0B4FA36
:10C38000032053F0F1FFB0EEC00AB4EEC80AF1EE9C
:10C3900010FA0FD5022053F0E7FFB0EEC00AB4EE5A
:10C3A000C80AF1EE10FA05D5182054F09DFA1920AC
:10C3B00054F09AFAD4F8BC0B811D0C303EF04CFEC0
:10C3C000D4F8C00B811D0C303EF046FED4F8C80BEB
:10C3D000811D0C303EF040FE094A052154E7BDECBA
:10C3E000028B38BD986C0020449D0C08CDCC4C3E8F
:10C3F000649D0C08E02E65428C9D0C080000003402
:10C40000A89D0C0810B500F5005494F976339BB143
:10C41000D4F8C40B52F0EAFBD4F8C42BB4F9783347
:10C4200030B1B2F906009842ACBF0020012010BD27
:10C43000B2F906008342F7E70120F8E710B5044699
:10C44000FFF7E0FF60B104F5804478F0F1FED4F826
:10C45000943DC01AB0F57A7F94BF0020012010BD32
:10C460000120FCE770B50546FFF7E8FF05F500542D
:10C4700008B3D4F8BC3B9A89DA80D4F8C03B9A89D7
:10C48000DA80D4F8C83B9A89DA80D4F8BC3B00261D
:10C490001E81D4F8C03B1E81D4F8C83B1E8105F52F
:10C4A0008043D3F8740DC3F8AC6D03685B6898479C
:10C4B000D4F8C43B1E8105F5C040043070F058FF2D
:10C4C00078B3002652F036FB437A13B952F032FBB0
:10C4D000837A94F97623012A22D106B103B3284640
:10C4E000FFF7ACFF05F5804494F88E3D30B301337F
:10C4F000DBB20A2B84F88E3D0BD11F4B1F4A04215F
:10C5000005F54E5049F058FF1D4A012384F8883D37
:10C51000937294F88E3D0A2B02D90A2384F88E3D3B
:10C5200070BD2846FCF718FE0028CAD152F002FB65
:10C5300052F0C4FA061E18BF0126C3E7002BEFD045
:10C54000013BDBB2032B88BF032384F88E3D94F8B4
:10C550008E3D012B08D105F54E500A4B074ABDE828
:10C560007040042149F028BF002BD9D1044A84F837
:10C57000883D9372D4E700BF93F90D08B89D0C086D
:10C58000058E00209B9F0C0800F500500A4690F98C
:10C59000A61BD0F8BC0BFFF733BD000000F5005020
:10C5A0000A4690F9A71BD0F8C00BFFF729BD000081
:10C5B00000F500500A4690F9A81BD0F8C80BFFF709
:10C5C0001FBD000010B54FF480610446F5F7D4FF9D
:10C5D00004F5005328B1BDE81040D3F8C40B52F065
:10C5E0008BBCBDE81040D3F8C40B52F08FBC0000E8
:10C5F0002DE9F04100F500530546D3F8C83BB3F9E7
:10C60000088000F5C044B8F1000F02D1012384F87E
:10C61000483005F5C0470437384670F0A9FE064695
:10C62000E0B9B8F57A6F2ADD78F002FE636C8046D7
:10C630008BB1C31A40F6B73293420DD905F5A04528
:10C64000012231463846F5F77DF9666484F8486082
:10C65000C5F83C8300E06064BDE8F08118F57A6FAE
:10C660000DDA78F0E5FD636C63B1C01A40F6B733BC
:10C670009842F1D9012200213846F5F789F90023C3
:10C680006364E9E76064E7E770B52DED028B04466B
:10C6900052F050FA52F008F930B9BDEC028B204646
:10C6A000BDE87040FFF7DEBE04F5804595F8883D93
:10C6B0001BB978F0BDFDC5F8980D2046FFF7A2FE26
:10C6C00018B178F0B5FDC5F8940D2046FFF7CAFE05
:10C6D0002046FCF7D1FB04F500560023C5F8AC3D1D
:10C6E00096F97A3363B3D6F8C43BB3F90830322BEA
:10C6F00026DD28B3323B1BB207EE903A04F5985082
:10C70000B8EEE78ADFED207A103028EE278A04F0B1
:10C710008DF838B3B6F9163396EDC67A07EE903A2F
:10C72000F8EEE77A77EEC77A27EE888ADFED177A98
:10C7300028EE278ABDEEC88A18EE103AA5F8AC3D5F
:10C740002046FFF755FFD5F8740D03685B689847DE
:10C75000BDEC028B014604F5C0405030BDE870408E
:10C7600054F044BF96F9093396F90B239B1A07EE50
:10C77000903AF8EEE77A27EE888ABDEEC88A18EE7E
:10C78000103AA5F8AE3DDBE70AD7A33C0000C8424B
:10C7900070B500F500540546D4F87C330BB9002081
:10C7A00041E094F90833002BF9DA00F58043D3F81F
:10C7B000740D03685B6898470138172832D801A3C5
:10C7C00053F820F0C1C80108FDC8010825C80108B8
:10C7D000F3C80108E9C80108D5C80108CBC8010899
:10C7E00025C8010825C8010829C80108B7C80108DB
:10C7F000ADC801089FC70108DFC80108DFC80108EC
:10C8000025C8010825C8010825C8010825C8010850
:10C8100025C8010825C8010825C8010825C8010840
:10C8200007C90108012070BD05F5A045B5F85A6497
:10C83000162EB4D0D4F87C1311F0020301F00102DB
:10C8400005D0A6F1150CDCF1000343EB0C0311F04D
:10C85000040043EA020303D0A6F11F0460426041D2
:10C8600043EA000211F0080007D01F2E1AD0A6F1EB
:10C87000110002288CBF0020012011F0100340EAB3
:10C88000020005D0102E0FD0A6F1520253425341A0
:10C89000034311F4006014BF95F82414014643EAE1
:10C8A0000100C0E70120E8E70123F1E7D4F87C03A9
:10C8B000C0F34010B7E7D4F87C03C0F38010B2E7B0
:10C8C000D4F87C03C0F3C010ADE7D4F87C03C0F308
:10C8D0000020A8E7D4F87C03C0F34020A3E7D4F8F5
:10C8E0007C03C0F380209EE7D4F87C03C0F30030C3
:10C8F00099E7D4F87C03C0F3403094E7D4F87C0384
:10C90000C0F380308FE7D4F87C03C0F3C0308AE7EF
:10C9100000F5005090F80803C009704738B5044688
:10C920000D4652F007F90368DB689847C8B104F573
:10C930000053D3F8C40B6DB152F0E2F907EE900A40
:10C94000B8EEE70A04F5C04494F8AB300BB1B1EE91
:10C95000400A38BDB0F9083000EE103AB8EEC00A0F
:10C96000F0E79FED010AF4E70000000038B52DED77
:10C97000028B04460D4652F0DDF80368DB689847E9
:10C9800000283FD0214BD3F8C43B5B69012B07D073
:10C99000BDEC028B29462046BDE83840FFF7BEBFFC
:10C9A0004FF480612046F5F7E7FD0028F0D004F54C
:10C9B0000053DFED177AD3F8C40B93F90B33028BD6
:10C9C00008EE903A00EE102AF8EEE88AB8EEC08A37
:10C9D00068EEA78A52F09EF9B6EE001AA0EE011A90
:10C9E00004F5C044DFED0B0AB0EE680A1CF0A0FDB0
:10C9F00094F8AB3028EE000A0BB1B1EE400ABDEC62
:10CA0000028B38BD9FED030AF9E700BF984C002068
:10CA10000AD7233C0000000073B500F5A04504468A
:10CA200095F8CC3D022B00F5546612D100F5AA40D2
:10CA3000012201A9343043F069FD50B1019BC6F8D1
:10CA40009C3230463EF008FF2046FAF76DF802B0FF
:10CA500070BDD5F8F833042B05D12046F9F73EFD1B
:10CA60008DED010AEAE705F634752B680193E5E7D9
:10CA700070B500F580460446D6F8740D03689B6BCC
:10CA80000D46984748B9D4ED460A9FED1C0A64212B
:10CA90002846BDE8704053F039BDD6F8740D04F552
:10CAA0009A4104F500520831884292F80A3392F90B
:10CAB000D4231FD104F5A04191F8A40350B94AB181
:10CAC000D3B204F5A041D1F8F8130139012998BF78
:10CAD000D3B207E091F94C0E60B1D1F8F8130429F4
:10CAE00008D1C3B207EE903AD4ED460AB8EE670A11
:10CAF0006421CDE7002AF5D0E3E700BF0000000085
:10CB00002DE9F04100F58048044604F59A43D8F831
:10CB1000740D4433984203D100252846BDE8F081C6
:10CB200003689B6B984750B104F5A04393F82855D0
:10CB300015F0010503D0012283F8F023EDE704F599
:10CB4000BB40503076F0F0FA054608B10125E4E725
:10CB500004F5A04696F8F033002BDDD0D8F8740D1C
:10CB600003689B6B984718B9002386F8F033D4E725
:10CB700094F8143494F85874B02202FB034393F8E9
:10CB8000F121B7BB012A0AD993ED837AF1EE047A39
:10CB9000B4EEE77AF1EE10FAACBF01270027D8F81F
:10CBA000742D04F59A4308339A4202D196F8A433BF
:10CBB00023B104F59A434C339A4240D104F5005313
:10CBC000204693F9C883FCF7C7FAA0B9204601F0C4
:10CBD0000BFC0028BAD0002386F8F03394F87124B7
:10CBE00004F58C63242101FB0233DB6AC6F89C3315
:10CBF00093E72F46D3E778F01BFBD6F804344FF4C5
:10CC0000FA62C01A642313FB082341F2883293426C
:10CC100038BF13469842D9D92046F9F7E5FBB0F55D
:10CC2000FA7FD3DD04F5805341F26E72D3F80C35F0
:10CC300003F6B7339342C9D8002FC7D094E706F65E
:10CC40003473D3ED007AB2EE047AF0EEE77AF4EEC4
:10CC5000C77AF1EE10FA87DA002F3FF477AF04F5C8
:10CC60009850103003F0E2FD00283FF47DAF04F54A
:10CC7000005304F5FF5093F84611183002F0F6FF08
:10CC8000F1EE047AB4EEE70AF1EE10FAFFF65EAFC9
:10CC90006AE70000F8B52DED048B044608461646F9
:10CCA0001D46BDF9287053F04FFB04F50054304683
:10CCB000B0EE408A53F048FBB4F9A423002AF0EE0A
:10CCC000408A37DAC2F1640307EE903A9FED207A8A
:10CCD000F8EEE77A67EE877A60EE278AD4EDE87A95
:10CCE0009FED1C1ADFED1C0A38EEC80ABC2020EEAE
:10CCF000270A1CF0EFFB38EE288AB0EE409A94ED3C
:10CD0000E80A9FED141ADFED140A28EE000ABD2090
:10CD10001CF0E0FB2846B0EE408AB0EE490A53F022
:10CD2000FFFAB0EE480ABDEC048B3846BDE8F84087
:10CD300053F0F6BAD2D002F1640307EE903A9FEDB9
:10CD4000047AF8EEE77A67EE877A28EE278AC5E755
:10CD50000AD7233C00A08C4500A08CC500B52DED62
:10CD6000048B042083B053F0EFFA0320B0EE408A26
:10CD700053F0FAFADFED189A9FED181ADFED180A52
:10CD80008DED011AF0EE408AB0EE480AA8EEA90A2D
:10CD9000CF20CDED000A1CF09DFBB0EE409AB0EE26
:10CDA000480A9DED011ADDED000AA8EEE90AD0203F
:10CDB0001CF090FB1820B0EE408AB0EE490A53F008
:10CDC000AFFAB0EE480A192003B0BDEC048B5DF851
:10CDD00004EB53F0A5BA00BF0000344200A08C451C
:10CDE00000A08CC5F8B52DED088B00F5005600F5B8
:10CDF000C04596F98E3B13F0040F03F0010203F0D7
:10CE0000020440F0F580D5F8B0707B1E5F425F41B0
:10CE1000002A00F0EF804D2053F096FA4E20F0EEFD
:10CE2000409A53F091FAB0EE408AB6F9A633DFED9E
:10CE300087AA0AEE103A1520B8EECAAA53F084FA6F
:10CE40002AEE2AAA20EE0AAA002C00F0DB80F0EEDF
:10CE5000488AB0EE699AB5EEC0AAF1EE10FA40F336
:10CE6000D6809FED7B1ADFED7B0A38EE0A0A4FF47D
:10CE700080701CF02FFB9FED761ADFED760AB0EE86
:10CE8000408A40F2011038EECA0A1CF023FBF0EE93
:10CE9000408A96F98F3B632B15DC07EE903A9FEDA5
:10CEA0006E7AF8EEE77AB4EEC79A67EEAA7AF1EEF8
:10CEB00010FAF4EEC78A98BF29EE279AF1EE10FA1D
:10CEC00098BF68EEA78AD5F8B03096F98C4B96F9E2
:10CED0008D6B022B00F0B48024B2002C01DC002EFC
:10CEE0006EDD032053F040FADFED5C7AB4EEE70A22
:10CEF000F1EE10FAB0EE40AA62DB002F00F0A28043
:10CF00009FED571ADFED570A40F2271030EE000A66
:10CF10001CF0E0FA9FED541ADFED520AB0EE40BA71
:10CF20004FF494703AEE410A1CF0D4FA70EE007A95
:10CF3000B0EE4BAA07EE104AF8EEC7AA9FED4BBA27
:10CF40009FED431ADFED430A6AEEA7AAB0EE690A25
:10CF500040F22B10AAEE8B0A1CF0BCFA07EE906A86
:10CF6000F0EE409AB8EEE70A9FED391ADFED390A84
:10CF70002AEE40AAB0EE490A4FF49670AAEE0B0AC8
:10CF80001CF0A8FAB0EE409AB0EE480A9FED301AB5
:10CF9000DFED300A40F22D10AAEE8B0A1CF09AFA4F
:10CFA000B0EE408AB0EE680AAAEE0B0A4FF4977012
:10CFB0009FED271ADFED270A1CF08CFAF0EE408A6D
:10CFC000B0EE690A102053F0ABF9B0EE490A5620D2
:10CFD00053F0A6F9B0EE480A112053F0A1F9B0EED3
:10CFE000680ABDEC088B5720BDE8F84053F098B9AB
:10CFF00001270DE7042053F0A7F9B0EE408AF1EEC7
:10D00000409A12E7DFED178AB0EE689A23E79FEDAA
:10D01000101ADFED100A39EECA0A4FF482701CF0C4
:10D0200059FA9FED0B1ADFED0B0AF0EE409A40F231
:10D03000051039EE0A0A1CF04DFAB0EE409A28E7C6
:10D0400000244CE7F0EE407A74E700BF0AD7233C97
:10D0500000A08C4500A08CC5000000B40000003486
:10D060000000C84200000000000048426666E63E3C
:10D0700038B52DED028B00F500550446D5F8D00BE0
:10D08000A0B304F5804393F8882D7ABB93F88E3DC6
:10D0900063BB51F0FBFE07EE900AB8EE678A4620AC
:10D0A00095F9085353F050F9002DF0EE408A20DA3C
:10D0B00004F5BB40503075F0B9FEE8B99FED101A89
:10D0C000DFED100A40F25110B1EE680A1CF002FACE
:10D0D000B4EE408AF1EE10FAC8BFB0EE480ABDECDB
:10D0E000028B6E20BDE8384053F01AB99FED058AD7
:10D0F000D5E79FED040AEBE79FED010AE8E700BFE3
:10D100000000C8420000000010B52DED028B4369FD
:10D11000002B4AD0037C0BB101330374037C002B3A
:10D1200041D0182B1FD803EB4303C3EB03139B0021
:10D130001CB2002307EE903AB8EEE78A0420B0EE66
:10D14000480A53F0EDF807EE904A1320B8EEE70ACC
:10D1500053F0E6F8B0EE480ABDEC028B1520BDE8AE
:10D16000104053F0DDB84A2B02D8C3F13203DAE79E
:10D17000632B01D8643BD6E77C2B08D8643B03EBD8
:10D180004303C3EB03139B001BB20024D2E7AE2B77
:10D1900002D8C3F19603F2E7C72B01D8C83BEEE7EC
:10D1A00000230374F1E71C46C4E7BDEC028B10BDFD
:10D1B00010B59FED1C7AD0ED017AF4EEC77A00230A
:10D1C000F1EE10FA044643722BDB90ED007AB4EED8
:10D1D000E77AF1EE10FA24D908F0F2F9217A07F093
:10D1E00043FED4ED010AF5EE007A60EEA77AB4EEC4
:10D1F000E70AF1EE10FA14D494ED001A40F2A510EB
:10D200001CF068F9F7EE007AB4EEE70AF1EE10FAD6
:10D2100007D494ED007AC7EE007A01236372C4ED5F
:10D22000037A10BD00000034437A7BB391F90030DB
:10D2300090ED037A07EE903AF8EEE77A67EE877A98
:10D240009FED137AF4EEC77AF1EE10FAD8BFF0EE44
:10D25000477AFDEEE77A17EE903A0B7092F90030BC
:10D2600090ED037A07EE903AF8EEE77A67EE877A68
:10D270009FED087AF4EEC77AF1EE10FA58BFF0EE9F
:10D28000477AFDEEE77A17EE903A1370704700BFC9
:10D290000000C8C20000C842437AF0EE407A5BB199
:10D2A00090ED030A9FED051ADFED050A27EE800ACF
:10D2B0004FF4E6701CF00EB9704700BF0000C84282
:10D2C0000000C8C2F8B504460E46174677F0B0FF16
:10D2D000054604F59B40403007F050FF04F5A0449C
:10D2E000D8B3462053F030F8DFED3D7AB4EEE70ACC
:10D2F000F1EE10FA10DB97F9002094F9F133193AA6
:10D30000934209DAD4F8F423AA4205D0C4F8F453BE
:10D31000013384F8F13344E0462053F015F8DFED93
:10D32000317AB4EEE70AF1EE10FA3AD896F9002015
:10D33000002A36DAC2F1FF2294F9F23302F57F02B5
:10D34000E73293422DDAD4F8F423AA4229D0C4F864
:10D35000F453013384F8F23323E0D4F8F433EB1AB6
:10D36000B3F57A7F1DD3462052F0EEFF94F9F133E6
:10D3700007EE903AF8EEE77AB4EEE70AF1EE10FA2B
:10D3800001DD002B22DC462052F0DEFF94F9F2335F
:10D3900007EE903AF8EEE77AB4EEE70AF1EE10FA0B
:10D3A00018D497F9000094F9F1230021821A1CF097
:10D3B00041F9387096F90000002806DA94F9F21362
:10D3C000002201441CF036F93070F8BDC4F8F45363
:10D3D000013B9EE7002BE4DDC4F8F453013BB9E7C1
:10D3E00000000034000000B410B52DED028B00F5F4
:10D3F000005282B092F9083392F809238DF8063072
:10D40000002B0446B0EE408A8DF8072004DAFFF7BF
:10D41000BFF908B98DF8060004F5A043D3F8F82346
:10D42000012A4CD0072A4AD004F5BB40503075F091
:10D43000FDFC002854D104F52E500DF106010DF12C
:10D4400007021030FFF7F0FE2046FFF73BFF9DF983
:10D4500006309DF90720DFED238A9342A8BF1346CB
:10D4600007EE903A04F53154B8EEE70A303420EE76
:10D47000280A20468DF8063074F0D0FE9DF907305A
:10D4800000EE103AB8EEC00A204620EE280A74F0EA
:10D49000CFFE9DF9073001EE103A9DF9063000EEFF
:10D4A000903AB8EEC11AF8EEE00A40F24D20B0EE24
:10D4B000480A1CF00FF802B0BDEC028B10BDD3ED92
:10D4C000D57AFDEEE77A17EE902AD3EDD67A8DF86D
:10D4D0000720FDEEE77A17EE903A8DF80630AAE7BE
:10D4E0000023FAE70AD7233C70B5044600F52E5511
:10D4F000103504F580462846FFF75AFED6F8740D1D
:10D5000003685B6D984740B1462052F01DFF2846E6
:10D51000FFF7C2FE462052F003FFD6F8740D0368F1
:10D520001B6D984740B1462052F00EFF2046FFF792
:10D530005BFF462052F0F4FE2046FFF7E1FA10B3FD
:10D5400004F5005595F9743343B101212046FFF7E6
:10D55000E5F9BDE87040462052F0E2BE04F5BB4458
:10D560005034204675F062FC50B1204675F0E6FD5F
:10D5700030B195F9083300EE103AB8EEC00AE8E78A
:10D580009FED010AE5E770BD0000000010B50446FC
:10D590002DED028B462052F0D7FE2046B0EE408A99
:10D5A000FBF7DAFD80BB04F5C04004306FF0E0FE0D
:10D5B00050B304F5AB53D3ED028A1BF053FA90F845
:10D5C00013339FED137A0C2202FB0300D0ED627A35
:10D5D000E8EEC77AF4EEC77AF1EE10FA0CDC04F547
:10D5E000005494F90B3307EE903AF8EEE77AF4EE34
:10D5F000C87AF1EE10FA07D5BDEC028B0548BDE8FC
:10D600001040012104F098BDBDEC028B10BD00BF9D
:10D610000AE81C41A83F00202DE9F04100F5005523
:10D620000646D5F8CC3BA3BB002706F58048D8F8C2
:10D63000740D03689B6B98470446002852D006F58A
:10D640009850103003F0F2F880B308F55A63D3ED28
:10D65000007A9FED3F7AF8EEE77A67EE877AFDEE83
:10D66000E77A17EE903A1BB295F9BB230AB19A42BA
:10D670001FDA95F9B943FCB906F5A042D2F8F833A0
:10D68000013B062B2ED8DFE803F01E2D24602D2D44
:10D690001E0051F04FFA0368DB6898470028C3D09A
:10D6A000D5F8CC0B51F0F2FB47B2BEE795F90B333E
:10D6B000DAE795F9BA43DFE724B29C42ACBF95F9AB
:10D6C000B8430024D8E795F9BC33002B18BF1C469B
:10D6D00008E095F9BC332BB13046FBF75BFD08B190
:10D6E00095F9BC4387EAE773A3EBE773DBB2A34288
:10D6F000C8BF3C4607EE904A0320B8EEE70A52F056
:10D700000FFE07EE907A0220B8EEE70A52F008FE0C
:10D7100095F9ED33D6ED460A00EE103A6421B8EEE5
:10D72000C00A032052F0F2FE95F9ED33D6ED460A19
:10D7300000EE103A0220B8EEC00A642152F0E6FE74
:10D740003046BDE8F041FFF709BB92F94B3EBCE71C
:10D750000AD7233C38B504462DED048B462052F001
:10D76000F3FD584BDFED587A93F9593B08EE903AA8
:10D77000F8EEE88A152068EEA78AB0EE408A52F0EB
:10D78000E3FD9FED527A20EE280A04F5C045C0EE75
:10D79000077A04F5BC405C30C5ED287A72F0A2FB34
:10D7A00010B10023C5F8A030B5EEC08AF1EE10FA32
:10D7B00043D52046FFF7ACF800287ED02046FEF780
:10D7C000E7FF002879D0D5ED287A9FED419A9FEDAB
:10D7D000411ADFED410AB0EE480AA7EE890A4FF47C
:10D7E0003B701BF077FED5ED287A9FED3A1ADFEDFE
:10D7F0003A0AF0EE408A40F2ED20B0EE480AA7EE79
:10D80000C90A1BF067FEB0EE408A04F5C045043536
:10D8100028466FF0B7FDD0BB284670F0B1FE022855
:10D8200027D10321492053F0D5F8BDEC048B032107
:10D83000BDE838404A2053F0CDB83ED9D5ED287A1E
:10D840009FED239A9FED251ADFED220AB0EE480ADC
:10D85000A7EE890A40F2F2201BF03CFED5ED287AB3
:10D860009FED1E1ADFED1B0AF0EE408A40F2F32016
:10D87000C3E79FED180A492052F052FDBDEC048B1E
:10D880009FED140ABDE838404A2052F049BDB0EE81
:10D89000680A492052F044FDB0EE480A4A2052F08E
:10D8A0003FFD20464921FFF7E3F8BDEC048B2046FD
:10D8B0004A21BDE83840FFF7DBB89FED068AF0EE5D
:10D8C000488AA2E7984C00200AD7233C00A08C4548
:10D8D00000004842000000000000C8C20000C8422A
:10D8E000F8B52DED028B00F5A046044696F9493EA9
:10D8F000002B32DD00F5804200F59A43D2F8742DFA
:10D9000008339A4229D196F9483E002B25DD00F5CF
:10D91000BB40503075F0FCFAF8B104F5C04004305B
:10D920006FF026FDC8B9124F9FED128A04463D687C
:10D930002D190ED0B5F9080052F018FB48B196F930
:10D94000493E012B0CD1B5F90800B0EE480A52F05F
:10D95000E7FC1434B4F5A07FE9D1BDEC028BF8BD2F
:10D96000022BF6D1B5F90800032153F033F8F0E7A4
:10D97000A09200200000000037B500F5A043044647
:10D9800093F850330BB39FED120A15204F2552F038
:10D99000C7FC20460095502313221521FFF77AF982
:10D9A000152052F05FFF80B9284652F05BFF60B946
:10D9B0009FED070A4E2052F0B3FC9FED050A4D2063
:10D9C00003B0BDE8304052F0ABBC03B030BD00BF87
:10D9D0000000000070470000F8B52DED048B00F545
:10D9E00080440546D4F8740D03689B6B984738B99A
:10D9F000D4F8742D05F599435C339A4240F0BE800B
:10DA000005F5C04004306FF0BDFC002800F0B68082
:10DA10002846FBF7A1FB002800F0B08005F5A046E2
:10DA2000D6F80C34002BB8BF5B42B3F52F7F00F360
:10DA3000A580D6F81034002BB8BF5B42B3F52F7F1A
:10DA400000F39C8077F0F4FBD6F8703FC31AB3F56F
:10DA5000FA7F0746C0F0928005F5B85393ED057A3A
:10DA6000F2EE007AB4EEE77AF1EE10FA00F1868079
:10DA700006F5836393ED007AB4EEE77AF1EE10FADF
:10DA80007CD405F5405393ED0B8AD3ED628A05F5FE
:10DA90001D540434B0EE480A0421204652F0B6FC6E
:10DAA000B0EE680A1321204652F0B0FC78EEC89A16
:10DAB0004D21B0EE690A204652F0A8FC38EE289AB3
:10DAC0004E21B0EE490A204652F0A0FCB0EE680AA2
:10DAD0004F21204652F09AFCB0EE680A50212046B1
:10DAE00052F094FC05F50055B0EE480A1821204686
:10DAF00052F08CFCB0EE480A1921204652F086FC08
:10DB000095F98E3B03F00202DB075CBFF1EE489A09
:10DB1000B0EE489A6AB3B0EE498AF0EE698AB0EE88
:10DB2000690A1021204652F071FCB0EE680A5621B5
:10DB3000204652F06BFCB0EE490A1121204652F00B
:10DB400065FCB0EE480A5721204652F05FFCD6F83B
:10DB5000743FC6F8707FFB1A42F2107293420DD9DF
:10DB6000C6F8747FBDEC048B2046BDE8F84053F046
:10DB700033B89FED048AF0EE488AD0E7BDEC048B01
:10DB8000F8BD00BF0000000073B5044653F03AF939
:10DB9000054653F0CDF82046FFF7DCFD4E230093F9
:10DBA00013224D2304212046FFF774F84F2315213B
:10DBB0001322009320465023FFF76CF82046FFF70E
:10DBC00011F92046FFF78CFE4FF400512046F4F780
:10DBD000D3FC10B12046FFF7CFFE04F50056D6F86F
:10DBE0005C0B50B104F5804204F59A43D2F8742DD1
:10DBF00044339A4201D152F06DFB53F02FF852F0AA
:10DC000083FA284653F09CF896F9303B2BB1204616
:10DC100002B0BDE87040FFF7DFBE02B070BD00008B
:10DC200073B5044604F5BC4553F0ECF85C3553F08D
:10DC30007FF8284672F056F904F5A046002866D110
:10DC4000D6F8F833042B04D104F5BB40503075F0FE
:10DC500019F92046FFF748FC04F5804204F59A4381
:10DC6000D2F8742D443304F5C0459A4205F10405F9
:10DC700023D028466FF086FBF8B99FED310A462085
:10DC800052F04EFB9FED2E0A492052F049FB9FEDCA
:10DC90002C0A4A2052F044FB284670F071FC0228FE
:10DCA0000BD10321462052F095FE0321492052F06A
:10DCB00091FE03214A2052F08DFE2046FFF766FCBC
:10DCC0002046FFF7A9FC2046FFF7D2F9204646215F
:10DCD000FEF7CEFE28466FF04BFB90B90190284628
:10DCE00070F04EFC68B102281AD10199462052F01A
:10DCF000DDFD0199492052F0D9FD01994A2052F0E9
:10DD0000D5FD204602B0BDE87040FFF73DBF284674
:10DD1000F8F7AEF896F9663E2B2B91D002B070BDA5
:10DD20009FED070A462052F0FBFA9FED050A4920B5
:10DD300052F0F6FA9FED020A4A2052F0F1FAE0E7BB
:10DD400000000000F6F7A8BE0148FAF7B5BF00BF13
:10DD5000982C002008B5044A0F2343F0A5FA80F060
:10DD60000100C0B208BD00BFC89E0C08F8B500F5A0
